:020000040800F2
:1000000000400220F9800008E7050008F10500081B
:1000100000000000000000000000000000000000E0
:1000200000000000000000000000000005060008BD
:1000300000000000000000000F060008190600087C
:10004000498100080000000049810008498100083A
:100050004981000849810008498100084981000858
:1000600049810008290600084106000865060008C5
:10007000498100084981000849810008000000000A
:10008000498100087D06000849810008498100086F
:100090004981000849810008498100084981000818
:1000A0004981000849810008498100089506000837
:1000B000AD0600084981000810B5064C2378002BD6
:1000C00007D1054B002B02D0044800E000BF0123FC
:1000D000237010BDF0000020000000001C910008FB
:1000E000044B10B5002B03D00349044800E000BFC7
:1000F00010BDC04600000000F40000201C91000864
:1001000003B47146490840004900095E49008E4425
:1001100003BC7047002243088B4274D303098B420F
:100120005FD3030A8B4244D3030B8B4228D3030CC7
:100130008B420DD3FF22090212BA030C8B4202D369
:100140001212090265D0030B8B4219D300E0090A91
:10015000C30B8B4201D3CB03C01A5241830B8B429A
:1001600001D38B03C01A5241430B8B4201D34B0383
:10017000C01A5241030B8B4201D30B03C01A5241E8
:10018000C30A8B4201D3CB02C01A5241830A8B426D
:1001900001D38B02C01A5241430A8B4201D34B0256
:1001A000C01A5241030A8B4201D30B02C01A5241BA
:1001B000CDD2C3098B4201D3CB01C01A524183096E
:1001C0008B4201D38B01C01A524143098B4201D3A8
:1001D0004B01C01A524103098B4201D30B01C01AD3
:1001E0005241C3088B4201D3CB00C01A524183084D
:1001F0008B4201D38B00C01A524143088B4201D37A
:100200004B00C01A5241411A00D2014652411046D9
:100210007047FFE701B5002000F0F0F802BDC046CE
:100220000029F7D076E7704703460B437FD40022BE
:1002300043088B4274D303098B425FD3030A8B427A
:1002400044D3030B8B4228D3030C8B420DD3FF22E4
:10025000090212BA030C8B4202D31212090265D0B2
:10026000030B8B4219D300E0090AC30B8B4201D365
:10027000CB03C01A5241830B8B4201D38B03C01AAC
:100280005241430B8B4201D34B03C01A5241030B23
:100290008B4201D30B03C01A5241C30A8B4201D3D4
:1002A000CB02C01A5241830A8B4201D38B02C01A7F
:1002B0005241430A8B4201D34B02C01A5241030AF6
:1002C0008B4201D30B02C01A5241CDD2C3098B42DB
:1002D00001D3CB01C01A524183098B4201D38B0158
:1002E000C01A524143098B4201D34B01C01A5241FB
:1002F00003098B4201D30B01C01A5241C3088B4240
:1003000001D3CB00C01A524183088B4201D38B002A
:10031000C01A524143088B4201D34B00C01A5241CC
:10032000411A00D201465241104670475DE0CA0FA3
:1003300000D04942031000D34042534000229C4663
:1003400003098B422DD3030A8B4212D3FC2289016D
:1003500012BA030A8B420CD3890192118B4208D343
:10036000890192118B4204D389013AD0921100E0A5
:100370008909C3098B4201D3CB01C01A52418309B9
:100380008B4201D38B01C01A524143098B4201D3E6
:100390004B01C01A524103098B4201D30B01C01A11
:1003A0005241C3088B4201D3CB00C01A524183088B
:1003B0008B4201D38B00C01A5241D9D243088B42E1
:1003C00001D34B00C01A5241411A00D20146634684
:1003D00052415B10104601D34042002B00D54942E8
:1003E000704763465B1000D3404201B5002000F027
:1003F00005F802BD0029F8D016E770477047C046DF
:1004000080B584B000AF7860094B1B68002B02D028
:10041000074B1B6800E0074BFB60391DF8680A2397
:10042000012204F0F5FB7B681800BD4604B080BDD6
:10043000380400209001002080B582B000AF7860C1
:100440007B681B68054A934203D1054B180003F0F3
:10045000EFF9C046BD4602B080BDC0460010004066
:100460003401002080B582B000AF00237B6001F032
:1004700005FF00F057F800F0EDF900F03DFA00F04C
:10048000ADFA00F02FFB00F07BFB00F063FA00F008
:10049000C5FA1E4B180007F083FF1D4B180004F02F
:1004A000C7F801F075FD1B4B180006F0D1FB0300E7
:1004B0007B607B68002B07D07A68174B110018000F
:1004C00007F008FF00F089F807F074F9031E12D155
:1004D000032001F091FD031E10D006F01FFC030065
:1004E0007B607B68002B09D07A680C4B11001800E8
:1004F00007F0F0FE02E0002007F024F9084B180096
:1005000007F04EFF01F0D0FDFCE7C046489100081F
:100510004401002048990008549100087491000893
:100520009091000890B593B000AF10243B191800CB
:1005300038231A00002108F049F83B001800102366
:100540001A00002108F042F880239B00180003F0F5
:100550007FF93B1909221A603B19802252025A6026
:1005600021007B1801229A617B180222DA617B1834
:1005700003221A627B1810225A627B1810229A6298
:100580007B1880229202DA627B18802292041A631E
:100590007B188022D2055A637B18180003F0A4F957
:1005A000031E01D000F019F83B0007221A603B003F
:1005B00002225A603B0000229A603B000022DA606F
:1005C0003B000221180003F0A9FC031E01D000F03B
:1005D00004F8C046BD4613B090BD80B500AF72B6FA
:1005E000C046C046FDE780B500AFC046FDE700004D
:1005F00080B500AF024B180007F0D2FEC046FDE701
:10060000A091000880B500AFC046BD4680BD80B552
:1006100000AFC046BD4680BD80B500AF01F098FE7A
:10062000C046BD4680BD000080B500AF034B18003A
:1006300002F0F8FBC046BD4680BDC046B8020020AF
:1006400080B500AF054B180002F0ECFB044B18001E
:1006500002F0E8FBC046BD4680BDC046180300203E
:10066000D803002080B500AF034B180002F0DAFB7E
:10067000C046BD4680BDC0467803002080B500AFAF
:10068000034B180004F030F8C046BD4680BDC0469C
:100690004401002080B500AF034B180004F010FCAB
:1006A000C046BD4680BDC0469001002080B500AF69
:1006B000034B180004F004FCC046BD4680BDC04694
:1006C0002402002080B582B000AF114B1A6C104B91
:1006D00001210A431A640E4B1B6C012213407B60FC
:1006E0007B680B4BDA6B0A4B802149050A43DA63BE
:1006F000074BDA6B80235B0513403B603B68C023EC
:10070000DB00180001F064FEC046BD4602B080BDAB
:100710000010024080B500AFC046BD4680BD80B528
:1007200086B000AFF860B9607A6000237B610AE0B0
:1007300000E000BF0100BB685A1CBA60CAB21A7060
:100740007B6901337B617A697B689A42F0DB7B6865
:100750001800BD4606B080BD80B586B000AFF86019
:10076000B9607A6000237B6109E0BB685A1CBA60FB
:100770001B781800FFF744FE7B6901337B617A69BF
:100780007B689A42F1DB7B681800BD4606B080BDED
:1007900080B582B000AF786001235B421800BD468F
:1007A00002B080BD80B582B000AF786039603B6830
:1007B000802292015A6000231800BD4602B080BD1D
:1007C00080B582B000AF786001231800BD4602B04A
:1007D00080BD80B584B000AFF860B9607A60002356
:1007E0001800BD4604B080BD80B586B000AF78600B
:1007F000144A154BD31A7B617B693B61134B1B6811
:10080000002B02D1114B124A1A60104B1A687B68F8
:10081000D3183A699A4207D207F02EFF03000C2240
:100820001A6001235B4209E0084B1B68FB60074B21
:100830001A687B68D218054B1A60FB681800BD4621
:1008400006B080BD00400220000800000C0100201E
:1008500048B8002090B589B000AF0C243B191800AF
:1008600014231A00002107F0B1FE214B5A6B204BD4
:1008700020210A435A631E4B5B6B20221340BB604E
:10088000BB681B4B5A6B1A4B01210A435A63184B26
:100890005B6B012213407B607B68154B5A6B144BDA
:1008A00008210A435A63124B5B6B082213403B60DA
:1008B0003B6880239B000F480022190002F048FF8C
:1008C0003B19802292001A603B1901225A603B19A1
:1008D00000229A603B190322DA603B19054A19008D
:1008E000100002F0C9FDC046BD4609B090BDC0462B
:1008F00000100240000C005080B582B000AF144BD5
:100900009A6B134B01210A439A63114B9B6B012293
:1009100013407B607B6800220021092001F01AFE51
:10092000092001F02CFE002200210A2001F012FE15
:100930000A2001F024FE002200210B2001F00AFE13
:100940000B2001F01CFEC046BD4602B080BDC04673
:100950000010024080B500AF0E4B0F4A1A600D4BDD
:1009600000221A710B4B00225A710A4B00225A6165
:10097000084B00229A61074B01221A62054B1800AE
:1009800001F01AFE031E01D0FFF727FEC046BD4648
:1009900080BDC046100100200030024080B584B008
:1009A00000AF78607B681B680A4A93420DD10A4BFE
:1009B0009A6B094B802149010A439A63064B9A6B53
:1009C00080235B011340FB60FB68C046BD4604B05A
:1009D00080BDC046003002400010024080B500AF2C
:1009E0000B4B0C4A1A600A4B03225A60084B0A4A06
:1009F000DA60074B084A9A60054B180002F0C6FE01
:100A0000031E01D0FFF7E9FDC046BD4680BDC046CC
:100A10003401002000300040B80B000080B584B0E5
:100A200000AF3B1D18000C231A00002107F0CEFD7B
:100A3000154B164A1A60144B154A5A60124B002285
:100A40009A60114B134ADA600F4B80229A610E4B69
:100A5000180003F095FD031E01D0FFF7BEFD3B1DFE
:100A600000221A603B1D00229A603A1D064B1100BD
:100A7000180003F0EFFF031E01D0FFF7AEFDC046E4
:100A8000BD4604B080BDC0464401002000100040B7
:100A9000FF180000E703000080B584B000AF786065
:100AA0007B681B680D4A934213D10D4BDA6B0C4BDC
:100AB00010210A43DA630A4BDB6B10221340FB6000
:100AC000FB6800220021112001F044FD112001F0FB
:100AD00056FDC046BD4604B080BDC0460010004073
:100AE0000010024080B500AF234B244A1A60224B0D
:100AF000E12252025A60204B00229A601E4B0022D3
:100B0000DA601D4B00221A611B4B0C225A611A4BF2
:100B100000229A61184B0022DA61174B00221A62F8
:100B2000154B00225A62144B00229A62124B180095
:100B300004F018F8031E01D0FFF74FFD0E4B002103
:100B4000180005F089FB031E01D0FFF746FD0A4B94
:100B50000021180005F0C0FB031E01D0FFF73DFD8A
:100B6000054B180005F03EFB031E01D0FFF735FDD5
:100B7000C046BD4680BDC0469001002000380140FF
:100B800080B500AF234B244A1A60224BE1221203A6
:100B90005A60204B00229A601E4B0022DA601D4BE7
:100BA00000221A611B4B0C225A611A4B00229A61D7
:100BB000184B0022DA61174B00221A62154B0022F3
:100BC0005A62144B00229A62124B180003F0CAFFBB
:100BD000031E01D0FFF701FD0E4B0021180005F0A8
:100BE0003BFB031E01D0FFF7F8FC0A4B0021180065
:100BF00005F072FB031E01D0FFF7EFFC054B180058
:100C000005F0F0FA031E01D0FFF7E7FCC046BD4631
:100C100080BDC046240200200044004090B597B03B
:100C200000AF78604423FB18180014231A00002139
:100C300007F0CCFC18243B1918002C231A000021C3
:100C400007F0C4FC7B681B68A34A934200D09BE07A
:100C50003B1901221A603B1900225A603B19180007
:100C600003F006FB031E01D0FFF7B7FC9B4B1A6C89
:100C70009A4B8021C9010A431A64984B1A6C80234D
:100C8000DB0113407B617B69944B5A6B934B0121D1
:100C90000A435A63914B5B6B012213403B613B69F2
:100CA00044217B18C022D2001A607B1802225A60AD
:100CB0007B1800229A607B180322DA607B180122DD
:100CC0001A617A18A023DB051100180002F0D4FB8A
:100CD000834B844A1A60824B32225A60804B002236
:100CE0009A607F4B0022DA607D4B80221A617C4B38
:100CF00000225A617A4B00229A61794B0022DA6114
:100D0000774B00221A62764B180001F091FE031E09
:100D100001D0FFF762FC7B688021714A5A50704B0A
:100D20007A689A62704B714A1A606F4B33225A602C
:100D30006D4B10229A606C4B0022DA606A4B802265
:100D40001A61694B00225A61674B00229A61664B17
:100D50000022DA61644B00221A62634B180001F032
:100D600067FE031E01D0FFF738FC7B685E4ADA6736
:100D70005D4B7A689A62002200211B2001F0EAFB99
:100D80001B2001F0FCFBA2E07B681B68584A9342E1
:100D900000D09CE018217B1802221A607B180022E8
:100DA0009A607B18180003F063FA031E01D0FFF766
:100DB00014FC4A4BDA6B494B802189020A43DA63FF
:100DC000464BDA6B80239B021340FB60FB68434B6E
:100DD0005A6B424B01210A435A63404B5B6B012221
:100DE0001340BB60BB6844217B180C221A607B183F
:100DF00002225A607B1800229A607B180322DA6074
:100E00007B1801221A617A18A023DB051100180053
:100E100002F032FB374B384A1A60364B34225A60A4
:100E2000344B00229A60334B0022DA60314B80222F
:100E30001A61304B00225A612E4B00229A612D4BD1
:100E40000022DA612B4B802292011A62294B180092
:100E500001F0EEFD031E01D0FFF7BFFB7B68802190
:100E6000244A5A50234B7A689A62244B244A1A60C7
:100E7000224B35225A60214B10229A601F4B0022D0
:100E8000DA601E4B80221A611C4B00225A611B4BF8
:100E900000229A61194B0022DA61184B80229201DC
:100EA0001A62164B180001F0C3FD031E01D0FFF7B4
:100EB00094FB7B68114ADA67104B7A689A620022C9
:100EC00000211C2001F046FB1C2001F058FBC0460D
:100ED000BD4617B090BDC04600380140001002402A
:100EE000B802002008000240180300201C00024045
:100EF000004400407803002044000240D803002052
:100F00003000024080B500AFBFF34F8FC046044BA6
:100F1000044ADA60BFF34F8FC046C046FDE7C046C3
:100F200000ED00E00400FA0580B584B000AF786001
:100F30000A00BB1C1A800E23FB1800221A8021E035
:100F40000E23FB181B887A68D2180D217B181278A3
:100F50001A700A00BB181B78012B0BD0BB181B782A
:100F6000022B07D0BB181B78042B03D0BB181B78AF
:100F7000182B01D101230DE00E217B181A887B1854
:100F800001321A800E23FA18BB1C12881B889A4261
:100F9000D6D300231800BD4604B080BD80B584B010
:100FA00000AF78600A00BB1C1A800E23FB180022D9
:100FB0001A800C23FB1800221A8034E00C23FB1843
:100FC0001B887A68D3181B781BB21B021AB20E2139
:100FD0007B1800201B5E53401AB27B181A80002336
:100FE000BB6017E00E217B1800229B5E002B08DA05
:100FF0007B181B88DB189AB27B1812494A401A806A
:1010000005E00E23FA18FB181B88DB181380BB6859
:101010000133BB60BB68072BE4DD0C217B181A8809
:101020007B1801321A800C23FA18BB1C12881B880B
:101030009A42C3D30E23FB181B881800BD4604B088
:1010400080BDC0462110000080B582B000AF78603E
:101050000A00FB1C1A707B68002B06D0F91C78680C
:101060003223012203F0D4FD00E0C046BD4602B0A9
:1010700080BD000080B500AF044B1B68062118003E
:10108000FFF7E2FFC046BD4680BDC04684B40020E5
:1010900080B500AF044B1B6815211800FFF7D4FF83
:1010A000C046BD4680BDC04684B4002080B584B033
:1010B00000AF78607B68002B18D001F05BF903006B
:1010C000FB6006E001F056F90200FB68D31A282BFA
:1010D00007D87B681B68DB6940221340402BF1D1A5
:1010E00000E0C0460A2001F04FF900E0C046BD46CE
:1010F00004B080BD80B584B000AF78607B68002B01
:1011000019D00F23FB1800221A700AE07B681821FF
:101110001800FFF799FF0F217B181A787B1801320E
:101120001A700F23FB181B78072BEFD97B68180068
:10113000FFF7BCFF00E0C046BD4604B080BD000024
:1011400080B582B000AF0200FB1D1A70FB1D1B783A
:10115000002B01D1034B00E0034B1800BD4602B049
:1011600080BDC046900100202402002080B500AF61
:10117000034B1B681800FFF7BDFFC046BD4680BD8E
:1011800084B4002080B582B000AFFB1D43221A70EA
:101190000F4B1B68002B0CD1F91D0E483223012286
:1011A00003F036FDF91D0C483223012203F030FD17
:1011B0000AE00A4B1B68002B06D0084B1868F91D83
:1011C0003223012203F024FDC046BD4602B080BD9B
:1011D0008CB40020900100202402002084B4002060
:1011E00080B500AF0A4B1A680A4B9A4204D10A4BE9
:1011F000180003F0B1FD08E0054B1A68064B9A424F
:1012000003D1044B180003F0A7FDC046BD4680BDC6
:1012100084B40020900100202402002080B582B018
:1012200000AF7860396080231A0139687B68180044
:1012300005F094F8031E0AD07B68180003F08CFDBB
:1012400080231A0139687B68180005F087F8C046CA
:10125000BD4602B080BD000080B500AF114B00223A
:101260001A60114B00221A60104B114A1A600F4B82
:101270001A68104B1A600E4B180003F06DFD0E4BF0
:10128000180003F069FD0D4A094B11001800FFF723
:10129000C5FF0B4A084B11001800FFF7BFFFC046FF
:1012A000BD4680BD8CB4002084B4002088B40020EA
:1012B0009001002038040020240200203C0400207B
:1012C0003C0C002080B582B000AF0200FB1D1A70FC
:1012D0000E4B1B68002B01D1012312E0FB1D1B7874
:1012E000002B07D10A4B1A680A4BD31A5A425341B2
:1012F000DBB206E0064B1A68074BD31A5A42534139
:10130000DBB21800BD4602B080BDC0468CB40020E0
:1013100084B40020900100202402002080B584B015
:1013200000AF39601100FB1D021C1A703B1D0A1C26
:101330001A80294B1B78DBB20133DAB20F203B183D
:101340000F210A401A70254B1B78DBB23A1812782D
:101350009A4202D101235B423AE01F4B1B78DBB279
:1013600019001F4A0B005B025B189B00F91D0978EE
:101370009954194B1B78DBB21900194A0B005B0218
:101380005B189B00D31802333A1D12881A803B1D4C
:101390001A8880231B019A4203D93B1D8022120127
:1013A0001A800D4B1B78DBB21A0013005B029B18EE
:1013B0009B000B4A9B18181D3B1D1A883B6819009F
:1013C00007F087F9044B0F22BA1812781A7000231D
:1013D0001800BD4604B080BD7C9400207D940020A0
:1013E0003C14002080B500AF054B1B68002B04D0D7
:1013F00006F028F9024B00221A60C046BD4680BDA7
:10140000ECB4002080B500AF1C4B00221A801B4BAF
:1014100000225A8080239A01194B0021180007F0FE
:10142000D5F8184B00221A60174B00221A70174B80
:10143000FF221A70164B00221A60164B3822002128
:10144000180007F0C3F8144B00221A80134B002237
:101450001A60134B00221A60124B00221A60124BC2
:1014600000221A70114B00221A70114B00221A70C0
:10147000FFF7B8FFC046BD4680BDC04680B400201F
:101480008094002098B400209CB400209DB40020DB
:10149000A0B40020A4B40020DCB40020E0B40020FC
:1014A000E4B40020E8B40020F0B40020F1B400203F
:1014B000F2B4002080B582B000AF78607B68002B6A
:1014C00001D07B6800E0174B174A1900100006F0A6
:1014D00001FFFFF787FFFFF795FF144B00221A600B
:1014E000134B00221A60134B134A1A6000F042FF9C
:1014F0000200124B1A60114B1A68114B1A60114B03
:1015000000221A70104B00221A70104B00221A7021
:101510000F4B00221A70FFF79FFEC046BD4602B077
:1015200080BDC046AC910008B09100088CB400208A
:1015300084B40020380400209001002094B40020DE
:1015400090B400207D9400207C9400207E940020A4
:101550007F94002080B582B000AF0200FB1D1A709E
:10156000164B01221A60FB1D1B78002B09D1144B6E
:10157000144A1A60144B154A1A60154B00225A80FF
:1015800008E00F4B114A1A600F4B0E4A1A60104BBD
:1015900000221A800C4B1A680E4B1A600E4B002268
:1015A0001A700E4B01221A600D4B00221A60FFF7D1
:1015B00017FEC046BD4602B080BDC0468CB40020B8
:1015C00084B400209001002088B400202402002070
:1015D00080B40020380400209CB4002098B400207F
:1015E000A0B40020B0B594B000AF78600A00BB1C76
:1015F0001A804E23FB1800221A80BDE0654B1B6841
:10160000002B00D072E0644B1A8844203B1838212C
:101610008A1A1A80BB1C1A884E217B181B88D21A82
:101620003B181B889A4206DABA1C7B1812881B8862
:10163000D31A9BB202E04423FB181B8842243A19B8
:101640001380554B1B881A00544BD0184E257B191C
:101650001B887A68D1183B191B881A0007F039F8E3
:101660004D4B1A8820003B191B88D3189AB24A4B5D
:101670001A807B1979193A18098812888A181A80F1
:10168000454B1B88372B00D876E008243A19434B8A
:101690001000190038231A0007F01BF83B19180036
:1016A00005F060FC031E03D03D4B14221A706DE060
:1016B0003C4B01221A60394B38221900002005F0FA
:1016C0001FFE031E03D0364B14221A705EE0314B0E
:1016D00001221A60344B38221A6008217B189A685C
:1016E0007B18DB68D218314B1A6045E02F4B1A6823
:1016F0002D4B1B689A4206D32C4B1A682A4B1B6849
:10170000D31ABB6401E00023BB64BB6C002B3CD04C
:1017100046203B18B91C4E22BA18098812888A1A2A
:101720001A803B181B88BA6C9A4202D23B18BA6CDA
:101730001A801D4B18684E23FB181B887A68D11835
:101740004623FB181B881A0005F0DAFD031E03D0A0
:10175000134B14221A7019E046203B181A88124BBA
:101760001B68D218104B1A604E22BB18B9183A18D1
:10177000098812888A181A804E23FA18BB1C12880E
:101780001B889A4200D239E700E0C046BD4614B03B
:10179000B0BDC046E0B40020DCB40020A4B40020FA
:1017A000F2B40020ECB40020E4B40020E8B400203F
:1017B00080B584B000AF0200FB1D1A703C4B1B6863
:1017C000002B03D03B4B1B68002B01D100236AE0A8
:1017D000394B1B68002B06D1FFF75AFC364B012210
:1017E0001A6000235FE0344B1B68012B01DD0023EE
:1017F00059E0314B02221A60FFF73CFC2D4B1B686D
:101800001800FFF753FCFFF7BDFC0F2000F0BCFDF4
:1018100000F042FBFB1D1B78180000F0D1F8254BAF
:101820001B684F211800FFF70FFC224B1B681800A4
:10183000FFF73CFC214B00221A70214B01221A7049
:1018400000F02AFBFB1D1B78180000F0B9F81D4BB7
:101850001B68002B22D01C4B1B68002B1ED005F0F0
:1018600021FE0300FB60FB68002B0CD1174B180016
:1018700006F096FD002005F065FF124B00221A606D
:1018800005F04CFA0AE0FA68114B1100180006F056
:1018900021FD05F0D7FE0B4B00221A600D4B1800FE
:1018A000FFF708FE01231800BD4604B080BDC04606
:1018B0008CB4002084B40020A0B40020F0B4002038
:1018C000F1B40020ECB40020E0B40020C491000882
:1018D000DC910008F091000880B582B000AF39605B
:1018E0001100FB1D021C1A703B1D0A1C1A802E4B96
:1018F0001B78FA1D12789A421BD02C4B1B78FA1DCC
:1019000012789A4202D1FFF7B5FB49E0FFF7C0FB1E
:10191000274B1B780133DAB2254B1A70244B1B7806
:10192000142B3CD9FFF722FC224B1800FFF7C2FD15
:1019300035E0214B1B68002B0FD01F4B00221A6093
:10194000194B01221A70194BFA1D12781A70FFF701
:1019500091FB174B00221A7022E03B1D1A883B684E
:1019600011001800FFF73EFE114B1B78132B06D910
:10197000FFF7FCFB114B1800FFF79CFD10E00B4B31
:10198000FA1D12781A70FB1D1B780133DAB2064B70
:101990001A70FFF76FFB064B00221A7000E0C0467A
:1019A000BD4602B080BDC0469CB400209DB400205E
:1019B000F2B40020F491000898B40020F8910008D7
:1019C000F0B58BB000AF0200FB1D1A70FB1D1B7839
:1019D0001A03B64BD3183B62FB1D1B785A00B44B5D
:1019E000D318FB61E5E12623FB1800221A8005E0ED
:1019F00026217B181A887B1801321A80FB691B8804
:101A000026217A1812889A421BD27B181B883A6AC0
:101A1000D3181B78012B14D07B181B883A6AD31873
:101A20001B78022B0DD07B181B883A6AD3181B78C1
:101A3000042B06D07B181B883A6AD3181B78182B06
:101A4000D6D126243B191B88002B16D03B191B88A6
:101A50003A6AD118FB691B881A003B191B88D31AF4
:101A60001A003B6A180006F09FFDFB691A883B19B3
:101A70001B88D31A9AB2FB691A80FB691B88002B5A
:101A800000D19CE18B4B1B68002B15D0FB1D1B78F4
:101A9000002B04D1884B1A68884B9A4208D1FB1D51
:101AA0001B78012B08D1844B1A68854B9A4203D0CE
:101AB000FB6900221A8087E13B6A1B78182B32D120
:101AC000804B1B78002B0FD03B6A591CFB691B888D
:101AD0005A1E3B6A180006F067FDFB691B88013B34
:101AE0009AB2FB691A8064E1774B1B780133DAB252
:101AF000754B1A703B6A591CFB691B885A1E3B6A5E
:101B0000180006F051FDFB691B88013B9AB2FB6986
:101B10001A806D4B1B78012B00D843E16B4B1800EA
:101B2000FFF7C8FC3EE1684B00221A703B6A1B7845
:101B3000042B19D13B6A591CFB691B885A1E3B6A4E
:101B4000180006F031FDFB691B88013B9AB2FB6966
:101B50001A805C4B1B78002B00D025E1FB1D1B7805
:101B60001800FFF725FE24E13B6A1B78012B04D007
:101B70003B6A1B78022B00D023E11B217B183A6AB9
:101B800012781A707B181B78012B01D1802201E09A
:101B90008023DA0018217B181A8016203B187A1847
:101BA000128805321A80FB691B883A1812889A42FB
:101BB00000D908E115217B183A6A52781A7014206E
:101BC0003B183A6A92781A707A183B1812781B7888
:101BD000D318DBB2FF2B16D03B6A591CFB691B885C
:101BE0005A1E3B6A180006F0DFFCFB691B88013BAC
:101BF0009AB2FB691A802F4B1B68002B00D1D5E0ED
:101C0000FFF746FAD2E03B6A03333B6118203B18EA
:101C10001B8803333A6AD3181B781BB21B021AB213
:101C20003B181B880433396ACB181B781BB213434B
:101C30001AB20E257B191A800C26BC193B181A887B
:101C40003B6911001800FFF7A9F9030023807A19F6
:101C5000BB1912881B889A423ED03B6A591CFB690B
:101C60001B885A1E3B6A180006F09EFCFB691B8805
:101C7000013B9AB2FB691A800E4B1B68002B00D106
:101C800096E0FFF705FA124B1B780133DAB2104BDE
:101C90001A700F4B1B78142B00D889E0FFF766FAF7
:101CA0000C4B1800FFF706FC82E0C0468094002031
:101CB00080B400208CB4002084B400209001002067
:101CC00024020020F1B40020F0B4002000920008AB
:101CD000F2B40020049200081B23FB181B78012B90
:101CE00034D11523FB181B78002B2FD13B691B78AF
:101CF000002B2BD1364B1B68002B27D0354B1B6894
:101D0000012B23DD344B1B68002B04D1FB1D1B78FA
:101D10001800FFF71FFCFFF7ADF916243B191B88CD
:101D20003A6AD118FB691B881A003B191B88D31A21
:101D30001A003B6A180006F037FCFB691A883B1949
:101D40001B88D31A9AB2FB691A8032E0224B1B68B7
:101D5000002B04D1FB1D1B781800FFF7FBFB182399
:101D6000FB181A8839691523FB181B781800FFF730
:101D7000B3FD16243B191B883A6AD118FB691B88EE
:101D80001A003B191B88D31A1A003B6A180006F088
:101D90000BFCFB691A883B191B88D31A9AB2FB69A2
:101DA0001A8006E0C04604E0C04602E0C04600E0FB
:101DB000C046FB691B88002B00D014E604E0C04637
:101DC00002E0C04600E0C046BD460BB0F0BDC046D4
:101DD000E0B40020A0B400208CB4002080B584B012
:101DE00000AF39601100FB1D021C1A703B1D0A1C5C
:101DF0001A80FB1D1A78244B5200D35A1A003B1D3F
:101E00001B88D21880235B019A4216D91F4B1B688E
:101E1000002B06D1FB1D1B781800FFF791F903007A
:101E200001E01A4B1B68FB60FB681800FFF762F9C2
:101E3000174B1800FFF73EFB23E0FB1D1B781A032E
:101E4000144BD318FA1D11780F4A49008A5A981872
:101E50003B1D1A883B68190006F03BFCFB1D1A78F5
:101E6000094B5200D15AFB1D1A783B1D1B88CB1819
:101E700099B2054B5200D152FB1D1B781800FFF799
:101E80009FFDBD4604B080BD80B4002084B4002016
:101E9000089200088094002090B5314CA54400AF12
:101EA000304B1B78DBB2002B4ED02F4B1B68002B26
:101EB00007D12E4B1B78DBB21800FFF741F9030066
:101EC00001E0294B1B682A4AB9180B60BB181B6834
:101ED0001800FFF70FF9274B1800FFF7EBFA3BE06C
:101EE000254B1B78DBB21900244B254C1B19D81944
:101EF000244A0B005B025B189B00D3181C4A190094
:101F000006F0E7FB1C4B1B78DBB20133DBB20F2280
:101F10001340DAB2184B1A70184B1B19DB191B78D7
:101F20001800FFF7CFF9031E0DD0144B1B19DB1956
:101F30001878124B1B19DB195A883B00043319001F
:101F4000FFF74CFF00E0C0460B4B1B78DAB20E4B9C
:101F50001B78DBB29A42C3D1BD460C4B9D4490BD69
:101F6000F4F7FFFF7E94002084B400207F940020CB
:101F700004080000149200087D940020F8F7FFFF89
:101F8000080800003C1400207C9400200C0800008D
:101F900080B500AF104B114A1A60FFF733FA0021E9
:101FA0000F4B0A1C1A700F4B0A1C1A700E4B0022A2
:101FB0001A700E4B00221A7000F0DCF902000C4B74
:101FC0001A600B4B1A680B4B1A60FFF745F9FFF7C5
:101FD000D9F8C046BD4680BD3804002090010020DD
:101FE0007C9400207D9400207E9400207F9400202B
:101FF00094B4002090B4002080B586B000AF786023
:102000007B68002B02D101235B4240E064233B61EB
:1020100000237B612BE0FFF7B5F800F0ABF902007D
:102020001D4B1A6000F0A6F90300BB6014E0FFF737
:1020300033FF1A4B1B68002B01D0002327E0184BFD
:102040001B88002B03D1164B5B88002B01D000238B
:102050001DE0012000F098F900F08CF90200BB6847
:10206000D31A3A699A42E2D87B6901337B617A6973
:102070007B689A42CFD300F07DF90300FB60094BE7
:10208000FA681A60044BFA681A6001235B42180070
:10209000BD4606B080BDC04694B400208CB400207C
:1020A00080B4002090B4002080B582B000AFFFF76C
:1020B000F3FE00F05FF903007B60194B1B687A6840
:1020C000D31AC72B08D9174B1B68002B01D1FFF778
:1020D00059F8134B7A681A60134B1B687A68D31A45
:1020E0003B603B68002B17DB3B68104A934213D9D7
:1020F0000C4B1B68002B01D0FFF738F804F000FFF1
:10210000031E05D00A4B180006F04AF9FEF7FAFE46
:10211000084B1800FFF7CEF9C046BD4602B080BD9F
:1021200094B400208CB4002090B40020B70B0000C1
:10213000209200083492000890B585B000AF786016
:102140000A00BB1C1A807A68314BD31A5A1E93417D
:10215000DAB20F217B181A707B181B78002B01D183
:102160002C4B00E02C4BBB60BB1C1A8880231B014E
:102170009A4203D9BB1C802212011A80BB1C1B8807
:10218000002B15D0BB1C1A88BB6811001800FEF785
:10219000CBFE031E07D10F23FB181B781800FFF797
:1021A00091F8031E04D000F0E5F802001B4B1A6002
:1021B0000F23FB181B781800FFF784F8031E06D1C5
:1021C000BA687B6811001800FFF728F81CE0BB1CF8
:1021D0001A88B9680F243B191B781800FFF79EF87E
:1021E000031E0BD00E4B3A1912781A700D4B0122B8
:1021F0001A707B68180002F0AFFD05E0BA687B68D2
:1022000011001800FFF70AF8BD4605B090BDC046A2
:10221000900100203C0400203C0C002090B40020E1
:102220007F9400207E94002080B584B000AF786059
:102230007B681B680F221A627A680D4BD31A5A1EEC
:102240009341DAB20F217B181A707B181B78002B90
:1022500001D1084B00E0084BBB60BA687B681100F5
:102260001800FEF7DBFFC046BD4604B080BDC04687
:10227000900100203C0400203C0C002080B582B07E
:1022800000AFFB1D00221A700B4B1A680A4B80210D
:1022900049000A431A60032000F010F8031E03D01F
:1022A000FB1D01221A7001E0FEF70CFAFB1D1B78E2
:1022B0001800BD4602B080BD0020024090B585B038
:1022C00000AF78600F23FB1800221A701D4B1B789B
:1022D000002B2BD01C4B1C681A4B1B781900FA23BF
:1022E0009800FDF717FF030019002000FDF712FF0B
:1022F0000300180000F053F9031E12D17B68032B72
:102300000AD8796801235B420022180000F022F904
:102310000E4B7A681A600DE00F23FB1801221A7029
:1023200008E00F23FB1801221A7003E00F23FB18AB
:1023300001221A700F23FB181B781800BD4605B048
:1023400090BDC046080000200000002004000020CE
:1023500080B500AF054B1B781A00054B1B68D218DF
:10236000034B1A60C046BD4680BDC0460800002031
:10237000F4B4002080B500AF024B1B681800BD46C6
:1023800080BDC046F4B4002080B584B000AF786052
:10239000FFF7F0FF0300BB607B68FB60FB68013365
:1023A00005D00A4B1B781A00FB689B18FB60C046DF
:1023B000FFF7E0FF0200BB68D31AFA689A42F7D829
:1023C000C046C046BD4604B080BDC04608000020DF
:1023D00080B582B000AF7860064B1B68064A134098
:1023E0001900044B7A680A431A60C046BD4602B021
:1023F00080BDC04600000140FFF9FFFF80B582B0FC
:1024000000AF0200FB1D1A70FB1D1B787F2B09D843
:10241000FB1D1B781A001F231A40044B0121914019
:102420000A001A60C046BD4602B080BD00E100E06F
:1024300090B583B000AF02003960FB1D1A70FB1D20
:102440001B787F2B28D82F4AFB1D1B785BB29B087B
:10245000C0339B009B58FA1D1278110003220A40DA
:10246000D200FF2191400A00D2431A4011003B687C
:102470009B01FF221A40FB1D1B7818000323034019
:10248000DB009A401F48FB1D1B785BB29B080A4388
:10249000C0339B001A5031E01B4AFB1D1B7819000A
:1024A0000F230B40083B9B0806339B00D3180433D3
:1024B0001B68FA1D1278110003220A40D200FF2186
:1024C00091400A00D2431A4011003B689B01FF2251
:1024D0001A40FB1D1B78180003230340DB009A40C1
:1024E0000948FB1D1B781C000F232340083B9B0859
:1024F0000A4306339B00C31804331A60C046BD4626
:1025000003B090BD00E100E000ED00E080B582B0D6
:1025100000AF78607B685A1E80235B049A4201D327
:10252000012310E00A4B7A68013A5A6001235B42AA
:1025300003211800FFF77CFF054B00229A60044B33
:1025400007221A6000231800BD4602B080BDC046B5
:1025500010E000E080B584B000AFB9607A600F2170
:102560007B18021C1A70BA687B181B785BB21100CA
:102570001800FFF75DFFC046BD4604B080BD80B5C2
:1025800082B000AF0200FB1D1A70FB1D1B785BB20E
:102590001800FFF733FFC046BD4602B080BD80B5CE
:1025A00082B000AF78607B681800FFF7AFFF0300D0
:1025B0001800BD4602B080BD80B582B000AF786023
:1025C0007B68002B01D1012356E07B685B7FDBB287
:1025D000002B06D17B6800221A777B681800FEF773
:1025E000DDF97B6802225A777B681B79002B0CD1BE
:1025F0007B681B68224A5A617B681B689A687B6803
:102600001B6818218A439A600BE07B6899687B6895
:10261000DA687B68180000F095F9031E01D00123E9
:102620002AE07B685B79002B05D17B681B6801225F
:1026300052421A6104E07B681B687A6812691A6169
:102640007B681B689B686022934319007B685A690A
:102650007B681B680A439A607B681B689B688022C2
:10266000934319007B689A697B681B680A439A60E8
:102670007B6801225A7700231800BD4602B080BD56
:10268000B71DC10480B586B000AFF860B9607A604C
:1026900000233B61FB6802225A77FB681B6A032B0D
:1026A00005D02DD8012B19D0022B20D028E00023F3
:1026B0007B610AE07B699B00BA68D218FB681B68E3
:1026C00012681A607B6901337B617A697B689A4280
:1026D000F0D3FB681B681B683B6112E07A68B9683D
:1026E000FB68180000F064F803003B6109E07A68B9
:1026F000B968FB68180000F0EEF803003B6100E0E9
:10270000C046FB6801225A773B691800BD4606B0F7
:1027100080BD80B586B000AFF860B9607A600023F4
:102720003B61FB6802225A77FB681B689A68FB686A
:102730001B6801210A439A60FB681B6A032B05D0C2
:102740002DD8012B19D0022B20D028E000237B614B
:102750000AE07B699B00BA68D218FB681B681268A4
:102760001A607B6901337B617A697B689A42F0D396
:10277000FB681B681B683B6112E07A68B968FB68FC
:10278000180000F015F803003B6109E07A68B968A9
:10279000FB68180000F09FF803003B6100E0C046B2
:1027A000FB6801225A773B691800BD4606B080BD20
:1027B00080B588B000AFF860B9607A600023FB6133
:1027C00023E0FB699B00BA68D3181B781A06FB69E3
:1027D0009B000133B968CB181B781B041A43FB69B3
:1027E0009B000233B968CB181B781B021A43FB69A4
:1027F0009B000333B968CB181B781900FB681B6872
:102800000A431A60FB690133FB617B689B08FA6924
:102810009A42D6D37B680322134055D07B680322AB
:102820001340012B07D1FB699B00BA68D218FB68E3
:102830001B6812781A707B6803221340022B1AD18E
:10284000FB699B00BA68D3181B781BB21B021AB233
:10285000FB699B000133B968CB181B781BB213438B
:102860001AB21A217B181A80FB681B687B617B698E
:102870007A1812881A807B6803221340032B23D115
:10288000FB699B00BA68D3181B781BB21B021AB2F3
:10289000FB699B000133B968CB181B781BB213434B
:1028A0001AB21A217B181A80FB681B687B617B694E
:1028B0007A1812881A80FB699B000233BA68D21812
:1028C000FB681B6812781A70FB681B681B6818008D
:1028D000BD4608B080BD80B586B000AFF860B96075
:1028E0007A6000237B6113E07B699B00BA68D31890
:1028F0001B881A047B699B000233B968CB181B88BC
:102900001900FB681B680A431A607B6901337B610D
:102910007B685B087A699A42E6D37B6801221340A0
:1029200009D0FB681B683B617B699B00BA68D318C0
:102930001A883B691A80FB681B681B681800BD4633
:1029400006B080BD80B586B000AFF860B9607A602F
:1029500017217B1800221A701F233B61BB680122DC
:10296000134003D17B1801221A7045E0C0463B6931
:102970005A1E3A61002B08D03B691F221340BA68E7
:10298000DA40130001221340F1D07B68182B0FD0DE
:102990007B68182B24D87B68102B11D07B68102BF8
:1029A0001ED87B68002B20D07B68082B10D017E046
:1029B0003B69062B1BD91723FB1801221A7016E05E
:1029C0003B69072B15D91723FB1801221A7010E059
:1029D0003B690F2B0FD91723FB1801221A700AE04D
:1029E0001723FB1801221A7006E0C04604E0C04617
:1029F00002E0C04600E0C0461723FB181B78002BFE
:102A00000ED1FB681B68BA685A61FB681B689B683B
:102A1000182293431900FB681B687A680A439A607E
:102A20001723FB181B781800BD4606B080BD0000B8
:102A300080B582B000AF78607B68002B01D10123A4
:102A400091E07B681B681A00494B9A4210D87B685A
:102A50001B68484A9446634414211800FDF75AFB4A
:102A600003009A007B685A647B68434A1A640FE04B
:102A70007B681B68414A9446634414211800FDF7A3
:102A800049FB03009A007B685A647B683C4A1A64DD
:102A90007B682522022199547B681B681A687B6831
:102AA0001B6838490A401A607B681B6819687B6894
:102AB0009A687B68DB681A437B681B691A437B68EA
:102AC0005B691A437B689B691A437B68DB691A431D
:102AD0007B681B6A1A437B681B680A431A607B6821
:102AE000180000F0A9FA7B689A688023DB019A42FB
:102AF00002D17B6800225A607B685A687B689B6CB5
:102B00007F210A401A607B68DB6C7A68126D5A601C
:102B10007B685B68002B11D07B685B68042B0DD849
:102B20007B68180000F0D2FA7B685B6D00221A60A7
:102B30007B689B6D7A68D26D5A6008E07B680022E2
:102B40005A657B6800229A657B680022DA657B689B
:102B50000022DA637B682522012199547B682422B4
:102B60000021995400231800BD4602B080BDC04624
:102B700007040240F8FFFDBF00000240F8FBFDBF64
:102B8000000402400F80FFFF80B586B000AFF86000
:102B9000B9607A603B601723FB1800221A70FB684B
:102BA00024229B5C012B01D102236FE0FB682422CD
:102BB00001219954FB6825229B5CDBB2012B57D184
:102BC000FB68252202219954FB680022DA63FB6826
:102BD0001B681A68FB681B6801218A431A603B68FE
:102BE0007A68B968F86800F0EBF9FB681B6B002B9A
:102BF00008D0FB681B681A68FB681B680E210A4333
:102C00001A600FE0FB681B681A68FB681B680421E8
:102C10008A431A60FB681B681A68FB681B680A21F4
:102C20000A431A60FB689B6C1A6880235B0213409E
:102C300008D0FB689B6C1A68FB689B6C802149007C
:102C40000A431A60FB685B6D002B08D0FB685B6D64
:102C50001A68FB685B6D802149000A431A60FB68B3
:102C60001B681A68FB681B6801210A431A600AE0A6
:102C7000FB688022DA63FB68242200219954172321
:102C8000FB1801221A701723FB181B781800BD4689
:102C900006B080BD80B582B000AF78607B68002B45
:102CA00001D101234FE07B6825229B5CDBB2022B24
:102CB00008D07B680422DA637B68242200219954BF
:102CC000012340E07B681B681A687B681B680E2143
:102CD0008A431A607B689B6C1A687B689B6C1C49F2
:102CE0000A401A607B681B681A687B681B680121B0
:102CF0008A431A607B685B6C1C221A407B681B6CE1
:102D0000012191400A005A607B68DB6C7A68126D81
:102D10005A607B685B6D002B0CD07B685B6D1A681A
:102D20007B685B6D0A490A401A607B689B6D7A6814
:102D3000D26D5A607B682522012199547B68242238
:102D40000021995400231800BD4602B080BDC04642
:102D5000FFFEFFFF80B584B000AF78600F217B18C5
:102D600000221A707B6825229B5CDBB2022B06D006
:102D70007B680422DA637B1801221A7048E07B68C2
:102D80001B681A687B681B680E218A431A607B687F
:102D90001B681A687B681B6801218A431A607B687C
:102DA0009B6C1A687B689B6C1D490A401A607B68A3
:102DB0005B6C1C221A407B681B6C012191400A004D
:102DC0005A607B68DB6C7A68126D5A607B685B6D59
:102DD000002B0CD07B685B6D1A687B685B6D1049BB
:102DE0000A401A607B689B6D7A68D26D5A607B6876
:102DF0002522012199547B682422002199547B6863
:102E00009B6B002B04D07B689B6B7A681000984703
:102E10000F23FB181B781800BD4604B080BDC046C8
:102E2000FFFEFFFF80B584B000AF78607B681B6C4D
:102E30001B68FB607B681B681B68BB607B685B6C06
:102E40001C22134004229A401300FA68134026D033
:102E5000BB680422134022D07B681B681B682022B9
:102E6000134007D17B681B681A687B681B680421C4
:102E70008A431A607B685B6C1C221A407B681B6C5F
:102E8000042191400A005A607B681B6B002B00D123
:102E900080E07B681B6B7A68100098477AE07B685B
:102EA0005B6C1C22134002229A401300FA68134004
:102EB0003CD0BB680222134038D07B681B681B687B
:102EC000202213400BD17B681B681A687B681B6843
:102ED0000A218A431A607B682522012199547B6864
:102EE0001B681A002E4B9A4209D97B685B6C1C2226
:102EF0001A402C4B022191400A005A6008E07B687E
:102F00005B6C1C221A40284B022191400A005A6037
:102F10007B682422002199547B68DB6A002B39D01E
:102F20007B68DB6A7A681000984733E07B685B6CEB
:102F30001C22134008229A401300FA6813402AD03A
:102F4000BB680822134026D07B681B681A687B6820
:102F50001B680E218A431A607B685B6C1C221A4036
:102F60007B681B6C012191400A005A607B6801223A
:102F7000DA637B682522012199547B682422002191
:102F800099547B685B6B002B05D07B685B6B7A6820
:102F900010009847C046C046BD4604B080BDC0463C
:102FA00080000240000402400000024080B582B070
:102FB00000AF78607B68DB6B1800BD4602B080BD57
:102FC00080B584B000AFF860B9607A603B60FB68A0
:102FD000DB6CFA68126D5A60FB685B6D002B04D0E5
:102FE000FB689B6DFA68D26D5A60FB685B6C1C22B3
:102FF0001A40FB681B6C012191400A005A60FB6873
:103000001B683A685A60FB689B68102B08D1FB6804
:103010001B687A689A60FB681B68BA68DA6007E028
:10302000FB681B68BA689A60FB681B687A68DA609C
:10303000C046BD4604B080BD80B584B000AF7860A6
:103040007B681B681A001D4B9A4214D87B685B6C26
:103050009B089B001A4A9A187B689A647B681B68D5
:103060001A00FF231340083B14211800FDF752F803
:103070000300FB6014E07B685B6C9B089B00114ABB
:103080009A187B689A647B681B681A00FF231340B8
:10309000083B14211800FDF73DF803000733FB60DF
:1030A0007B68094ADA64FB681F22134001229A40B8
:1030B0007B681A65C046BD4604B080BD0704024067
:1030C000000802401C0802408008024080B584B01D
:1030D00000AF78607B685B687F221340FB60FB6811
:1030E0000A4A944663449B001A007B685A657B68D1
:1030F000074A9A65FB68013B0322134001229A406C
:103100007B68DA65C046BD4604B080BD3F820010D2
:1031100040090240B0B586B000AFF860B9603A60CF
:103120007B60214B1B78012B01D1022338E01E4B21
:1031300001221A701C4B00225A6017257C19FA23B1
:103140009B00180000F07AF8030023707B191B78AD
:10315000002B1FD1FB68012B06D13A687B68B96848
:10316000080000F0B9F805E03A68BB6811001800E3
:1031700005F0E2FF1723FC18FA239B00180000F06B
:103180005DF803002370094B5A69FB68D943074B6C
:103190000A405A61044B00221A701723FB181B784F
:1031A0001800BD4606B0B0BDF8B4002000200240B3
:1031B00080B582B000AFFB1D00221A700B4B5B691B
:1031C000002B0CDA094B0A4A9A60084B094A9A60AC
:1031D000064B5B69002B02DAFB1D01221A70FB1DF6
:1031E0001B781800BD4602B080BDC04600200240DA
:1031F00023016745AB89EFCD80B582B000AFFB1DE1
:1032000001221A70FA239B00180000F017F80A4BED
:103210005A69094B802109060A435A61064B5B69CA
:10322000002B02DAFB1D00221A70FB1D1B78180010
:10323000BD4602B080BDC0460020024080B584B0CB
:1032400000AF7860FFF796F80300FB60C0239B0295
:10325000BB600CE07B68013309D0FFF78BF80200FC
:10326000FB68D31A7A689A4201D8032328E0164BE8
:103270001B69BA681340EDD1134B1B69134A134005
:10328000BB60114B124A1A61BB68002B11D0114B65
:10329000BA685A60012313E07B68013309D0FFF755
:1032A00069F80200FB68D31A7A689A4201D80323AE
:1032B00006E0054B1A698023DB021340ECD10023A2
:1032C0001800BD4604B080BD00200240FA83000013
:1032D000FB830800F8B40020B0B584B000AFF860FC
:1032E0003A607B600B4B5A690A4B01210A435A61D1
:1032F000FB683A681A60BFF36F8FC0467B681C009A
:1033000000231D00FB68043322001A60C046BD463E
:1033100004B0B0BD00200240B0B584B000AF78600A
:103320003960334B1B78012B01D102235CE0304B19
:1033300001221A702E4B00225A600F257C19FA23A5
:103340009B001800FFF77AFF030023702C003B1945
:103350001B78002B42D17B681B68042B0DD17B6846
:103360005B68180000F048F83C19FA239B0018002D
:10337000FFF764FF0300237030E03B6801225242F4
:103380001A607B689B68BB601AE07B685B68BA6800
:103390001100180000F044F80F257C19FA239B0057
:1033A0001800FFF74BFF030023707B191B78002BDD
:1033B00003D03B68BA681A600AE0BB680133BB609F
:1033C0007B689A687B68DB68D318BA689A42DCD35A
:1033D000084B5A69074B02218A435A61044B002269
:1033E0001A700F23FB181B781800BD4604B0B0BD3F
:1033F000F8B400200020024080B582B000AF7860B1
:10340000064B5A697B681A43044B802149020A43E0
:103410005A61C046BD4602B080BDC0460020024091
:1034200080B584B000AF786039600F4B5B690F4A9C
:103430001340FB607B68042B05D0FB68802292015F
:103440001343FB6003E0FB68094A1340FB603B68E1
:10345000DA00FB681A43044B06490A435A61C04626
:10346000BD4604B080BDC0460020024007E0FFFF1B
:10347000FFDFFFFF0200010080B586B000AF78607B
:10348000396000237B614DE13B681B6801217A694B
:1034900091400A001340FB60FB68002B00D13EE125
:1034A0003B685B6803221340012B05D03B685B68D7
:1034B00003221340022B30D17B689B683B617B6900
:1034C0005B0003229A401300DA433B6913403B61DF
:1034D0003B68DA687B695B009A4013003A691343E2
:1034E0003B617B683A699A607B685B683B6101225B
:1034F0007B699A401300DA433B6913403B613B68A8
:103500005B681B0901221A407B699A4013003A69E3
:1035100013433B617B683A695A603B685B680322EE
:103520001340032B17D07B68DB683B617B695B0032
:1035300003229A401300DA433B6913403B613B6826
:103540009A687B695B009A4013003A6913433B61B8
:103550007B683A69DA603B685B6803221340022BA0
:1035600023D17B69DA087B6808329200D3583B612B
:103570007B69072213409B000F229A401300DA4315
:103580003B6913403B613B681A697B6907210B402B
:103590009B009A4013003A6913433B617B69DA0848
:1035A0007B68083292003969D1507B681B683B61A7
:1035B0007B695B0003229A401300DA433B691340A6
:1035C0003B613B685B6803221A407B695B009A4061
:1035D00013003A6913433B617B683A691A603B68A0
:1035E0005A68C0239B02134000D198E0534A7B697C
:1035F0009B0818339B009B583B617B690322134057
:10360000DB000F229A401300DA433B6913403B6111
:103610007A68A023DB059A4219D07B68484A934216
:1036200013D07B68474A93420DD07B68464A934249
:1036300007D07B68454A934201D1042308E0052363
:1036400006E0032304E0022302E0012300E000235C
:103650007A6903210A40D20093403A6913433B61DF
:1036600036497B699B0818339B003A695A50334BA3
:103670001B683B61FB68DA433B6913403B613B6875
:103680005A6880235B03134003D03A69FB681343F5
:103690003B612A4B3A691A60284B5B683B61FB68C7
:1036A000DA433B6913403B613B685A6880239B03C4
:1036B000134003D03A69FB6813433B611F4B3A69DF
:1036C0005A601E4A8423D3583B61FB68DA433B6946
:1036D00013403B613B685A6880239B02134003D030
:1036E0003A69FB6813433B61144984223B698B5060
:1036F000124A8023D3583B61FB68DA433B6913408D
:103700003B613B685A6880235B02134003D03A69EF
:10371000FB6813433B61094980223B698B507B69FD
:1037200001337B613B681A687B69DA40131E00D065
:10373000AAE6C046C046BD4606B080BD001802409D
:103740000004005000080050000C00500010005011
:1037500080B582B000AF786008001100BB1C021C6D
:103760001A807B1C0A1C1A707B1C1B78002B04D04F
:10377000BB1C1A887B689A6103E0BB1C1A887B68B3
:103780009A62C046BD4602B080BD000080B584B0DC
:1037900000AF78607B68002B01D101233DE07B689E
:1037A0001B68204A1A607B681B681F4A1A607B6886
:1037B0001B687A6852685A607B681B687A689268EE
:1037C0009A60FEF7D7FD0300FB600EE0FEF7D2FD26
:1037D0000200FB68D31A312B07D97B681B68DB68B2
:1037E0000722134001D0032317E07B681B68DB68C6
:1037F00007221340EAD17B681B681A697B68DB6883
:103800009A4205D07B681B687A68D2681A6103E027
:103810007B681B68054A1A6000231800BD4604B087
:1038200080BDC046CCCC000055550000AAAA0000BF
:1038300080B582B000AF78607B681B68034A1A606D
:1038400000231800BD4602B080BDC046AAAA0000F1
:1038500080B584B000AF7860194B1B68194A1340DB
:103860001900174B7A680A431A607A6880239B0014
:103870009A421FD1144B1A6813005B009B185B001F
:1038800012491800FCF746FC03000133FB6008E016
:10389000FB68002B03D0FB68013BFB6001E00323C6
:1038A00009E0074B5A698023DB001A408023DB00C4
:1038B0009A42EDD000231800BD4604B080BDC0463A
:1038C00000700040FFF9FFFF0000002040420F00A1
:1038D00080B500AF034B9A68E023DB01134018006A
:1038E000BD4680BD0010024080B588B000AF786052
:1038F0007B68002B01D10123FEE27B681B6801225B
:10390000134000D17CE0C34B9B6838221340BB615D
:10391000C04BDB68032213407B61BB69102B02D1D3
:103920007B69032B02D0BB69082B0BD1B94B1A68FA
:1039300080239B02134062D07B685B68002B5ED1C2
:103940000123D9E27B685A6880235B029A4207D13F
:10395000B04B1A68AF4B802149020A431A6020E03D
:103960007B685A68A023DB029A420ED1A94B1A68E1
:10397000A84B8021C9020A431A60A64B1A68A54BBE
:10398000802149020A431A600BE0A24B1A68A14B3E
:10399000A1490A401A609F4B1A689E4B9F490A40F2
:1039A0001A607B685B68002B14D0FEF7E3FC030011
:1039B0003B6108E0FEF7DEFC02003B69D31A642B92
:1039C00001D9032398E2934B1A6880239B0213408A
:1039D000F0D015E0FEF7CEFC03003B6108E0FEF7F7
:1039E000C9FC02003B69D31A642B01D9032383E28B
:1039F000884B1A6880239B021340F0D100E0C04638
:103A00007B681B680222134000D199E0814B9B68C0
:103A100038221340BB617F4BDB68032213407B617C
:103A2000BB69102B02D17B69022B02D0BB69002B32
:103A300035D1784B1A688023DB00134005D07B68B2
:103A4000DB68002B01D1012356E2724B5B68744A9C
:103A5000134019007B685B691A026E4B0A435A6077
:103A6000BB69002B12D16B4B1B686E4A13401900C7
:103A70007B681A69674B0A431A60664B1B68DB0A4E
:103A800007221340684ADA40684B1A60684B1B688B
:103A90001800FEF713FC031E51D001232CE27B68B3
:103AA000DB68002B30D05B4B1B685E4A134019006B
:103AB0007B681A69574B0A431A60564B1A68554B74
:103AC000802149000A431A60FEF754FC03003B6161
:103AD00008E0FEF74FFC02003B69D31A022B01D924
:103AE000032309E24B4B1A688023DB001340F0D01C
:103AF000484B5B684A4A134019007B685B691A02AD
:103B0000444B0A435A601BE0424B1A68414B4949F7
:103B10000A401A60FEF72EFC03003B6108E0FEF746
:103B200029FC02003B69D31A022B01D90323E3E1EC
:103B3000384B1A688023DB001340F0D100E0C04608
:103B40007B681B680822134047D0324B9B683822A1
:103B50001340182B0AD12F4B1B6E022213403CD06E
:103B60007B689B69002B38D10123C5E17B689B6989
:103B7000002B19D0274B1A6E264B01210A431A66D7
:103B8000FEF7F8FB03003B6108E0FEF7F3FB0200E1
:103B90003B69D31A022B01D90323ADE11D4B1B6EE8
:103BA00002221340F1D018E01A4B1A6E194B012172
:103BB0008A431A66FEF7DEFB03003B6108E0FEF76E
:103BC000D9FB02003B69D31A022B01D9032393E1ED
:103BD000104B1B6E02221340F1D17B681B6804223C
:103BE000134000D1C6E01F23FB1800221A70094BB6
:103BF0009B6838221340202B1ED1064BDB6D02221E
:103C0000134000D1B6E07B689B68002B00D0B1E088
:103C1000012371E100100240FFFFFEFFFFFFFBFFE9
:103C2000FF80FFFFFFC7FFFF0024F400000000201B
:103C300004000020FFFEFFFFB14BDA6B80235B0521
:103C4000134001D1012300E00023002B11D0AC4B25
:103C5000DA6BAB4B802149050A43DA63A84BDA6B78
:103C600080235B051340FB60FB681F23FB180122C8
:103C70001A70A44B1A6880235B0013401AD1A14B21
:103C80001A68A04B802149000A431A60FEF772FBB4
:103C900003003B6108E0FEF76DFB02003B69D31AAD
:103CA000022B01D9032327E1964B1A6880235B007E
:103CB0001340F0D07B689B68012B06D1904BDA6DE6
:103CC0008F4B01210A43DA651CE07B689B68052B5A
:103CD0000CD18B4BDA6D8A4B04210A43DA65884B91
:103CE000DA6D874B01210A43DA650BE0844BDA6D0C
:103CF000834B01218A43DA65814BDA6D804B0421C5
:103D00008A43DA657B689B68002B14D0FEF732FB90
:103D100003003B6109E0FEF72DFB02003B69D31A6B
:103D2000794A934201D90323E6E0754BDB6D022209
:103D30001340F0D013E0FEF71DFB03003B6109E0E8
:103D4000FEF718FB02003B69D31A6F4A934201D970
:103D50000323D1E06A4BDB6D02221340F0D11F2315
:103D6000FB181B78012B05D1654BDA6B644B674957
:103D70000A40DA637B68DB69002B00D1BBE0604B53
:103D80009B6838221340102B00D17BE07B68DB69F5
:103D9000022B56D15A4B1A68594B5D490A401A609A
:103DA000FEF7E8FA03003B6108E0FEF7E3FA0200E1
:103DB0003B69D31A022B01D903239DE0504B1A68AB
:103DC00080239B041340F0D14D4BDB68514A1340D4
:103DD00019007B681A6A7B685B6A1A437B689B6A76
:103DE0001B021A437B68DB6A1A437B681B6B1A430E
:103DF0007B685B6B1A43424B0A43DA60404B1A689C
:103E00003F4B802149040A431A603D4BDA683C4B22
:103E1000802149050A43DA60FEF7ACFA03003B61F2
:103E200008E0FEF7A7FA02003B69D31A022B01D97A
:103E3000032361E0324B1A6880239B041340F0D0C7
:103E400059E02F4B1A682E4B31490A401A60FEF791
:103E500091FA03003B6108E0FEF78CFA02003B692F
:103E6000D31A022B01D9032346E0254B1A6880237D
:103E70009B041340F0D1224BDA68214B26490A40BB
:103E8000DA6038E07B68DB69012B01D1012333E084
:103E90001B4BDB687B617B6903221A407B681B6AD2
:103EA0009A4226D17B6970221A407B685B6A9A42EB
:103EB0001FD17A69FE23DB011A407B689B6A1B02D3
:103EC0009A4216D17A69F8239B031A407B68DB6A11
:103ED0009A420ED17A69E0231B051A407B681B6B5E
:103EE0009A4206D17B695B0F5A077B685B6B9A42EB
:103EF00001D0012300E000231800BD4608B080BDBA
:103F0000001002400070004088130000FFFFFFEF28
:103F1000FFFFFFFE8C80C111FCFFFEEE80B584B078
:103F200000AF786039607B68002B01D10123E9E0A4
:103F3000764B1B68072213403A689A421ED9734B8E
:103F40001B68072293431900704B3A680A431A60B2
:103F5000FEF710FA0300FB6009E0FEF70BFA02001F
:103F6000FB68D31A6A4A934201D90323CAE0674B1C
:103F70001B68072213403A689A42EED17B681B689F
:103F80000222134015D07B681B680422134006D020
:103F9000604B9A685F4BE021C9010A439A605D4B10
:103FA0009B685D4A134019007B689A68594B0A4325
:103FB0009A607B681B680122134057D07B685B685E
:103FC000012B07D1534B1A6880239B0213402BD13E
:103FD000012397E07B685B68022B07D14D4B1A6881
:103FE00080239B0413401FD101238BE07B685B6817
:103FF000002B07D1474B1A688023DB00134013D1F5
:1040000001237FE07B685B68032B06D1414B1B6E6D
:104010000222134008D1012374E03E4BDB6D0222E3
:10402000134001D101236DE03A4B9B680722934373
:1040300019007B685A68374B0A439A60FEF79AF971
:104040000300FB6009E0FEF795F90200FB68D31A54
:104050002F4A934201D9032354E02E4B9B68382208
:104060001A407B685B68DB009A42ECD1274B1B68E7
:10407000072213403A689A421ED2244B1B6807223B
:1040800093431900214B3A680A431A60FEF772F90C
:104090000300FB6009E0FEF76DF90200FB68D31A2C
:1040A0001B4A934201D903232CE0184B1B680722BB
:1040B00013403A689A42EED17B681B680422134091
:1040C00009D0144B9B68154A134019007B68DA68C5
:1040D000104B0A439A6000F029F801000D4B9B68D1
:1040E0001B0A0F221A400E4B9200D3581F22134076
:1040F0000A00DA400B4B1A600B4B1B681800FEF7E6
:10410000DDF803001800BD4604B080BD0020024069
:104110008813000000100240FFF0FFFFFF8FFFFF39
:10412000A4980008000000200400002080B586B09C
:1041300000AF3C4B9B68382213400FD1394B1B68B2
:10414000DB0A0722134001229A4013003B603968C2
:104150003548FBF7DFFF03003B615DE0314B9B68B7
:1041600038221340082B02D1304B3B6154E02D4BD9
:104170009B6838221340102B38D12A4BDB6803226E
:104180001340FB60274BDB681B09072213400133F8
:10419000BB60FB68032B0DD1B9682448FBF7BAFF5D
:1041A000030019001F4BDB681B0A7F2213404B439F
:1041B0007B610DE0B9681C48FBF7ACFF03001900F8
:1041C000184BDB681B0A7F2213404B437B61C046C0
:1041D000144BDB685B0F0722134001337B60796867
:1041E0007869FBF797FF03003B6115E00D4B9B6877
:1041F00038221340202B03D180231B023B610BE0AC
:10420000084B9B6838221340182B03D1FA23DB019B
:104210003B6101E000233B613B691800BD4606B0ED
:1042200080BDC046001002400024F40000366E013C
:1042300080B500AF024B1B681800BD4680BDC0466C
:1042400000000020B0B500AFFFF7F2FF0400FFF759
:104250003FFB03001A0B054B9200D3581F2213405B
:10426000DC4023001800BD46B0BDC046E4980008FD
:1042700080B586B000AF78601323FB1800221A7057
:104280001223FB1800221A707B681A6880239B0295
:10429000134000D1A3E011203B1800221A70B04B4C
:1042A000DA6B80235B05134010D1AD4BDA6BAC4B5E
:1042B000802149050A43DA63A94BDA6B80235B0549
:1042C0001340BB60BB683B1801221A70A54B1A68EB
:1042D000A44B802149000A431A60FEF74BF8030003
:1042E000FB600BE0FEF746F80200FB68D31A022BD6
:1042F00004D91323FB1803221A7005E0994B1A689E
:1043000080235B001340EDD01323FB181B78002B98
:1043100054D1934BDA6DC0239B0013407B617B69C2
:10432000002B19D07B685B6A7A699A4214D08C4B57
:10433000DB6D8D4A13407B61894BDA6D884B8021A0
:1043400049020A43DA65864BDA6D854B87490A4094
:10435000DA65834B7A69DA657B690122134016D0EE
:10436000FEF708F80300FB600CE0FEF703F802001C
:10437000FB68D31A7E4A934204D91323FB18032205
:104380001A7004E0764BDB6D02221340EDD013234C
:10439000FB181B78002B0AD1714BDB6D724A13405E
:1043A00019007B685A6A6E4B0A43DA650CE01223E7
:1043B000FB181322BA1812781A7005E01223FB18A2
:1043C0001322BA1812781A701123FB181B78012BCC
:1043D00005D1634BDA6B624B66490A40DA637B684E
:1043E0001B680122134009D05D4B5B6D0322934390
:1043F00019007B685A685A4B0A435A657B681B68E8
:104400000222134009D0564B5B6D0C2293431900D6
:104410007B689A68524B0A435A657B681B68042282
:10442000134009D04E4B5B6D3022934319007B68DB
:10443000DA684B4B0A435A657B681B68202213409D
:1044400009D0474B5B6D4C4A134019007B681A69D1
:10445000434B0A435A657B681B684022134009D0CE
:104460003F4B5B6D454A134019007B685A693C4BD2
:104470000A435A657B681A688023DB01134015D014
:10448000374B5B6D9B0099087B681A6A344B0A4373
:104490005A657B681A6A8023DB059A4206D1304B45
:1044A000DA682F4B802149020A43DA607B681A6878
:1044B00080231B01134014D0294B9B6D032293438F
:1044C00019007B689A69264B0A439A657B689B6949
:1044D000012B06D1224BDA68214B802149020A4385
:1044E000DA607B681A6880239B01134014D01C4B50
:1044F0009B6D0C22934319007B68DA69184B0A43C1
:104500009A657B68DB69042B06D1154BDA68144B7E
:10451000802149020A43DA607B681A6880235B04C1
:10452000134016D00E4B9B6D134A134019007B6845
:104530009A6A0B4B0A439A657B689A6A80239B01AF
:104540009A4206D1064BDA68054B802149040A439A
:10455000DA601223FB181B781800BD4606B080BD38
:104560000010024000700040FFFCFFFFFFFFFEFF55
:1045700088130000FFFFFFEFFFCFFFFFFF3FFFFFAC
:1045800080B582B000AF78607B68002B01D1012339
:104590004AE07B683D229B5CDBB2002B07D17B6845
:1045A0003C22002199547B681800FCF775FA7B685F
:1045B0003D22022199547B681A687B6804331900F4
:1045C000100000F0B9F97B684822012199547B68FA
:1045D0003E22012199547B683F22012199547B6836
:1045E0004022012199547B684122012199547B6822
:1045F0004222012199547B684322012199547B680E
:104600004422012199547B684522012199547B68F9
:104610004622012199547B684722012199547B68E5
:104620003D220121995400231800BD4602B080BDEF
:1046300080B584B000AF78607B683D229B5CDBB2C4
:10464000012B01D0012341E07B683D2202219954D6
:104650007B681B68DA687B681B6801210A43DA60A3
:104660007B681B681B4A93420ED07B681B681A4A02
:10467000934209D07B681B68184A934204D07B6838
:104680001B68174A934216D17B681B689B68154AC2
:104690001340FB60FB68062B16D0FA6880235B0290
:1046A0009A4211D07B681B681A687B681B680121DD
:1046B0000A431A6008E07B681B681A687B681B68FD
:1046C00001210A431A6000E0C04600231800BD46DD
:1046D00004B080BD002C01400004004000080040F0
:1046E000004001400700010080B584B000AF786051
:1046F0007B681B68DB68FB607B681B681B69BB60B1
:10470000BB680222134021D0FB68022213401DD057
:104710007B681B68032252421A617B6801221A7768
:104720007B681B689B690322134004D07B681800D8
:1047300000F0EAF807E07B68180000F0DDF87B681D
:10474000180000F0E9F87B6800221A77BB680422A1
:10475000134022D0FB68042213401ED07B681B68E4
:10476000052252421A617B6802221A777B681B6815
:104770009A69C0239B00134004D07B68180000F0A6
:10478000C3F807E07B68180000F0B6F87B681800F3
:1047900000F0C2F87B6800221A77BB680822134039
:1047A00021D0FB68082213401DD07B681B680922BA
:1047B00052421A617B6804221A777B681B68DB69A6
:1047C0000322134004D07B68180000F09DF807E036
:1047D0007B68180000F090F87B68180000F09CF8E7
:1047E0007B6800221A77BB681022134022D0FB6836
:1047F000102213401ED07B681B68112252421A619E
:104800007B6808221A777B681B68DA69C0239B00E3
:10481000134004D07B68180000F076F807E07B684E
:10482000180000F069F87B68180000F075F87B68E4
:1048300000221A77BB68012213400CD0FB680122CA
:10484000134008D07B681B68022252421A617B68C1
:104850001800FBF7F1FDBB688022134004D1BA6851
:1048600080239B0113400BD0FB688022134007D0AC
:104870007B681B681E4A1A617B68180000F062F9A9
:10488000BA6880235B0013400BD0FB688022134082
:1048900007D07B681B68174A1A617B68180000F014
:1048A00059F9BB68402213400CD0FB6840221340EA
:1048B00008D07B681B68412252421A617B6818004D
:1048C00000F032F8BB68202213400CD0FB68202295
:1048D000134008D07B681B68212252421A617B6812
:1048E000180000F027F9C046BD4604B080BDC046A0
:1048F0007FDFFFFFFFFEFFFF80B582B000AF786073
:10490000C046BD4602B080BD80B582B000AF7860C1
:10491000C046BD4602B080BD80B582B000AF7860B1
:10492000C046BD4602B080BD80B582B000AF7860A1
:10493000C046BD4602B080BD80B584B000AF78608F
:1049400039607B681B68FB607B683A4A934207D0FA
:104950007B68394A934203D07B68384A934208D136
:10496000FB6870229343FB603B685B68FA68134303
:10497000FB607B682F4A934217D07B682E4A934294
:1049800013D07B682D4A93420FD07B682C4A934208
:104990000BD07B682B4A934207D07B682A4A93420C
:1049A00003D07B68294A934208D1FB68284A134008
:1049B000FB603B68DB68FA681343FB60FB6880229E
:1049C00093431A003B685B691343FB607B68FA689A
:1049D0001A603B689A687B68DA623B681A687B6891
:1049E0009A627B68134A93420BD07B68154A9342C4
:1049F00007D07B68144A934203D07B68134A9342E2
:104A000003D13B681A697B681A637B6801225A618B
:104A10007B681B6901221340012B06D17B681B694F
:104A2000012293431A007B681A61C046BD4604B058
:104A300080BDC046002C014000040040000800403A
:104A40000020004000400140004401400048014077
:104A5000FFFCFFFF80B584B000AF786039607B68F1
:104A60003C229B5C012B01D1022354E07B683C2259
:104A7000012199547B683D22022199547B681B686F
:104A80005B68FB607B681B689B68BB607B681B681E
:104A9000234A934208D1FB68224A1340FB603B68DB
:104AA0005B68FA681343FB60FB6870229343FB600A
:104AB0003B681B68FA681343FB607B681B68FA68F5
:104AC0005A607B681B68164A93420ED07B681B684D
:104AD000154A934209D07B681B68144A934204D05C
:104AE0007B681B68124A93420CD1BB6880229343B7
:104AF000BB603B689B68BA681343BB607B681B68FC
:104B0000BA689A607B683D22012199547B683C22F7
:104B10000021995400231800BD4604B080BDC04652
:104B2000002C0140FFFF0FFF000400400008004080
:104B30000040014080B582B000AF7860C046BD46FD
:104B400002B080BD80B582B000AF7860C046BD467F
:104B500002B080BD80B582B000AF7860C046BD466F
:104B600002B080BD80B582B000AF78607B68002B5A
:104B700001D1012346E07B6888229B58002B07D196
:104B80007B688422002199547B681800FCF746F862
:104B90007B688822242199507B681B681A687B688F
:104BA0001B6801218A431A607B689B6A002B03D033
:104BB0007B68180000F0A4FE7B68180000F0BEFCC3
:104BC0000300012B01D101231CE07B681B685A689C
:104BD0007B681B680D490A405A607B681B689A68AD
:104BE0007B681B682A218A439A607B681B681A6865
:104BF0007B681B6801210A431A607B68180000F07B
:104C000033FF03001800BD4602B080BDFFB7FFFFB1
:104C100080B58AB002AFF860B9603B60BB1D1A80F6
:104C2000FB6888229B58202B00D090E0BB68002BAB
:104C300003D0BB1D1B88002B01D1012388E0FB683A
:104C40009A6880235B019A4209D1FB681B69002B9B
:104C500005D1BB680122134001D0012378E0FB6835
:104C6000902200219950FB68882221219950FDF75C
:104C700081FB03007B61FB68BA1D542112885A52E4
:104C8000FB68BA1D562112885A52FB689A68802325
:104C90005B019A4208D1FB681B69002B04D10023F9
:104CA000FB61BB68BB6103E0BB68FB610023BB61C8
:104CB00030E07A69F8683B68009313000022802195
:104CC00000F07CFF031E05D0FB688822202199504C
:104CD00003233DE0FB69002B0BD1BB691B881A0045
:104CE000FB681B68D205D20D9A62BB690233BB61B7
:104CF00007E0FB691A78FB681B689A62FB6901335D
:104D0000FB61FB6856229B5A9BB2013B99B2FB6840
:104D100056229952FB6856229B5A9BB2002BC8D14F
:104D20007A69F8683B68009313000022402100F084
:104D300045FF031E05D0FB688822202199500323DC
:104D400006E0FB68882220219950002300E002231E
:104D50001800BD4608B080BD80B592B000AF786045
:104D6000EFF310833B623B6A7B6401237B627B6AC7
:104D700083F31088C0467B681B681A687B681B68D1
:104D80004D490A401A607B6CBB62BB6A83F3108892
:104D9000C046EFF31083FB62FB6A3B6401233B6375
:104DA0003B6B83F31088C0467B681B689A687B68FE
:104DB0001B6842490A409A603B6C7B637B6B83F3C0
:104DC0001088C0467B68DB6E012B18D1EFF310838F
:104DD0007B617B69FB630123BB61BB6983F3108843
:104DE000C0467B681B681A687B681B6810218A4371
:104DF0001A60FB6BFB61FB6983F31088C0467B681C
:104E00001B689B6840221340402B39D1EFF310837D
:104E1000BB60BB68BB630123FB60FB6883F3108846
:104E2000C0467B681B689A687B681B6840218A4380
:104E30009A60BB6B3B613B6983F31088C0467B681B
:104E400080229B58002B1BD07B6880229B5800221D
:104E50009A637B6880229B581800FDF71BFF031E96
:104E60000ED07B6880229B581800FEF79FF8030045
:104E7000202B05D17B68902210219950032317E045
:104E80007B685E22002199527B681B680F221A62A0
:104E90007B681B689A697B681B6808210A439A61D2
:104EA0007B688C22202199507B680022DA660023DF
:104EB0001800BD4612B080BDDFFEFFFFFEFFFFEF12
:104EC000B0B5AAB000AF78607B681B68DB69A4222C
:104ED000B9180B607B681B681B68A02039180B6031
:104EE0007B681B689B689C2439190B601100BB18F8
:104EF0001B68A24A13409822BD182B60BB181B6880
:104F0000002B1AD17B181B682022134015D03B18A8
:104F10001B682022134005D13B191A6880235B05CA
:104F200013400AD07B685B6F002B00D1DCE27B680A
:104F30005B6F7A6810009847D6E29823FB181B68CD
:104F4000002B00D122E19C23FB181B688C4A1340E4
:104F500006D1A023FB181B688A4A134000D115E133
:104F6000A423FB181B680122134012D0A023FB18B6
:104F70001A6880235B0013400BD07B681B680122FA
:104F80001A627B6890229B5801221A437B68902109
:104F90005A50A423FB181B680222134011D09C23F3
:104FA000FB181B68012213400BD07B681B68022290
:104FB0001A627B6890229B5804221A437B689021D6
:104FC0005A50A423FB181B680422134011D09C23C1
:104FD000FB181B68012213400BD07B681B6804225E
:104FE0001A627B6890229B5802221A437B689021A8
:104FF0005A50A423FB181B680822134017D0A02383
:10500000FB181B682022134005D19C23FB181B684A
:105010005B4A13400BD07B681B6808221A627B68CE
:1050200090229B5808221A437B6890215A50A4234F
:10503000FB181A6880231B01134013D0A023FB1810
:105040001A688023DB0413400CD07B681B68802225
:1050500012011A627B6890229B5820221A437B68B7
:1050600090215A507B6890229B58002B00D13DE242
:10507000A423FB181B682022134015D0A023FB1883
:105080001B682022134006D19C23FB181A6880233A
:105090005B05134008D07B685B6F002B04D07B68F6
:1050A0005B6F7A68100098477B6890229B58942128
:1050B0007A1813607B681B689B6840221340402B62
:1050C00004D07B181B68282213404CD07B68180042
:1050D00000F0CAFE7B681B689B6840221340402B8F
:1050E0003CD1EFF310833B663B6E90203A1813607F
:1050F00001237B667B6E83F31088C0467B681B6848
:105100009A687B681B6840218A439A603B181B6839
:10511000BB66BB6E83F31088C0467B6880229B58B9
:10512000002B16D07B6880229B58174A9A637B68B5
:1051300080229B581800FDF70DFE031E1CD07B68D3
:1051400080229B589B6B7A688021525810009847A8
:1051500012E07B681800FDF767F80DE07B68180027
:10516000FDF762F808E07B681800FDF75DF87B68E2
:10517000902200219950B9E1C046B7E10F08000024
:1051800001000010200100042D6100087B68DB6E27
:10519000012B00D03EE1A423FB181B681022134012
:1051A00000D137E1A023FB181B681022134000D167
:1051B00030E17B681B6810221A627B681B689B6861
:1051C00040221340402B00D0A4E07B6880229B58F3
:1051D0001B685A687E217B181A807B181B88002B5D
:1051E00000D185E17B685C229B5A7A1812889A422A
:1051F00000D37DE17B687A185E2112885A527B6861
:1052000080229B581B681B682022134070D1EFF34B
:1052100010833B633B6BBB6701237B637B6B83F337
:105220001088C0467B681B681A687B681B68B44995
:105230000A401A60BB6FBB63BB6B83F31088C04628
:10524000EFF31083FB63FB6B7B6701233B643B6CD9
:1052500083F31088C0467B681B689A687B681B686C
:1052600001218A439A607B6F7B647B6C83F3108897
:10527000C046EFF31083BB64BB6C3B670123FB6448
:10528000FB6C83F31088C0467B681B689A687B6858
:105290001B6840218A439A603B6F3B653B6D83F3FB
:1052A0001088C0467B688C22202199507B680022A0
:1052B000DA66EFF310837B657B6DFB660123BB65CC
:1052C000BB6D83F31088C0467B681B681A687B68D7
:1052D0001B6810218A431A60FB6EFB65FB6D83F32C
:1052E0001088C0467B6880229B581800FDF7D2FCCE
:1052F0007B6802221A677B685C229A5A7B685E216F
:105300005B5A9BB2D31A9AB27B6811001800FCF763
:1053100013FFEDE07B685C22995A7B685E229B5A02
:105320009AB28E203B188A1A1A807B685E229B5A9A
:105330009BB2002B00D1DDE03B181B88002B00D175
:10534000D8E0EFF31083FB60FB6888243A19136000
:1053500001233B613B6983F31088C0467B681B686F
:105360001A687B681B6867490A401A603B191B680A
:105370007B617B6983F31088C046EFF31083BB61C8
:10538000BB6984243A1913600123FB61FB6983F331
:105390001088C0467B681B689A687B681B685A49FE
:1053A0000A409A603B191B683B623B6A83F3108892
:1053B000C0467B688C22202199507B680022DA66E7
:1053C0007B6800225A67EFF310837B627B6A80243C
:1053D0003A1913600123BB62BB6A83F31088C0468D
:1053E0007B681B681A687B681B6810218A431A60F7
:1053F0003B191B68FB62FB6A83F31088C0467B681D
:1054000002221A673B181A887B6811001800FCF703
:1054100093FE6FE0A423FB181A6880235B031340FC
:1054200010D09C23FB181A688023DB03134009D09B
:105430007B681B68802252031A627B68180000F0A8
:10544000B8FE5AE0A423FB181B688022134016D034
:10545000A023FB181B688022134006D19C23FB1855
:105460001A6880231B04134009D07B689B6F002BB4
:1054700042D07B689B6F7A68100098473CE0A42379
:10548000FB181B68402213400AD0A023FB181B689E
:105490004022134004D07B68180000F05EFE2CE030
:1054A000A423FB181A6880231B0413400BD0A023ED
:1054B000FB181A688023DB05134004D07B681800B2
:1054C00000F087FE19E0A423FB181A6880235B0410
:1054D000134012D0A023FB181B68002B0DDA7B6849
:1054E000180000F06EFE08E0C04606E0C04604E08A
:1054F000C04602E0C04600E0C046BD462AB0B0BD8E
:10550000FFFEFFFFDFFEFFFFFEFFFFEF80B582B073
:1055100000AF7860C046BD4602B080BD80B582B0A5
:1055200000AF7860C046BD4602B080BD80B582B095
:1055300000AF7860C046BD4602B080BD80B588B07F
:1055400000AF78601B23FB1800221A707B689A68F2
:105550007B681B691A437B685B691A437B68DB695C
:105560001343FB617B681B681B68B44A1340190036
:105570007B681B68FA690A431A607B681B685B6872
:10558000AF4A134019007B68DA687B681B680A43DE
:105590005A607B689B69FB617B681B6AFA691343ED
:1055A000FB617B681B689B68A64A134019007B68F7
:1055B0001B68FA690A439A607B681B68DB6A0F22E2
:1055C000934319007B685A6A7B681B680A43DA6256
:1055D0007B681B689C4A934227D19C4B5B6D0322DE
:1055E0001340032B17D01BD8022B0AD018D8002B3E
:1055F00002D0012B0AD013E01A23FB1800221A70E4
:105600008FE01A23FB1802221A708AE01A23FB1873
:1056100004221A7085E01A23FB1808221A7080E011
:105620001A23FB1810221A707BE07B681B68884ADB
:10563000934227D1854B5B6D0C2213400C2B17D066
:105640001BD8082B0AD018D8002B02D0042B0AD064
:1056500013E01A23FB1800221A7062E01A23FB18C9
:1056600002221A705DE01A23FB1804221A7058E017
:105670001A23FB1808221A7053E01A23FB18102271
:105680001A704EE07B681B68724A934227D16F4BB9
:105690005B6D30221340302B17D01BD8202B0AD043
:1056A00018D8002B02D0102B0AD013E01A23FB18B5
:1056B00000221A7035E01A23FB1802221A7030E01B
:1056C0001A23FB1804221A702BE01A23FB18082255
:1056D0001A7026E01A23FB1810221A7021E07B684A
:1056E0001B685D4A934204D11A23FB1800221A70EA
:1056F00017E07B681B68594A934204D11A23FB18B0
:1057000000221A700DE07B681B68554A934204D151
:105710001A23FB1800221A7003E01A23FB18102228
:105720001A707B68DA6980231B029A4200D065E018
:105730001A23FB181B78082B15D018DC042B0DD06E
:1057400015DC002B02D0022B05D010E0FEF77AFD0D
:1057500003007B6112E0434B7B610FE0FEF7E6FC48
:1057600003007B610AE080231B027B6106E00023CB
:105770007B611B23FB1801221A70C0467B69002B3A
:1057800000D1A6E07B685A6A374B5200D35A190001
:105790007869FAF7BFFC03005A007B685B685B0816
:1057A000D2187B685B6819001000FAF7B3FC03009D
:1057B0003B613B690F2B1CD93A6980235B029A42FB
:1057C00017D23B699AB20E203B180F218A431A80E8
:1057D0003B695B089BB20722134099B23B183A1809
:1057E00012880A431A807B681B683A181288DA60AC
:1057F0006FE01B23FB1801221A706AE01A23FB18C2
:105800001B78082B15D031DC042B0DD02EDC002B9F
:1058100002D0022B05D029E0FEF714FD03007B61C6
:105820002BE0104B7B6128E0FEF780FC03007B61DE
:1058300023E080231B027B611FE0C046F369FFCF9A
:10584000FFCFFFFFFFF4FF110038014000100240BE
:105850000044004000480040004C00400050004020
:10586000003C01400024F4000499000800237B61FF
:105870001B23FB1801221A70C0467B69002B28D01D
:105880007B685A6A1D4B5200D35A19007869FAF79F
:1058900041FC03001A007B685B685B08D2187B68D8
:1058A0005B6819001000FAF735FC03003B613B69A7
:1058B0000F2B0AD93A6980235B029A4205D23B69D1
:1058C0009AB27B681B68DA6003E01B23FB18012295
:1058D0001A707B686A22012199527B686822012133
:1058E00099527B6800225A677B6800229A671B23C3
:1058F000FB181B781800BD4608B080BD049900084D
:1059000080B582B000AF78607B689B6A0822134044
:105910000BD07B681B685B684A4A134019007B68A0
:105920009A6B7B681B680A435A607B689B6A0122FA
:1059300013400BD07B681B685B68434A1340190017
:105940007B68DA6A7B681B680A435A607B689B6ADB
:10595000022213400BD07B681B685B683B4A1340F4
:1059600019007B681A6B7B681B680A435A607B6866
:105970009B6A042213400BD07B681B685B68344A27
:10598000134019007B685A6B7B681B680A435A6096
:105990007B689B6A102213400BD07B681B689B6856
:1059A0002C4A134019007B68DA6B7B681B680A433A
:1059B0009A607B689B6A202213400BD07B681B682F
:1059C0009B68254A134019007B681A6C7B681B682A
:1059D0000A439A607B689B6A402213401DD07B6813
:1059E0001B685B681D4A134019007B685A6C7B6812
:1059F0001B680A435A607B685A6C80235B039A4297
:105A00000BD17B681B685B68154A134019007B68E3
:105A10009A6C7B681B680A435A607B689B6A802289
:105A200013400BD07B681B685B680E4A134019005B
:105A30007B68DA6C7B681B680A435A60C046BD46C7
:105A400002B080BDFF7FFFFFFFFFFDFFFFFFFEFFF6
:105A5000FFFFFBFFFFEFFFFFFFDFFFFFFFFFEFFF9A
:105A6000FFFF9FFFFFFFF7FF80B592B002AF7860A6
:105A70007B68902200219950FCF77CFC0300FB63BB
:105A80007B681B681B6808221340082B2DD1FB6B19
:105A9000802291037868474A0092002200F08EF835
:105AA000031E22D0EFF310837B627B6ABB6301236A
:105AB000BB62BB6A83F31088C0467B681B681A68A8
:105AC0007B681B6880218A431A60BB6BFB62FB6AA0
:105AD00083F31088C0467B688822202199507B6818
:105AE000842200219954032360E07B681B681B68B3
:105AF00004221340042B46D1FB6B8022D10378682B
:105B00002C4A0092002200F059F8031E3BD0EFF31C
:105B10001083FB60FB687B6301233B613B6983F37C
:105B20001088C0467B681B681A687B681B6822491E
:105B30000A401A607B6B7B617B6983F31088C046E7
:105B4000EFF31083BB61BB693B630123FB61FB691E
:105B500083F31088C0467B681B689A687B681B6863
:105B600001218A439A603B6B3B623B6A83F3108856
:105B7000C0467B688C22202199507B6884220021BA
:105B80009954032312E07B688822202199507B6876
:105B90008C22202199507B680022DA667B680022E3
:105BA0001A677B6884220021995400231800BD469F
:105BB00010B080BDFFFFFF01DFFEFFFF80B584B0A6
:105BC00000AFF860B9603B60FB1D1A7051E0BB6923
:105BD00001334ED0FCF7CEFB02003B68D31ABA6902
:105BE0009A4202D3BB69002B01D1032351E0FB6829
:105BF0001B681B68042213403BD0BB68802B38D045
:105C0000BB68402B35D0FB681B68DB69082213405A
:105C1000082B11D1FB681B6808221A62FB68180068
:105C200000F022F9FB68902208219950FB68842239
:105C30000021995401232CE0FB681B68DA6980235A
:105C40001B011A4080231B019A4212D1FB681B687A
:105C5000802212011A62FB68180000F005F9FB6847
:105C6000902220219950FB6884220021995403231B
:105C70000FE0FB681B68DB69BA681340BA68D31A87
:105C80005A425341DBB21A00FB1D1B789A429ED048
:105C900000231800BD4604B080BD000080B590B060
:105CA00000AFF860B960BB1D1A80FB68BA689A65DE
:105CB000FB68BA1D5C2112885A52FB6890220021B1
:105CC0009950FB688C2222219950FB6880229B58B6
:105CD000002B2DD0FB6880229B58404ADA62FB687B
:105CE00080229B583E4A1A63FB6880229B583D4A9B
:105CF0005A63FB6880229B5800229A63FB688022CB
:105D00009858FB681B6824331900FB689B6D1A00C8
:105D1000BB1D1B88FCF738FF031E09D0FB689022CF
:105D200010219950FB688C2220219950012350E0CA
:105D3000FB681B69002B19D0EFF31083BB62BB6AB1
:105D4000FB630123FB62FB6A83F31088C046FB6898
:105D50001B681A68FB681B68802149000A431A60A7
:105D6000FB6B3B633B6B83F31088C046EFF3108300
:105D70003B613B69BB6301237B617B6983F31088D3
:105D8000C046FB681B689A68FB681B6801210A43D0
:105D90009A60BB6BBB61BB6983F31088C046EFF3AD
:105DA0001083FB61FB697B6301233B623B6A83F3E6
:105DB0001088C046FB681B689A68FB681B68402116
:105DC0000A439A607B6B7B627B6A83F31088C046D0
:105DD00000231800BD4610B080BDC046355F0008E6
:105DE00065600008A760000880B58AB000AF7860E1
:105DF000EFF31083BB60BB687B620123FB60FB6831
:105E000083F31088C0467B681B681A687B681B6830
:105E1000C0218A431A607B6A3B613B6983F3108827
:105E2000C046EFF310837B617B693B620123BB615A
:105E3000BB6983F31088C0467B681B689A687B68DF
:105E40001B6808490A409A603B6AFB61FB6983F35F
:105E50001088C0467B68882220219950C046BD46E4
:105E60000AB080BDFFFF7FFF80B58EB000AF7860C5
:105E7000EFF310837B617B697B630123BB61BB69AB
:105E800083F31088C0467B681B681A687B681B68B0
:105E900026490A401A607B6BFB61FB6983F310881B
:105EA000C046EFF310833B623B6A3B6301237B6296
:105EB0007B6A83F31088C0467B681B689A687B689E
:105EC0001B681B490A409A603B6BBB62BB6A83F349
:105ED0001088C0467B68DB6E012B18D1EFF310836E
:105EE000BB60BB68FB620123FB60FB6883F3108827
:105EF000C0467B681B681A687B681B6810218A4350
:105F00001A60FB6A3B613B6983F31088C0467B687B
:105F10008C22202199507B680022DA667B6800225F
:105F20005A67C046BD460EB080BDC046DFFEFFFFCB
:105F3000FEFFFFEF80B594B000AF78607B689B6A8E
:105F4000FB647B681B681B68202213406FD1FB6CCD
:105F50005E2200219952EFF31083BB61BB69BB64E1
:105F60000123FB61FB6983F31088C046FB6C1B684F
:105F70001A68FB6C1B683A490A401A60BB6C3B62AA
:105F80003B6A83F31088C046EFF310837B627B6A21
:105F90007B640123BB62BB6A83F31088C046FB6C41
:105FA0001B689A68FB6C1B6801218A439A607B6CB2
:105FB000FB62FB6A83F31088C046EFF310833B63F8
:105FC0003B6B3B6401237B637B6B83F31088C04690
:105FD000FB6C1B689A68FB6C1B6840218A439A60C3
:105FE0003B6CBB63BB6B83F31088C046FB6C8C229D
:105FF00020219950FB6CDB6E012B18D1EFF310833D
:10600000FB60FB68FB6301233B613B6983F3108802
:10601000C046FB6C1B681A68FB6C1B6810218A4326
:106020001A60FB6B7B617B6983F31088C046FB6C55
:1060300000221A67FB6CDB6E012B08D1FB6C5C2223
:106040009A5AFB6C11001800FCF776F803E0FB6C21
:106050001800FFF763FAC046BD4614B080BDC046C5
:10606000FFFEFFFF80B584B000AF78607B689B6A5D
:10607000FB60FB6801221A67FB68DB6E012B0AD10B
:10608000FB685C229B5A5B089AB2FB6811001800FF
:10609000FCF752F803E0FB681800FFF747FAC04628
:1060A000BD4604B080BD80B586B000AF78607B6827
:1060B0009B6A7B617B6988229B583B617B698C2250
:1060C0009B58FB607B691B689B6880221340802B78
:1060D0000AD13B69212B07D17B69562200219952B5
:1060E0007B691800FFF780FE7B691B689B68402274
:1060F0001340402B0AD1FB68222B07D17B695E221B
:10610000002199527B691800FFF7AEFE7B6990224F
:106110009B5810221A437B6990215A507B691800C2
:10612000FCF782F8C046BD4606B080BD80B584B09D
:1061300000AF78607B689B6AFB60FB685E22002191
:106140009952FB68562200219952FB681800FCF70F
:106150006BF8C046BD4604B080BD80B586B000AFC8
:106160007860EFF31083BB60BB687B610123FB6049
:10617000FB6883F31088C0467B681B681A687B68DD
:106180001B6840218A431A607B693B613B6983F34A
:106190001088C0467B688822202199507B680022A5
:1061A0009A677B681800FFF7B1F9C046BD4606B094
:1061B00080BD80B582B000AF7860C046BD4602B0F9
:1061C00080BD80B582B000AF7860C046BD4602B0E9
:1061D00080BD80B582B000AF7860C046BD4602B0D9
:1061E00080BD000080B584B000AF78607B688422F9
:1061F0009B5C012B01D1022327E07B6884220121D3
:1062000099547B688822242199507B681B681B68FD
:10621000FB607B681B681A687B681B6801218A43E6
:106220001A60FB680B4A1340FB607B6800225A66C9
:106230007B681B68FA681A607B6888222021995065
:106240007B6884220021995400231800BD4604B0C5
:1062500080BDC046FFFFFFDF80B584B000AF78602F
:1062600039607B6884229B5C012B01D102232EE0E4
:106270007B688422012199547B68882224219950CB
:106280007B681B681B68FB607B681B681A687B68FF
:106290001B6801218A431A607B681B689B68DB00CE
:1062A000D9087B681B683A680A439A607B681800C3
:1062B00000F0BCF87B681B68FA681A607B6888226B
:1062C000202199507B6884220021995400231800D2
:1062D000BD4604B080BD000080B584B000AF7860DA
:1062E00039607B6884229B5C012B01D102232FE063
:1062F0007B688422012199547B688822242199504B
:106300007B681B681B68FB607B681B681A687B687E
:106310001B6801218A431A607B681B689B680E4AD0
:10632000134019007B681B683A680A439A607B68CF
:10633000180000F07BF87B681B68FA681A607B68BD
:106340008822202199507B688422002199540023BF
:106350001800BD4604B080BDFFFFFFF1B0B58AB0A4
:1063600000AFF860B960BB1D1A80FB688C229B5897
:10637000202B56D1BB68002B03D0BB1D1B88002BE4
:1063800001D101234EE0FB689A6880235B019A42A9
:1063900009D1FB681B69002B05D1BB6801221340A2
:1063A00001D001233EE0FB680122DA66FB6800228F
:1063B0001A6727257C19BB1D1A88B968FB68180065
:1063C000FFF76CFC030023707B191B78002B24D192
:1063D000FB68DB6E012B1CD1FB681B6810221A6264
:1063E000EFF310837B617B693B620123BB61BB6977
:1063F00083F31088C046FB681B681A68FB681B683B
:1064000010210A431A603B6AFB61FB6983F3108821
:1064100003E02723FB1801221A702723FB181B789F
:1064200000E002231800BD460AB0B0BDF0B585B04B
:1064300000AF78607B685B6E002B08D17B686A22B6
:10644000012199527B6868220121995243E00F266D
:10645000BB1908221A700E203B1808221A707B689C
:106460001B689B685B0EDAB20D243B1907210A40BA
:106470001A707B681B689B685B0FDAB20C257B196E
:1064800007210A401A703B181B787A1912781449B0
:106490008A5C5A4310007B191B78124AD35C19009E
:1064A000F9F7C2FE030099B27B686A229952BB19C0
:1064B0001B783A1912780A498A5C5A4310003B1932
:1064C0001B78084AD35C1900F9F7AEFE030099B2B5
:1064D0007B6868229952C046BD4605B0F0BDC046F3
:1064E0001C9900082499000880B584B000AF78603A
:1064F00039607B68BB600023FB6007E0BA68FB681B
:10650000D31800221A70FB680133FB60FA683B68FD
:106510009A42F3D3C046C046BD4604B080BD80B5A4
:1065200084B000AFF860B9607A607A68B968FB68D7
:106530000020984703001800BD4604B080BD00004D
:1065400080B584B000AF78607B68FB601623BB60C9
:10655000054B9B6BBA68F9681800FFF7E0FF030072
:106560001800BD4604B080BD14B5002080B584B0CD
:1065700000AF78607B68FB603423BB60054B9B6B8E
:10658000BA68F9681800FFF7CAFF03001800BD4693
:1065900004B080BD14B50020B0B58AB000AF7860FB
:1065A0007B68002B02D101235B425CE0304B1B680F
:1065B000002B02D102235B4255E008257B191A21EA
:1065C0001800FFF791FF2B4BDC6A2A4B1878294BF8
:1065D00059687A191A23A047031E0ED07A68264BF1
:1065E000100019001A231A0002F073F8234B180048
:1065F00001F0D6FE05235B4235E00823FB181B683B
:106600001F4A93420AD07A681B4B100019001A23C4
:106610001A0002F05EF806235B4224E008243B19CE
:106620001800FFF78DFF03007B623B19DA8A1B8B92
:106630001B0413431A007B6A93420AD07A680E4BFC
:10664000100019001A231A0002F043F806235B42D7
:1066500009E07A680823FB18100019001A231A00B1
:1066600002F037F800231800BD460AB0B0BDC0469E
:1066700054B5002014B500202C9900083C92000865
:106680004F54415490B58BB000AF78607B68002BBD
:1066900002D101235B4257E02D4B1B68002B02D136
:1066A00002235B4250E00C243A197B681000190069
:1066B0001A231A0002F00DF83B19264A1A603B19FA
:1066C0001800FFF73DFF02003B19163311040C0CB4
:1066D000198800200140081C211C01431980100C5E
:1066E0005A8800210A40111C021C0A435A801A4B86
:1066F0001878194B5B681A22190000F063F8031E22
:1067000006D0164B180001F04BFE04235B421BE041
:10671000114B1C6B104B18780F4B59680C23FA184F
:106720001A23A047031E06D00D4B180001F038FEB7
:1067300004235B4208E0084B1C6B074B18780023CE
:1067400000220021A04700231800BD460BB090BDD9
:1067500054B500204F54415414B5002068920008ED
:106760009492000880B582B000AF786039603B68D1
:10677000002B01D17B680BE07A683B68D318013BA2
:1067800039681800F9F7C6FC03001A003B68534348
:106790001800BD4602B080BD80B582B000AF786001
:1067A00039603B68002B01D17B6807E03968786865
:1067B000F9F7B0FC03001A003B6853431800BD46CC
:1067C00002B080BDB0B588B000AFB9607A600F216B
:1067D0007B18021C1A707B181A781C4B0832920026
:1067E000D358FB61FB69002B02D101235B4229E0F6
:1067F000FA69BB6811001800FFF7CEFF0300BB6108
:10680000BA687B68D218BB69D31AFA6911001800FC
:10681000FFF7A8FF03007B610C4B5B6B7C69B969D8
:106820000F257A19107822009847031E09D07B198A
:1068300019787B69BA69064801F04CFD04235B4274
:1068400000E000231800BD4608B0B0BD14B500201C
:10685000C092000880B586B000AF786039607B6870
:10686000002B02D03B68002B02D101235B4259E090
:106870000123BB6000237B6112E079687A69130011
:10688000DB009B1A5B00CB1804331B78012B04D16F
:106890003B687A691A60002344E07B6901337B61BD
:1068A0007A69BB689A42E8D300233B6112E07968B9
:1068B0003A691300DB009B1A5B00CB1804331B788A
:1068C000002B04D13B683A691A6000232AE03B6937
:1068D00001333B613A69BB689A42E8D30023FB600D
:1068E00012E07968FA681300DB009B1A5B00CB1892
:1068F00004331B78042B04D13B68FA681A60002328
:1069000010E0FB680133FB60FA68BB689A42E8D389
:10691000BB68012B04D13B6800221A60002301E010
:1069200009235B421800BD4606B080BD80B586B025
:1069300000AF786039607B68002B02D03B68002B89
:1069400002D101235B4251E00123BB6000237B6144
:1069500012E079687A691300DB009B1A5B00CB18A0
:1069600004331B78022B04D13B687A691A60002338
:106970003CE07B6901337B617A69BB689A42E8D36A
:1069800000233B6112E079683A691300DB009B1A2F
:106990005B00CB1804331B78032B04D13B683A69A6
:1069A0001A60002322E03B6901333B613A69BB680E
:1069B0009A42E8D30023FB6012E07968FA6813007A
:1069C000DB009B1A5B00CB1804331B78042B04D12B
:1069D0003B68FA681A60002308E0FB680133FB603B
:1069E000FA68BB689A42E8D310235B421800BD46A0
:1069F00006B080BD90B585B000AF78600023FB6025
:106A00007B68002B01D1FB6863E07B689A79D979B8
:106A100009020A43197A09040A435B7A1B061343E5
:106A2000FB602E4BDB6A002B01D1FB6851E07B68D9
:106A30009A7AD97A09020A43197B09040A435B7BD3
:106A40001B061343372B01D8FB6842E0244B382147
:106A50001800FFF749FD214BDC6A7B6858797B6899
:106A60009A79D97909020A43197A09040A435B7AA7
:106A70001B06134319001A4A3823A047031E01D0EE
:106A8000FB6826E0164B1B68164A934201D0FB6850
:106A90001FE0134B5C6B124B1800FFF767FD030000
:106AA0009C4201D0FB6814E00D4B9A687B68997A90
:106AB000D87A00020143187B000401435B7B1B066C
:106AC0000B439A4201D3FB6803E0054B9A68FB68CD
:106AD000D3181800BD4605B090BDC04614B50020BF
:106AE000B0B600204F54415490B58BB000AFF86061
:106AF000B9607A6000237B6200233B620023FB6164
:106B00000023BB611723FB1801221A70FB68002BBE
:106B100005D0BB68002B02D07B68002B02D101237B
:106B20005B428CE0BB681A7A597A09020A43997A67
:106B300009040A43DB7A1B0613431800BB681A7B5F
:106B4000597B09020A43997B09040A43DB7B1B0634
:106B50001343C218FB68997AD87A00020143187B64
:106B6000000401435B7B1B060B439A4202D90A23B4
:106B70005B4264E0BB681A7B597B09020A43997B3C
:106B800009040A43DB7B1B0613433B62FB689A79CB
:106B9000D97909020A43197A09040A435B7A1B0668
:106BA00013431800BB681A7A597A09020A43997A82
:106BB00009040A43DB7A1B061343C318FB6137E061
:106BC0003B6ABB61BA6980235B009A4202D9802389
:106BD0005B00BB611C4BDC6AFB685879BB691B4AD4
:106BE000F969A047031E02D004235B4227E0172463
:106BF0003B191B78002B0BD0134B9B6BBA691349C5
:106C00000020984703007B623B1900221A7007E0BE
:106C10000D4B9B6BBA690D490120984703007B62BD
:106C2000FA69BB69D318FB613A6ABB69D31A3B6244
:106C30003B6A002BC4D17B687A6A1A600023180073
:106C4000BD460BB090BDC04614B50020B0B50020C5
:106C500090B58BB000AF78607B68002B02D1012328
:106C60005B424BE07B68DB6A002B0FD07B681B6BC1
:106C7000002B0BD07B685B6B002B07D07B689B6B7A
:106C8000002B03D07B68DB6B002B06D11D4B18005B
:106C900001F086FB01235B4230E01B4A7B68100059
:106CA000190040231A0001F014FD184B01221A604C
:106CB000174B58211800FFF717FC08243B19180040
:106CC000FFF76AFC03007B627B6A002B15D03A1940
:106CD000104B100019001A231A0001F0FAFC3B199E
:106CE0000D4A1A603B191800FFF7CCFC03007B62C9
:106CF0007B6A002B01D07B6A00E000231800BD46B0
:106D00000BB090BD0893000814B5002054B50020C6
:106D100058B500202C9900084F544154B0B590B09C
:106D200000AF0823FB181800FFF736FC03003B6395
:106D30000023FB630123FB620023BB6300237B630F
:106D400013E00823F9187A6B1300DB009B1A5B0031
:106D5000CB1804331B78022B04D17B6BFB6301231C
:106D6000BB6306E07B6B01337B637A6BFB6A9A4201
:106D7000E7D3BB6B002B00D18CE008203918FA6BED
:106D80001300DB009B1A5B00CB180433BB62BB6AA9
:106D90005A78997809020A43D97809040A431B7979
:106DA0001B0613430133022B1FD9BB6A00221A7042
:106DB000BB6A01331A7800210A401A705A78002100
:106DC0000A405A709A7800210A409A70DA780021B5
:106DD0000A40DA703B181800FFF754FC03003B63CD
:106DE0003B6B002B56D03B6B82E0BB6A5A7899789C
:106DF00009020A43D97809040A431B791B06134385
:106E00005A1CBB6A0133FF2111400C001978002085
:106E10000140081C211C01431970110AFF20014088
:106E20000C00597800200140081C211C01435970B6
:106E3000110CFF2001400C00997800200140081C33
:106E4000211C01439970100EDA7800210A40111CB0
:106E5000021C0A43DA700823FB181800FFF712FC23
:106E600003003B633B6B002B01D03B6B40E0224BAC
:106E7000DC6BBB6A1800FFF7BDFD03001800A047DC
:106E800003003B633B6B002B02D011235B422FE0DE
:106E900000232DE000237B603A1D08257B1911009B
:106EA0001800FFF743FD03007B627B6A002B19D1BA
:106EB000114BDC6B7A6879191300DB009B1A5B00BD
:106EC000CB1804331800FFF795FD03001800A04706
:106ED00003003B633B6B002B02D011235B4207E0B6
:106EE000002305E0054B180001F05AFA10235B421D
:106EF0001800BD4610B0B0BD14B500204493000882
:106F000080B58AB000AF164B1B68002B01D100235F
:106F100021E03B1D1800FFF73FFB031E01D00023BB
:106F200019E001233B6200237B620FE0391D7A6A7E
:106F30001300DB009B1A5B00CB1804331B78032B78
:106F400001D1012307E07B6A01337B627A6A3B6AE5
:106F50009A42EBD300231800BD460AB080BDC0465C
:106F600054B5002090B58FB000AF78607B68002BDF
:106F700002D101235B42A6E1D54B1B68002B02D155
:106F800002235B429FE1D34B1B68002B02D00323FB
:106F90005B4298E17B681A78597809020A4399782C
:106FA00009040A43DB781B0613431A00CA4B9A42B2
:106FB00006D0CA4B180001F0F3F907235B4282E1C7
:106FC0007B681800FFF7D2FA03007B637B683422EA
:106FD0009A5C3521595C09020A433621595C09043F
:106FE0000A4337215B5C1B0613431A007B6B9342F9
:106FF00006D0BB4B180001F0D3F908235B4262E1D5
:107000000C243B191800FFF7C7FA03003B63002369
:10701000BB600823FA183B1911001800FFF71AFC8F
:10702000031E06D0AF4B180001F0BAF909235B42EA
:1070300049E1BA680C23F9181300DB009B1A5B00C6
:10704000CB180433FB627B681A7A597A09020A4327
:10705000997A09040A43DB7A1B0613431800FB6A7A
:107060009A7AD97A09020A43197B09040A435B7B9D
:107070001B061343984206D39B4B180001F090F96E
:107080000A235B421FE17B681A7A597A09020A4394
:10709000997A09040A43DB7A1B06134318007B68BC
:1070A0001A7B597B09020A43997B09040A43DB7B5B
:1070B0001B061343C218FB6A997AD87A000201436F
:1070C000187B000401435B7B1B060B439A4206D9E5
:1070D000864B180001F064F90A235B42F3E07B68F9
:1070E0001A7B597B09020A43997B09040A43DB7B1B
:1070F0001B0613431800FB6A9A7AD97A09020A43DD
:10710000197B09040A435B7B1B061343984206D98B
:10711000774B180001F044F90A235B42D3E07B6807
:107120001A7A597A09020A43997A09040A43DB7ADE
:107130001B06134318007B681A7B597B09020A431C
:10714000997B09040A43DB7B1B061343C318BB620C
:10715000FB6A9A7AD97A09020A43197B09040A431D
:107160005B7B1B0613431A00BB6A934206D9614B33
:10717000180001F015F90A235B42A4E0FB6A587974
:10718000FB6A9A79D97909020A43197A09040A43F0
:107190005B7A1B0613431900BB6A1A00FFF712FB48
:1071A000031E06D0544B180001F0FAF804235B428A
:1071B00089E0FB6A01221A70FB6A01331A78002108
:1071C0000A401A705A7800210A405A709A780021B1
:1071D0000A409A70DA7800210A40DA700C203B18D5
:1071E00016331A8800210A401A805A8800210A4062
:1071F0005A8004003B181800FFF744FA03003B6371
:107200003B6B002B0CD03D4B180001F0C9F8FB6A1A
:1072100000221A703B191800FFF734FA3B6B52E05A
:107220002C4B58211800FFF75FF92A4B01221A60F6
:10723000BA68284B5A60274B7A6808331100382205
:10724000180001F046FA7B681A7B597B09020A4351
:10725000997B09040A43DB7B1B0613431A001D4B71
:107260001A647B681A7A597A09020A43997A0904DE
:107270000A43DB7A1B06134318007B681A7B597B91
:1072800009020A43997B09040A43DB7B1B0613436B
:10729000C218104B5A647B681A7C597C09020A4355
:1072A000997C09040A43DB7C1B0613431A00094B33
:1072B0009A64084B0022DA64064B00221A65054BDB
:1072C00000225A6500231800BD460FB090BDC0468D
:1072D00054B5002058B500204F5441547C93000809
:1072E000B0930008E4930008209400085894000824
:1072F00098940008CC94000804950008389500087C
:1073000090B591B000AFF860B9607A60BB68002BAF
:1073100005D17B68002B02D001235B42ABE0584BC8
:107320001B68002B02D102235B42A4E0554B1B6873
:10733000002B02D10B235B429DE01423FB181800A5
:10734000FFF72AF90300FB63FB6B002B07D0FA6BF6
:107350004D4B1100180000F0BDFFFB6B8BE0494B5B
:107360005B68BB631423F918BA6B1300DB009B1A2C
:107370005B00CB1804337B637B6B1B78012B0AD03B
:107380007B6B1B781A00414B1100180000F0A2FF24
:107390000B235B426FE03B4BDB6CFA689A4209D0EF
:1073A000384BD96CFA683A4B180000F093FF0C2365
:1073B0005B4260E0FA687B68D218324B5B6C9A42A1
:1073C00009D9304B5B6C7A68F968324800F082FF6B
:1073D0000D235B424FE07B68002B01D100234AE084
:1073E0007B6B9A79D97909020A43197A09040A430D
:1073F0005B7A1B0613431A00FB689B183B633A6BCE
:107400007B68D2187B6B9979D87900020143187A8E
:10741000000401435B7A1B060B431C007B6B997ACB
:10742000D87A00020143187B000401435B7B1B06F2
:107430000B43E3189A4206D9174B180000F0B0FF2F
:107440000A235B4217E0154B1C6B7B6B58797B68FA
:10745000BA68396BA047031E06D0114B180000F024
:107460009FFF04235B4206E0064BDA6C7B68D21870
:10747000044BDA6400231800BD4611B090BDC0462D
:1074800054B5002058B500206C950008A095000860
:10749000D4950008109600085896000814B50020EE
:1074A0008C96000890B58DB000AF5F4B1B68002B29
:1074B00002D102235B42B2E05C4B1B68002B02D17D
:1074C0000B235B42ABE00823FB181800FFF764F8BE
:1074D0000300FB62FB6A002B01D0FB6A9FE0534B69
:1074E0005B68BB620823F918BA6A1300DB009B1AB9
:1074F0005B00CB1804337B627B6A1B78012B0AD0BC
:107500007B6A1B781A004A4B1100180000F0E2FE5B
:107510000E235B4283E0454BDA6C444B5B6C9A4232
:107520000AD0424BD96C414B5A6C424B180000F0C8
:10753000D1FE0D235B4272E03F4B1C6B7B6A587996
:10754000002300220021A04700237B603A1D3B4915
:107550007B6A1800FFF7C8FA0300FB62FB6A002B86
:1075600001D0FB6A5BE0314B9A6C7B689A422FD06A
:1075700079682E4B9A6C324B180000F0ABFE7B6A98
:1075800000221A707B6A01331A7800210A401A70AF
:107590005A7800210A405A709A7800210A409A705D
:1075A000DA7800210A40DA700823FB181800FFF788
:1075B00069F80300FB62FB6A002B01D0FB6A2EE036
:1075C0001A4B58211800FEF78FFF0F235B4226E06D
:1075D0007B6A02221A707B6A01331A7800210A4002
:1075E0001A705A7800210A405A709A7800210A408D
:1075F0009A70DA7800210A40DA700823FB18180024
:10760000FFF740F80300FB62FB6A002B01D0FB6A26
:1076100005E0064B58211800FEF766FF002318000E
:10762000BD460DB090BDC04654B5002058B50020F1
:10763000B8960008F496000814B5002060B5002044
:107640004097000880B58CB000AF3A4B1B68002B08
:1076500002D102235B4269E03B001800FEF79CFF69
:1076600003007B6201235B42FB62334B1B68002BF0
:1076700003D0314B5B68FB6219E001233B620023BE
:10768000BB6210E03900BA6A1300DB009B1A5B0092
:10769000CB1804331B78012B02D1BB6AFB6206E0D6
:1076A000BB6A0133BB62BA6A3B6A9A42EAD3FB6A9D
:1076B000002B06DA214B180000F072FE09235B4212
:1076C00034E0FA6A39001300DB009B1A5B00CB1828
:1076D0000433FB61FB6900221A70FB6901331A78DD
:1076E00000210A401A705A7800210A405A709A788C
:1076F00000210A409A70DA7800210A40DA703B00D3
:107700001800FEF7BFFF03007B627B6A002B01D0ED
:107710007B6A0BE0084B58211800FEF7E5FEFA6A79
:10772000074B1100180000F0D5FD00231800BD46DE
:107730000CB080BD54B5002058B5002084970008D7
:10774000BC97000890B58BB000AF7860184B1B68F1
:10775000002B02D102235B4226E008243B191800CB
:10776000FEF71AFF03007B623B1912333A1D1088A3
:107770001A8800210A40111C021C0A431A80BA1DF3
:1077800010885A8800210A40111C021C0A435A80A2
:107790003B191800FEF776FF03007B627B6A002B23
:1077A00001D07B6A00E000231800BD460BB090BDFD
:1077B00054B5002080B588B000AF0A4B1B68002B81
:1077C00001D100230AE03B001800FEF7E5FE0300AC
:1077D000FB613B005A8A9B8A1B0413431800BD4679
:1077E00008B080BD54B5002080B584B000AF78608B
:1077F000EFF31083FB60FA687B681A6072B6C046CC
:10780000C046BD4604B080BD80B582B000AF786090
:107810007B68002B01D162B6C046C046BD4602B0AF
:1078200080BD80B582B000AF786039603B68002BC6
:1078300001D17B6807E039687868F8F76BFC0300D2
:107840001A003B6853431800BD4602B080BD80B5A6
:1078500082B000AF786039603B68002B01D17B6853
:107860000BE07A683B68D318013B39681800F8F7D9
:1078700051FC03001A003B6853431800BD4602B098
:1078800080BD000080B500AF084B00225A73074B43
:1078900000221A73054B00221A60054B08220021B2
:1078A000180000F093FEC046BD4680BDE8B600203B
:1078B000ECB6002090B589B000AF786039607B6885
:1078C00014243A191000190008231A0000F001FFCF
:1078D00039683B190822180000F058FE031E01D138
:1078E000002341E00023FB611EE01423FA18FB692A
:1078F000D3181B783968FA698A1812781340DAB2FB
:107900003968FB69CB181B789A420AD07A68FB6900
:10791000D218174B1100180000F0DCFC01235B4269
:1079200022E0FB690133FB61FB69072BDDD90022F3
:107930000023BA60FB6039680823FB18082218008E
:1079400000F0C7FEBA68FB6879680120FBF7E2FB2C
:10795000031E08D07A68074B1100180000F0BAFC2B
:1079600001235B4200E000231800BD4609B090BD32
:107970005C9800088498000880B582B000AF0B4B7B
:107980005B7B002B01D100230BE0084B1B68084AEE
:1079900011001800FFF78EFF03007B60FFF772FFF6
:1079A0007B681800BD4602B080BDC046E8B6002026
:1079B000ECB6002080B582B000AF7860314B1A6819
:1079C000C0239B0413400ED02E4B1A68C0239B0487
:1079D0001A4080235B049A420FD12B4B1A688023F4
:1079E0009B03134009D1294B1B689B02284A134073
:1079F000802212059446634409E0244B1B689B02D5
:107A00005B08244A134080221205944663447A6836
:107A1000934206D97B68F822120694466344DB0A37
:107A20002BE0184B1A68C0239B0413400ED0154B53
:107A30001A68C0239B041A4080235B049A420FD12A
:107A4000114B1A6880239B03134009D10F4B1B680D
:107A50009B020F4A1340802212059446634409E0BA
:107A60000A4B1B689B025B080A4A134080221205DE
:107A7000944663447A68D31ADB0A1800BD4602B004
:107A800080BDC0460075FF1F20200240E075FF1F2B
:107A900000FC0F0000FE070080B582B000AF7860E8
:107AA000194B1A68C0239B0413400ED0164B1A685A
:107AB000C0239B041A4080235B049A420FD1134BCE
:107AC0001A6880239B03134009D1114B1B689B024A
:107AD000104A1340802212059446634409E00C4B7F
:107AE0001B689B025B080C4A1340802212059446D7
:107AF00063447A68934201D9042301E080231B0286
:107B00001800BD4602B080BD0075FF1F2020024056
:107B1000E075FF1F00FC0F0000FE070080B582B07B
:107B200000AF78607B68042B29D0184B1A68C023FB
:107B30009B0413400ED0154B1A68C0239B041A40B7
:107B400080235B049A420FD1114B1A6880239B0358
:107B5000134009D10F4B1B689B020F4A1340802230
:107B60001205944663440CE00A4B1B689B025B08B9
:107B70000A4A1340802212059446634401E08023A0
:107B80001B051800BD4602B080BDC0460075FF1F32
:107B900020200240E075FF1F00FC0F0000FE0700E0
:107BA00090B591B000AF786039603B68002B01D18F
:107BB0000023B5E0FFF766FE80231A017B68110001
:107BC0001800FFF72EFE03007B6080231A013B683C
:107BD00011001800FFF73BFE03003B602023FB1859
:107BE0001800FFF701FEFBF7E3FA031E06D03B6A1D
:107BF0001800FFF709FE01235B4291E04A4B802207
:107C000012021A611023FB18180010231A00002119
:107C100000F0DCFC7B68FB633B68BB630023FB601C
:107C20006BE0FB6B1800FFF737FF03003B633B6B18
:107C30001800FFF773FF0300FB623C4B1A68C02378
:107C40009B0413400ED0394B1A68C0239B041A4082
:107C500080235B049A420BD1354B1A6880239B0327
:107C6000134005D1334B1B689B02334A134005E098
:107C7000304B1B689B025B08304A1340FA6A9B1822
:107C8000BB62BA6AFB6BD31ADB0A7B62BB6BDB0A93
:107C90007B637A6B7B6A9A4201D97B6A7B6310248F
:107CA0003B1902221A603B193A6B5A60FB6B1800B1
:107CB000FFF780FE020021007B189A607B187A6B28
:107CC000DA600C23FA187B1811001800FBF724FB6C
:107CD000031E08D0FBF790FA3B6A1800FFF794FDEB
:107CE00001235B421CE07B6BDB02FA6BD318FB6366
:107CF0007B6BDB02BA6BD31ABB63BB6B002B90D1DF
:107D0000FBF77AFA031E06D03B6A1800FFF77CFDEA
:107D100001235B4204E03B6A1800FFF775FD002376
:107D20001800BD4611B090BD002002400075FF1F35
:107D300020200240E075FF1F00FC0F0000FE07003E
:107D400090B593B000AFF860B9607A607B68002BA3
:107D500001D10023C3E0FA687B68D318BB63FB68DA
:107D600008211800FFF75DFD03007B63BB6B013B3F
:107D700008211800FFF755FD03003B635A4B5B7B5E
:107D8000002B0DD0584B1B687A6B9A4208D9FFF72D
:107D9000F3FD0300FB62FB6A002B01D0FB6A9EE04F
:107DA0007B6B7B6495E043243B1900221A704E4B99
:107DB0005B7B002B0FD04C4B1B687A6C9A420AD12C
:107DC0001423FA18484B043303CB03C23B19464A29
:107DD000127B1A700CE07B6C1422BA181000190088
:107DE00008231A0000F075FC4323FB1800221A70C8
:107DF0000023FB6325E07A6CFB6BD318FB61FA6907
:107E0000FB689A421AD3FA69BB6B9A4216D2FA6996
:107E1000FB68D31ABA68D31819781423FA18FB6BC5
:107E2000D3180A1C1A700122FB6B9A401300D9B2B6
:107E30004322BB18BA1812780A431A70FB6B01333D
:107E4000FB63FB6B072BD6D97A6C3B6BD31A5A4278
:107E50005341DBB2BB6243217B181B78FF3B5A4284
:107E60005341DBB27B62BB6A002B16D07B6A002BCE
:107E700013D11D4B01225A731B4B7A6C1A601A4B9B
:107E80007A1812781A73184B1422BA18043303CADA
:107E900003C37B6C08337B641BE01423FA187B6CF0
:107EA00011001800FFF706FD03003B623B6A002B40
:107EB00001D03B6A13E00C4B5B7B002B06D00A4BD6
:107EC0001B687A6C9A4201D1FFF7DCFC7B6C0833AB
:107ED0007B647A6CBB6B9A4200D264E70023180083
:107EE000BD4613B090BDC046E8B6002080B584B052
:107EF00000AFB9607A603B600F23FB18021C1A7058
:107F00003B68002B01D1002314E07B68002B02D1D9
:107F100001235B420EE00F23FB181B78002B07D1D7
:107F2000B9683A687B68180000F0D3FB002301E0D1
:107F300001235B421800BD4604B080BD80B588B007
:107F400000AFB9607A603B600F217B18021C1A7089
:107F50007B181B78002B02D001235B424BE03B686F
:107F6000002B1FD11023FB181800FFF73DFCFBF777
:107F70001FF9031E06D03B691800FFF745FC0123DB
:107F80005B4238E01E4B802212021A61FFF7F4FCBC
:107F90000300BB61FBF730F93B691800FFF734FCC5
:107FA000BB6928E07B68002B02D101235B4222E001
:107FB0001423FB181800FFF717FCFBF7F9F8031E52
:107FC00006D07B691800FFF71FFC01235B4212E01B
:107FD0000B4B802212021A613A687968BB6818005C
:107FE000FFF7AEFE0300FB61FBF706F97B691800A3
:107FF000FFF70AFCFB691800BD4608B080BDC0460B
:108000000020024080B584B000AFB9607A600F21D3
:108010007B18021C1A707B181B78002B02D00123DE
:108020005B4206E07A68BB6811001800FFF7B8FDF4
:1080300003001800BD4604B080BD000080B584B0C8
:1080400000AFB9607A600F23FB18021C1A707B68BE
:10805000002B02D0BB68002B01D100231BE00F23B3
:10806000FB181B78002B0FD10D4B1B689A680C4B2B
:108070001B6801210A439A607A68B968084B1800A6
:10808000FAF747FB030006E07A68B968044B18006A
:10809000FAF7F8FA03001800BD4604B080BDC046E8
:1080A0001001002080B584B000AF78607B68002BA1
:1080B00002D101235B4216E072B6C0460C4B7A68CF
:1080C0009A607B6804331B681A000A4B1A607B684D
:1080D0001B68FB60FB6883F30888C046054B1B6880
:1080E0009847C046FDE71800BD4604B080BDC046B5
:1080F00000ED00E0F8B600200D488546F8F70AFBD1
:108100000C480D490D4A002302E0D458C4500433F2
:10811000C4188C42F9D30A4A0A4C002301E01360C8
:108120000432A242FBD300F0ADFAF8F79BF9FEE768
:108130000040022000000020F0000020C499000848
:10814000F000002048B80020FEE70000002310B532
:10815000040003604360836081814366C2810361E0
:1081600043618361190008225C3000F02FFA0B4B49
:10817000246263620A4BA3620A4BE3620A4B2363E5
:108180000A4B9C4205D00A4B9C4202D0094B9C42B0
:1081900003D12000583000F099FA10BDB5830008D3
:1081A000DD8300081584000841840008FCB6002027
:1081B00064B70020CCB7002010B5034A0349044837
:1081C00000F06CF810BDC0460C000020698F00085C
:1081D0001C00002041680B4B10B50400994201D0EF
:1081E00000F0C2FEA168084B994202D0200000F0C6
:1081F000BBFEE168054B994202D0200000F0B4FEBE
:1082000010BDC046FCB6002064B70020CCB70020EB
:1082100010B5094B094A04211A6009480022FFF7EA
:1082200095FF012209210748FFF790FF0222122142
:108230000548FFF78BFF10BD34B80020B981000856
:10824000FCB6002064B70020CCB7002010B502486F
:1082500000F03DFA10BDC0463DB8002010B5024800
:1082600000F036FA10BDC0463DB8002010B504003D
:10827000FFF7ECFF236A002B02D0FFF7EFFF10BDE2
:10828000044B2362044B1B68002BF6D1FFF7C0FFA1
:10829000F3E7C046D581000834B80020F7B51400D4
:1082A000002600900191A5686768013F04D5246805
:1082B000002CF8D13000FEBDAB89012B08D90E226D
:1082C000AB5E013304D029000098019B9847064318
:1082D0006835EAE70FB407B5054904AB086804CB75
:1082E0008168019300F022FB03B008BC04B018477A
:1082F00018000020036A70B505000E008468002B8A
:1083000001D1FFF7B3FF636EDB0705D4A3899B059B
:1083100002D4A06D00F0DBF9A3891B0702D5236905
:10832000002B1FD12100280000F0D2F8002819D01E
:1083300001256D42636EDB0705D4A3899B0502D43A
:10834000A06D00F0C5F9280070BD0136A360002BB8
:1083500004DAA2699A4216DC0A2914D023685A1C4E
:1083600022601970A3683178013B0029EDD1A36028
:10837000002B0FDA220028000A3100F067F80130E4
:10838000D6D00A25D6E72200280000F05FF8013099
:10839000E8D1CDE723685A1C22600A221A70F0E760
:1083A00010B5034B01001868FFF7A4FF10BDC046CD
:1083B0001800002070B50C000E25495F00F034F95C
:1083C000002803DB636D1B18636570BDA389024A37
:1083D0001340A381F9E7C046FFEFFFFFF8B51F0088
:1083E0008B8905000C001600DB0505D50E23C95E40
:1083F0000022022300F004F9A389054A2800134053
:10840000A38132000E23E15E3B0000F021F9F8BDAC
:10841000FFEFFFFF70B50C000E25495F00F0F0F88C
:10842000A389421C03D1054A1340A38170BD802259
:1084300052011343A3816065F8E7C046FFEFFFFFD9
:1084400010B50E23C95E00F0C9F810BDF8B50600DE
:108450000D001400002804D0036A002B01D1FFF79F
:1084600005FFA369A360A3891B0702D52369002B1D
:1084700009D12100300000F02BF8002803D001259D
:108480006D422800F8BD23692068EFB2C01A636905
:10849000EDB2834205DC2100300000F065FD0028CC
:1084A000EDD1A3680130013BA36023685A1C226010
:1084B0001F706369834204D0A389DB07E1D50A2DCD
:1084C000DFD12100300000F04FFD0028D9D0D6E7E1
:1084D0002D4B70B5050018680C00002804D0036A05
:1084E000002B01D1FFF7C2FE0C22A35E1A0723D492
:1084F000DA0607D409222A60402201201343A3810F
:1085000040423AE05B0713D5616B002908D0230095
:108510004433994202D0280000F0E4F8002363635A
:108520002422A3899343A3810023636023692360EA
:108530000823A2891343A3812369002B0BD1A02117
:108540008022A389890092000B40934203D021002E
:10855000280000F05FFD0C22A35E01211A000A40F2
:108560000B420BD00022A26062695242A26100203D
:108570002269824201D11A06BED470BD990700D487
:108580006269A260F3E7C0461800002030B50024FD
:108590000139A24201D1002005E0035D01340D5DE7
:1085A000AB42F6D0581B30BD10B5884202D98B18AB
:1085B000984208D300239A4207D0CC5CC4540133BC
:1085C000F9E78B5C8354013AFBD210BD030082189B
:1085D000934200D1704719700133F9E7002370B559
:1085E000064D040008002B60F8F7D2F8431C03D1B5
:1085F0002B68002B00D0236070BDC04638B8002027
:1086000070B50400080011001A000023054D2B600E
:10861000F8F7DFF8431C03D12B68002B00D0236050
:1086200070BDC04638B8002070B5040008001100C5
:108630001A000023054D2B60F8F771F8431C03D195
:108640002B68002B00D0236070BDC04638B80020D6
:1086500070B50400080011001A000023054D2B60BE
:10866000F8F77AF8431C03D12B68002B00D0236065
:1086700070BDC04638B80020014B18687047C0462E
:108680001800002070B500260C4C0D4D641BA41082
:10869000A64209D1002600F041FD0A4C0A4D641B98
:1086A000A410A64205D170BDB300EB58984701361F
:1086B000EEE7B300EB5898470136F2E7BC990008A3
:1086C000BC990008C0990008BC9900087047704721
:1086D0007047002310B59A4200D110BDCC5CC45441
:1086E0000133F8E770B505000C1E10D0043C236878
:1086F000002B00DAE418280000F0E0F81D4A1368A7
:10870000002B05D163601460280000F0DFF870BD15
:10871000A34208D9206821188B42F3D119685B68FD
:1087200009182160EEE71A005B68002B01D0A34214
:10873000F9D911685018A0420BD1206809185018B7
:1087400011608342E0D118685B6841181160536082
:10875000DAE7A04202D90C232B60D5E72068211864
:108760008B4203D119685B6809182160636054600B
:10877000CAE7C04644B8002070B50F4E0D003168FE
:108780000400002902D100F0ABFC30602900200079
:1087900000F0A6FC431C03D101256D42280070BDEA
:1087A0000323C51C9D43A842F8D0291A200000F0DD
:1087B00097FC0130F2D1EFE740B80020F7B5032273
:1087C000CB1C9343083305001F000C2B34D20C271D
:1087D000B94233D8280000F071F8374E33681C00D6
:1087E000002C2FD139002800FFF7C6FF0400431CDE
:1087F0005FD134680094009B002B4AD1002C52D0EA
:1088000023682800E3180099019300F069FC019B9C
:10881000834248D123682800FF1A3900FFF7ACFFD4
:10882000013040D02368DB19236033685A68002A7E
:1088300033D1009B336019E0002BC9DA0C232B6085
:108840000020FEBD2168C91B20D40B290AD9E219DA
:108850002760A34204D1326063681160536005E071
:108860005A60F9E76268A3420ED13260280000F036
:108870002DF8200007220B30231D9043C21A984286
:10888000DFD01B1AA350DCE75A60EFE723006468CF
:10889000A6E7009C63680093ADE71A005B68A342FB
:1088A000FBD10023DAE70C2328002B6000F00EF840
:1088B000C6E70760DAE7C04644B8002010B50248B2
:1088C000FFF705FF10BDC0463CB8002010B50248B8
:1088D000FFF7FEFE10BDC0463CB80020936810B5FF
:1088E000013B9360002B04DA9469A34207DB0A2959
:1088F00005D01368581C10601970080010BDFFF7F0
:10890000A5FD0100F9E7F8B506000F001400D51821
:10891000AC4201D1002007E021783A003000FFF797
:10892000DDFF0134431CF3D1F8BD0000F0B5A1B068
:108930000F0015001E000390002804D0036A002BCE
:1089400001D1FFF793FC7B6EDB0705D4BB899B0548
:1089500002D4B86DFFF7BBFEBB891B0702D53B698C
:10896000002B13D139000398FFF7B2FD00280DD07A
:108970007B6EDB0703D50120404221B0F0BDBB89EF
:108980009B05F8D4B86DFFF7A3FEF4E7002308AC0D
:108990006361203363761033A37607962E00337815
:1089A000002B01D0252B48D1731B0593AE420BD071
:1089B0002A0039000398FFF7A6FF013000D1AEE08E
:1089C0006369059A9B1863613378002B00D1A6E098
:1089D000012200235242626004A954325218751CCD
:1089E0002360E360A3601370A365594B0522180050
:1089F0002978059300F086FB6E1C00281FD12268A1
:108A0000D30604D5532304A95B182021197013073A
:108A100004D5532304A95B182B2119702B782A2B1A
:108A200016D02E0000210A20E3683278751C303AF7
:108A3000092A50D9002911D117E00136AFE7059B6B
:108A40002268C01A01238340134335002360CCE71A
:108A5000079B191D1B680791002B01DB0B9304E09A
:108A60005B42E36002231343236033782E2B0CD147
:108A700073782A2B34D1079B02361A1D1B68079284
:108A8000002B01DA01235B420993324D03222800B7
:108A9000317800F037FB002806D04023401B83408C
:108AA0002268013613432360317806222A48751C58
:108AB000217600F027FB002840D0284B002B22D144
:108AC0000722079B07339343083307936369049A8C
:108AD0009B18636162E743432E0001219B18A4E7C2
:108AE00000230A201900013663603278751C303A81
:108AF000092A03D9002BC8D00991C6E741432E00AB
:108B000001238918F1E707AA009221003A00144BCB
:108B1000039800E000BF0490049B0133D6D17B6E24
:108B2000DB0705D4BB899B0502D4B86DFFF7D0FDE8
:108B3000BB895B0600D51EE70D981EE707AA0092C9
:108B400021003A00064B039800F07CF8E3E7C046AA
:108B5000889900088E99000892990008000000008A
:108B600007890008F7B5160001938A680B690C00A5
:108B70000090934200DA13002200336043321278EF
:108B8000002A01D00133336023689B0602D5336885
:108B9000023333602268062315001D401A4227D095
:108BA000230043331B785A1E93412268920630D427
:108BB000220001990098089D4332A847013025D032
:108BC0000622236800251340042B05D13368E5688D
:108BD000ED1AEB43DB171D40A3682269934201DDC8
:108BE0009B1AED180026B54220D1002010E0013577
:108BF000E36832689B1AAB42D2DD2200012301995F
:108C00000098089F1932B8470130F0D10120404246
:108C1000FEBD3020E1184331087021005A1C453157
:108C20000978A218433202331170C1E722000123F0
:108C300001990098089F1A32B8470130E6D00136F2
:108C4000D1E70000F0B58BB006920A0043320793DB
:108C5000059003920A7E0C00109B782A09D8622A9C
:108C60000BD8002A00D1BAE07A490491582A00D1E1
:108C70008EE0250042352A7022E010006338152866
:108C8000F7D8F7F73DFA16001F00F6FFF6FFF6FFDC
:108C9000F6FF1F00F6FFF6FFF6FFF6FF9F00360017
:108CA0007E00F6FFF6FFB000F6FF3600F6FFF6FF97
:108CB000820025001A684235111D196013682B7057
:108CC00001239EE018680968021D0D060BD5066891
:108CD0001A60002E03DA2D23039A764213705D4B3F
:108CE0000A27049318E006681A604906F1D536B2DF
:108CF000EFE70868196840C9050602D4400600D5A8
:108D0000B6B21960534B0A2704936F2A00D1023F71
:108D10002300002243331A706368A360002B06DB34
:108D200004212268039D8A43226033430CD0039DB3
:108D300030003900F7F774FA049B013D5B5C2B703F
:108D4000330006009F42F3D9082F09D12368DB07BF
:108D500006D5626823699A4202DC3023013D2B70FC
:108D6000039B5B1B2361079B210000930598069BD7
:108D700009AAFFF7F7FE013048D1012040420BB0AD
:108D8000F0BD202209680A4322607822324904910A
:108D9000210045310A701968226840C9100602D4C2
:108DA000500600D5B6B21960D30702D5202313436D
:108DB0002360002E01D01027AAE7202223689343C6
:108DC0002360F8E71A680D68101D49691860136878
:108DD0002E0601D5196002E06D06FBD5198000232F
:108DE000039D2361BFE71A68111D196015680021F2
:108DF0002800626800F086F9002801D0401B6060FE
:108E0000636823610023039A1370ACE72A00236987
:108E100006990598079DA8470130AED023689B07A7
:108E200015D4099BE0689842A9DA1800A7E7220048
:108E3000012306990598079E1932B04701309CD04E
:108E40000135E368099A9B1AAB42F0DCE9E700259B
:108E5000F7E7C04699990008AA990008F7B50C22CF
:108E60008B5E05000C001A0756D44A68002A02DC03
:108E70000A6C002A4EDDE76A002F4BD000228020CA
:108E80002E682A601A004001216A0240034233D052
:108E9000626DA3895B0706D56368D21A636B002BEA
:108EA00001D0236CD21A00232800E76A216AB84750
:108EB000A289431C06D129681D2946D8294BCB40DD
:108EC000DB0742D50023636023692360D20405D504
:108ED000431C02D12B68002B00D16065616B2E60B2
:108EE000002917D023004433994202D02800FFF70D
:108EF000F9FB002363630DE001232800B84702005B
:108F0000431CC6D12B68002BC3D01D2B01D0162BC0
:108F10001AD12E6000201EE00E69002EFAD00F68D4
:108F20000E60BA1B019200229B0700D14A69A26021
:108F3000019B002BEEDDA36A32001F002800019B7D
:108F4000216AB847002807DCA28940230120134387
:108F50001BB2A3814042FEBD019B36181B1A019330
:108F6000E6E7C046010040200B6970B505000C0023
:108F7000002B02D10025280070BD002804D0036A10
:108F8000002B01D1FFF772F90C22A35E002BF1D068
:108F9000626ED20704D49B0502D4A06DFFF797FB45
:108FA00028002100FFF75AFF636E0500DB07E2D4BB
:108FB000A3899B05DFD4A06DFFF78AFBDBE70000E8
:108FC00070B50E001D000E23C95E140096B0002976
:108FD0000CDAB2898023110019401A4214D180237F
:108FE000DB0000202960236016B070BD6A4600F0E7
:108FF00053F80028EDDBF02301991B021940044BC4
:10900000C9184B425941EAE700214023E9E7C0462D
:1090100000E0FFFFF0B502268B8905000C0085B04B
:10902000334207D023004733236023610123636168
:1090300005B0F0BD03AB02AAFFF7C2FF029F01908B
:1090400039002800FFF7BAFB002808D10C22A35EE4
:109050009A05EDD4032293431E43A681E2E78023C1
:10906000A28920601343A381039B20616761002BC9
:109070000CD028000E23E15E00F020F8002805D077
:109080000323A2899A43023B1343A381A389019A34
:109090001343A381CCE70000002370B5064D040004
:1090A000080011002B60F7F77DFB431C03D12B68F0
:1090B000002B00D0236070BD38B80020002370B5AD
:1090C000064D040008002B60F7F77AFB431C03D120
:1090D0002B68002B00D0236070BDC04638B800203C
:1090E000002370B5064D040008002B60F7F77CFBE9
:1090F000431C03D12B68002B00D0236070BDC046F9
:1091000038B80020C9B28218904201D100207047BF
:1091100003788B42FBD00130F6E70000F8B5C0467B
:10912000F8BC08BC9E467047F8B5C046F8BC08BC01
:109130009E4670470000000001B40248844601BC0E
:10914000604700BF69000020626F6F74696E672E10
:109150002E2E0D006F74615F6D6F64756C655F69B5
:109160006E6974206661696C65643A2025640D0A35
:1091700000000000626F6F745F70726570726F63E1
:10918000657373206572722025640D0A000000006B
:10919000596D6F64656D20776169740D0000000082
:1091A000486172644661756C740D00003F000000F8
:1091B0005B594D5D2072657365743A2025730D0A05
:1091C000000000004F5441204F4B2C20626F6F7401
:1091D000206170702E2E2E0D000000006F74612033
:1091E00066696E697368206572722025640D0A00D5
:1091F000656F7400736571006F7461207772000091
:1092000063616E006372630073747265616D206FD9
:10921000766600006368756E6B206F7666000000EE
:10922000796D6F64656D2069646C652C207265735F
:1092300065740D0072782069646C65005B4F544161
:109240005D5B455D207265636F72645F6C6F616426
:109250003A20666C6173682072656164206661699A
:109260006C65640D000000005B4F54415D5B455D23
:10927000207265636F72645F73746F72653A206603
:109280006C617368206572617365206661696C65E5
:10929000640D00005B4F54415D5B455D207265636A
:1092A0006F72645F73746F72653A20666C61736885
:1092B000207772697465206661696C65640D0000D1
:1092C0005B4F54415D5B455D20666C6173685F6513
:1092D000726173655F736C6F743A20657261736558
:1092E000206661696C656420747970653D256C75D4
:1092F00020616464723D256C752073697A653D2533
:109300006C750D0A000000005B4F54415D5B455DCC
:10931000206F74615F6D6F64756C655F696E6974F1
:109320003A206D697373696E6720636F6E66696753
:109330002066756E6374696F6E20706F696E7465F8
:1093400072730D005B4F54415D5B455D206F74612E
:109350005F6D6F64756C655F626F6F745F7072656F
:1093600070726F636573733A206E6F20626F6F74F3
:109370002063616E6469646174650D005B4F5441E4
:109380005D5B455D206F74615F646F776E6C6F61CC
:10939000645F73746172743A207061636B616765B6
:1093A000206D6167696320696E76616C69640D0088
:1093B0005B4F54415D5B455D206F74615F646F7707
:1093C0006E6C6F61645F73746172743A206865617A
:1093D0006465722063726320696E76616C69640DE6
:1093E000000000005B4F54415D5B455D206F746180
:1093F0005F646F776E6C6F61645F73746172743AEF
:10940000206E6F20746172676574204F5441207321
:109410006C6F7420617661696C61626C650D00002F
:109420005B4F54415D5B455D206F74615F646F7796
:109430006E6C6F61645F73746172743A20617070F6
:109440005F6F6666736574206F7574206F66207237
:10945000616E67650D0000005B4F54415D5B455DCB
:10946000206F74615F646F776E6C6F61645F73749B
:109470006172743A206170705F6F66667365742BF9
:109480006170705F73697A65206578636565647380
:1094900020736C6F740D00005B4F54415D5B455D44
:1094A000206F74615F646F776E6C6F61645F73745B
:1094B0006172743A206170705F73697A6520746FAD
:1094C0006F206C617267650D000000005B4F5441B6
:1094D0005D5B455D206F74615F646F776E6C6F617B
:1094E000645F73746172743A2065726173655F6C56
:1094F000656E206578636565647320736C6F740DA9
:10950000000000005B4F54415D5B455D206F74615E
:109510005F646F776E6C6F61645F73746172743ACD
:1095200020666C617368206572617365206661698D
:109530006C65640D000000005B4F54415D5B455D50
:10954000206F74615F646F776E6C6F61645F7374BA
:109550006172743A207265636F72645F73746F72C4
:1095600065206661696C65640D0000005B4F5441C5
:109570005D5B455D206F74615F646F776E6C6F61DA
:10958000643A207265636F72645F6C6F6164206619
:1095900061696C65642072633D25640D0A000000FA
:1095A0005B4F54415D5B455D206F74615F646F7715
:1095B0006E6C6F61643A20746172676574207374B5
:1095C00061747573206D69736D617463683D2564A2
:1095D0000D0A00005B4F54415D5B455D206F746177
:1095E0005F646F776E6C6F61643A206F6666736557
:1095F00074206D69736D61746368206578703D25B2
:109600006C7520676F743D256C750D0A00000000B5
:109610005B4F54415D5B455D206F74615F646F77A4
:109620006E6C6F61643A2073697A65206D69736D41
:1096300061746368206F66667365743D256C752080
:1096400073697A653D256C7520746F74616C3D2576
:109650006C750D0A000000005B4F54415D5B455D79
:10966000206F74615F646F776E6C6F61643A206421
:1096700073742061646472206F7574206F66207348
:109680006C6F742072616E67650D00005B4F544112
:109690005D5B455D206F74615F646F776E6C6F61B9
:1096A000643A20666C61736820777269746520661D
:1096B00061696C65640D00005B4F54415D5B455D05
:1096C000206F74615F646F776E6C6F61645F666951
:1096D0006E6973683A20746172676574207374618F
:1096E000747573206D69736D617463683D25640DD5
:1096F0000A0000005B4F54415D5B455D206F746163
:109700005F646F776E6C6F61645F66696E697368C2
:109710003A2073697A65206D69736D61746368209E
:10972000646F776E6C6F616465643D256C75206550
:10973000787065637465643D256C750D0A000000E2
:109740005B4F54415D5B455D206F74615F646F7773
:109750006E6C6F61645F66696E6973683A206372EC
:1097600063206D69736D6174636820666C617368F2
:109770003D256C752065787065637465643D256C66
:10978000750D0A005B4F54415D5B455D206F746150
:109790005F646F776E6C6F61645F61626F72743A61
:1097A000206E6F20646F776E6C6F6164696E6720E6
:1097B000736C6F7420666F756E640D005B4F54415F
:1097C0005D5B455D206F74615F646F776E6C6F6188
:1097D000645F61626F72743A207461726765745F6E
:1097E0006964783D256C750D0A0000005B4F54419B
:1097F0005D5B455D206F74615F6170705F6D61726C
:109800006B5F76657269666965643A206E6F205594
:109810004E5645524946494544206F746120736C49
:109820006F740D005B4F54415D5B455D206F74614B
:109830005F6170705F6D61726B5F7665726966699A
:1098400065643A207265636F72645F73746F7265EA
:10985000206661696C65640D00000000666C6173D0
:10986000682070726F6772616D20696E76616C69D5
:109870006420302D3E31206174202530386C780D05
:109880000A000000666C6173682070726F67726115
:109890006D206661696C6564206174202530386CC8
:1098A000780D0A0000000000000000000000000029
:1098B00000000000000000000000000000000000A8
:1098C0000000000001000000020000000300000092
:1098D000040000000600000007000000080000006F
:1098E000090000000000000000000000000000006F
:1098F0000000000001000000020000000300000062
:1099000004000000010002000400060008000A0034
:109910000C00100020004000800000010101010344
:109920000701000008040204080101014F544154DA
:109930000300000000000000010800000700000014
:1099400000000000000000000000000000E000082F
:1099500000000008000000000000000000000800F7
:1099600000000000000000000008000000000000EF
:1099700000000000ED7E00083D7F00080580000823
:109980003D800008A5800008232D302B2000686C46
:109990004C00656667454647003031323334353612
:1099A000373839414243444546003031323334354B
:1099B000363738396162636465660000E10000088B
:1099C000B90000080024F4000400000001000000B9
:1099D0000000000003000000FCB600201C00002076
:1099E00000000000FCB6002064B70020CCB70020C7
:1099F0000000000000000000000000000000000067
:109A00000000000000000000000000000000000056
:109A10000000000000000000000000000000000046
:109A200000000000000000000000000080B588B0C9
:109A300000AF786039601F23FB1800221A707B6822
:109A4000BB613B687B611A4B5A69194B8021C90283
:109A50000A435A61EFF31083FB60FB683B6172B607
:109A6000C0460FE07A69BB6912681A607B690433EB
:109A70007B61BB690433BB611F217B181A787B189B
:109A800001321A701F23FB181B783F2BEAD9C046FE
:109A9000074B1A69C0239B021340F9D13B69BB6095
:109AA000BB6883F31088C046C046BD4608B080BD81
:049AB0000020024050
:10E00000FFFFFFFFFFFFFFFFFFFFFFFFFFFFFFFF20
:10E01000FFFFFFFFFFFFFFFFFFFFFFFFFFFFFFFF10
:10E02000FFFFFFFFFFFFFFFFFFFFFFFFFFFFFFFF00
:10E03000FFFFFFFFFFFFFFFFFFFFFFFFFFFFFFFFF0
:020000040801F1
:100000004F54415461C0616A000200000C64020058
:100010006D000AC7302E312E3700000000000000AE
:1000200000000000000000000000000000000000D0
:1000300000000000F9DD5E0E00000000000000007E
:1000400000000000000000000000000000000000B0
:1000500000000000000000000000000000000000A0
:100060000000000000000000000000000000000090
:100070000000000000000000000000000000000080
:100080000000000000000000000000000000000070
:100090000000000000000000000000000000000060
:1000A0000000000000000000000000000000000050
:1000B0000000000000000000000000000000000040
:1000C0000000000000000000000000000000000030
:1000D0000000000000000000000000000000000020
:1000E0000000000000000000000000000000000010
:1000F0000000000000000000000000000000000000
:1001000000000000000000000000000000000000EF
:1001100000000000000000000000000000000000DF
:1001200000000000000000000000000000000000CF
:1001300000000000000000000000000000000000BF
:1001400000000000000000000000000000000000AF
:10015000000000000000000000000000000000009F
:10016000000000000000000000000000000000008F
:10017000000000000000000000000000000000007F
:10018000000000000000000000000000000000006F
:10019000000000000000000000000000000000005F
:1001A000000000000000000000000000000000004F
:1001B000000000000000000000000000000000003F
:1001C000000000000000000000000000000000002F
:1001D000000000000000000000000000000000001F
:1001E000000000000000000000000000000000000F
:1001F00000000000000000000000000000000000FF
:1002000000400220D9EE0208C9320108D1320108AB
:1002100000000000000000000000000000000000DE
:10022000000000000000000000000000CD7C01087C
:100230000000000000000000F17D010805830108B6
:1002400029EF02080000000029EF020829EF020848
:1002500029EF020829EF0208E5320108FB32010804
:1002600029EF0208253301083D33010861330108F5
:10027000B533010829EF020829EF02080000000049
:1002800029EF020829EF020829EF020829EF0208E6
:1002900029EF020829EF0208CD33010829EF0208EF
:1002A00029EF0208E533010829EF0208FD330108B0
:1002B000153401082D340108000000000000000082
:1002C00010B5064C2378002B07D1054B002B02D02C
:1002D000044800E000BF0123237010BD8C03002000
:1002E00000000000A82B0308044B10B5002B03D01E
:1002F0000349044800E000BF10BDC04600000000F4
:1003000090030020A82B030802780B78002A03D062
:10031000013001319A42F7D0D01A70470023C25CF5
:100320000133002AFBD1581E7047000002B4714609
:1003300049084900095C49008E4402BC7047C04628
:1003400003B47146490840004900095E49008E44E3
:1003500003BC7047002243088B4274D303098B42CD
:100360005FD3030A8B4244D3030B8B4228D3030C85
:100370008B420DD3FF22090212BA030C8B4202D327
:100380001212090265D0030B8B4219D300E0090A4F
:10039000C30B8B4201D3CB03C01A5241830B8B4258
:1003A00001D38B03C01A5241430B8B4201D34B0341
:1003B000C01A5241030B8B4201D30B03C01A5241A6
:1003C000C30A8B4201D3CB02C01A5241830A8B422B
:1003D00001D38B02C01A5241430A8B4201D34B0214
:1003E000C01A5241030A8B4201D30B02C01A524178
:1003F000CDD2C3098B4201D3CB01C01A524183092C
:100400008B4201D38B01C01A524143098B4201D365
:100410004B01C01A524103098B4201D30B01C01A90
:100420005241C3088B4201D3CB00C01A524183080A
:100430008B4201D38B00C01A524143088B4201D337
:100440004B00C01A5241411A00D201465241104697
:100450007047FFE701B5002000F0F0F802BDC0468C
:100460000029F7D076E7704703460B437FD400227C
:1004700043088B4274D303098B425FD3030A8B4238
:1004800044D3030B8B4228D3030C8B420DD3FF22A2
:10049000090212BA030C8B4202D31212090265D070
:1004A000030B8B4219D300E0090AC30B8B4201D323
:1004B000CB03C01A5241830B8B4201D38B03C01A6A
:1004C0005241430B8B4201D34B03C01A5241030BE1
:1004D0008B4201D30B03C01A5241C30A8B4201D392
:1004E000CB02C01A5241830A8B4201D38B02C01A3D
:1004F0005241430A8B4201D34B02C01A5241030AB4
:100500008B4201D30B02C01A5241CDD2C3098B4298
:1005100001D3CB01C01A524183098B4201D38B0115
:10052000C01A524143098B4201D34B01C01A5241B8
:1005300003098B4201D30B01C01A5241C3088B42FD
:1005400001D3CB00C01A524183088B4201D38B00E8
:10055000C01A524143088B4201D34B00C01A52418A
:10056000411A00D201465241104670475DE0CA0F61
:1005700000D04942031000D34042534000229C4621
:1005800003098B422DD3030A8B4212D3FC2289012B
:1005900012BA030A8B420CD3890192118B4208D301
:1005A000890192118B4204D389013AD0921100E063
:1005B0008909C3098B4201D3CB01C01A5241830977
:1005C0008B4201D38B01C01A524143098B4201D3A4
:1005D0004B01C01A524103098B4201D30B01C01ACF
:1005E0005241C3088B4201D3CB00C01A5241830849
:1005F0008B4201D38B00C01A5241D9D243088B429F
:1006000001D34B00C01A5241411A00D20146634641
:1006100052415B10104601D34042002B00D54942A5
:10062000704763465B1000D3404201B5002000F0E4
:1006300005F802BD0029F8D016E770477047C0469C
:100640008446100062468C461900634600E0C046AE
:100650001FB501F079FC002801D40021C8421FBD5C
:1006600010B501F0BDFB4042013010BD10B501F0E6
:100670006BFC002801DB002010BD012010BDC0462E
:1006800010B501F061FC002801DD002010BD012043
:1006900010BDC04610B501F0E7FB002801DC0020CA
:1006A00010BD012010BDC04610B501F0DDFB0028D3
:1006B00001DA002010BD012010BDC04684460800AC
:1006C0006146FFE71FB500F0A5FA002801D400211C
:1006D000C8421FBD10B500F02DFA4042013010BDD8
:1006E00010B500F097FA002801DB002010BD0120B2
:1006F00010BDC04610B500F08DFA002801DD0020C5
:1007000010BD012010BDC04610B500F03BFA002816
:1007100001DC002010BD012010BDC04610B500F066
:1007200031FA002801DA002010BD012010BDC046BA
:10073000002B11D1002A0FD1002900D1002802D0AE
:100740000021C943080007B4024802A140180290E2
:1007500003BDC046E9FEFFFF03B4684601B5029839
:1007600000F006F8019B9E4602B00CBC7047C046E4
:10077000F0B557464E464546DE46E0B504000D004E
:100780009246994683B08B4230D82DD04946504688
:1007900002F0D0FC29000600200002F0CBFC331A46
:1007A0009846203B34D49B4653465A469340424693
:1007B0001F00534693401E00AF423BD8AF4200D1CA
:1007C00079E05B46A41BBD41002B00DA76E00022F5
:1007D00000230092019301235A4693400193012381
:1007E00042469340009329E08242CFD90022002361
:1007F000009201930C9B002B01D01C605D6000985F
:10080000019903B0F0BCBB46B246A946A046F0BD74
:1008100042469B4620239B1A5246DA40414613002B
:100820004A468A40170042461F43534693401E00E3
:10083000AF42C3D900220023009201934346002B0C
:10084000D8D0FB0772081A4346467B080EE0AB423D
:1008500001D1A2420CD8A41A9D41012024196D4156
:100860000021013E24184D41002E06D0AB42EED9A6
:10087000013E24196D41002EF8D1009801995B4684
:1008800000196941002B24DB2B005A464446D34013
:100890002A00E2401C005B461500002B2ADB2600E4
:1008A0009E40330026004746BE403200801A9941E0
:1008B000009001919EE7A342BCD882E742462023E4
:1008C00000219B1A0022009101920122DA4001923C
:1008D00085E7424620239B1A2A0046469A40230079
:1008E000F340444613432A00E2401C005B461500D7
:1008F000002BD4DA42462F002023260097409B1A73
:10090000DE403B003343CDE7F0B546464F46D64682
:100910004502C0B5C30F470098460E1C6D0A3F0E36
:100920005BD0FF2F21D08023ED00DB041D4300238B
:1009300099469A467F3F74027300640A1B0EF60FB5
:10094000002B20D0FF2B43D080220020E400D204D3
:1009500014437F3B4246FF1A4B4672400F2B00D98F
:100960009DE071499B00CB589F46002D5AD108232A
:100970009946063B74029A467300FF27640A1B0ED1
:10098000F60F002BDED1002C3BD101234246494615
:10099000724019430E2918D86448890041588F467F
:1009A0005346022B00D1B8E0032B6ED042462C00F8
:1009B000012B40D100200024C0052043D207104362
:1009C000E0BCBA46B146A846F0BDFF200024F3E7DC
:1009D000002C20D10223FF3FD8E7002D05D10423AE
:1009E0009946033B00279A46A5E7280002F084FBBE
:1009F0007627431F9D4000237F4299469A463F1A1F
:100A000099E7200002F078FB431F9C4076235B426D
:100A10001B1A00209EE703234A461A4391460320EF
:100A2000FC3397E70C239946093BFF279A4682E758
:100A300003282CD0320038007F30002847DD6307C0
:100A400004D00F232340042B00D00434230103D50A
:100A50003800374B80301C40FE28B6DCA401640A05
:100A6000C0B2A9E780240022FF20E403A4E780238A
:100A7000DB031D4201D01C420BD08024E4032C4335
:100A800064024246FF20640A96E746462C00802313
:100A9000DB031C4364023200FF20640A8CE76D0113
:100AA000600185422DD21B230024013F012629002D
:100AB00064006D00002901DB854201D32D1A344307
:100AC000013B002BF3D16B1E9D412C43B3E7012367
:100AD0001B1A1B2B00DD6DE721009E37D940BC405F
:100AE0000B00611E8C412343590704D00F2119408C
:100AF000042900D00433590113D49B0100205C0A5F
:100B00005AE71A2301242D1AD0E7981E4342584170
:100B1000404232000024C0B24EE74246FF2000248B
:100B20004AE70120002447E7245A0308645A0308CF
:100B3000FFFFFFF770B542004E024C0045026D0A00
:100B4000120EC30F760A240EC90FFF2A10D0FF2CF5
:100B50000CD00120A2420AD1B54208D18B420FD05D
:100B6000002A04D12800431E984100E0012070BDF6
:100B70000120FF2CFBD13543F9D14B401800F6E79B
:100B80000020F4E730B5420044024D02C30F480094
:100B9000640A120E6D0A000EC90FFF2A18D0FF2832
:100BA0000AD0002A1ED100280AD1002D29D0002CFD
:100BB0002DD14800013830BD002D25D1002A01D1AA
:100BC000002CF6D08B4219D001205B421843F2E78B
:100BD000002C19D1FF28F7D1002D15D100208B4210
:100BE000F2D1E8E70028EFD08B42EDD18242EBDC76
:100BF00004DBAC42E8D80020AC42DCD2580001381B
:100C0000D9E7002CD7D0DFE702204042D3E78B4260
:100C1000DAD1EEE730B5420044024D02C30F48007E
:100C2000640A120E6D0A000EC90FFF2A17D0FF28A2
:100C30000AD0002A1BD100280AD1002D1DD0002C7B
:100C40002DD14800013811E0002D0ED1002A01D12C
:100C5000002CF6D08B420CD15800013806E0002C55
:100C600003D1FF2805D1002D15D0022030BD00286A
:100C700006D101205B421843F8E7002CF6D0F8E7D4
:100C80008B42F6D18242F4DCE6DBAC42F1D80020A4
:100C9000AC42EBD2E0E700208B42EAD1E6E78B42A0
:100CA000E7D1F2E7F0B54F464646D6464400C0B518
:100CB00046020F1C760A240EC50F002C00D1DAE084
:100CC000FF2C74D08023F600DB041E4300239946DA
:100CD0009A467F3C7B025B0A98467B001B0EFF0F07
:100CE000002B74D0FF2B00D18EE042468021D20031
:100CF000C90411437F3B2A00E4184B467A408846DA
:100D0000D2B20A2B75DC4B460020022B0FDD494680
:100D100001238B40A621C9000B4269D19021890093
:100D20000B4200D000E18821194200D0F5E0414695
:100D30000904090C43460800350C36041B0C360C1C
:100D4000704369435E435D437618030C9B199942D7
:100D500003D9802149028C46654400041904000C23
:100D600009188E01701E86411B0C890E5B190E43FB
:100D70009B011E431B016CD423007F33002B00DC3E
:100D8000B1E0150071070BD00F202100304004287E
:100D900006D00436320103D56E4B1E400B00803363
:100DA000FE2B00DDBDE0B201520ADBB248E0002EAE
:100DB00000D092E008239946063B9A467B025B0AE4
:100DC00098467B00FF241B0EFF0F002B8AD1424662
:100DD000002A64D149460132114389460A2908DCB8
:100DE0007D400120EAB2022991DC1500002227E0B3
:100DF00015005346022B00D193E0032B1AD0012B90
:100E00002CD1002300221BE04346FF34002B55D099
:100E100003214B460B4319000A2B00DC92E00F2BF9
:100E200000D08CE08022D203164203D04346134206
:100E300000D17DE08022D20332435202520AFF23C6
:100E4000D805ED0710432843E0BCBA46B146A84692
:100E5000F0BD0123150071081E400E4323008033AE
:100E6000611C002B41DD720794D00F223240042A0E
:100E700000D08EE78EE7002E05D104239946033B70
:100E800000249A4626E7300002F036F97624431F04
:100E90009E400023644299469A46241A1AE7404627
:100EA00002F02AF94B46241A763C0A2BA1DC434671
:100EB000053883407D409846EAB224E74A4602332B
:100EC00013432A007A40D2B20A2B92DC494615001D
:100ED000002926D09946022019E70C239946093BA0
:100EE000FF249A46F6E6150021000122D31A1B2B97
:100EF00000DD86E79E3132008E40DA40731E9E414F
:100F00003243530704D00F231340042B00D0043284
:100F1000530110D50123002292E73D004646824648
:100F200067E7FF2300228BE780220025D20386E7B4
:100F30003D001A4383E792010023520A80E73D00F7
:100F4000464677E72A0001237A408B400320D2B23D
:100F5000E9E6C046FFFFFFF741024200C30F490A1E
:100F60000020120E7E2A03DD9D2A02DD094A981810
:100F70007047802000040143952A07DC9620821ADE
:100F8000D1404842002BF3D10800F1E7963A914056
:100F9000F7E7C046FFFFFF7F10B5041E0DD002F03B
:100FA000ABF89E231B1A962B0CDC082834D008388B
:100FB00084406402640AD8B201E000200024C00525
:100FC000204310BD992B13DC421F9440144A224049
:100FD00061071CD00F212140042918D00432D40805
:100FE000520115D59F236402181A640AC0B2E6E7BD
:100FF000020021001B3291400A00511E8A41052146
:10100000091ACC401443064A22406107E2D1D408B1
:101010006402640AD8B2D2E76402640A8E30CEE772
:10102000FFFFFFFBF0B54F464646D646C0B582B03F
:10103000009001910E034C00CD0F710A009E5F00DD
:10104000760F0E43009900920193C9008946190357
:101050007B0D9846019B490ADB0F9C46009B009A3A
:101060005B0F0B434146640DD200611A654500D108
:10107000A6E0002972DD4746002F00D1DDE0CC4F0D
:10108000BC4200D19AE10127382917DC80273F04B0
:101090003B431F2900DDDDE12027781A1F00874030
:1010A000BA461700CF40844638005746074360468B
:1010B0008240CB40501E8241F61A17434B46DF1B3D
:1010C000B94580414042361A330200D4FFE076022F
:1010D000760A002E00D13CE1300002F00DF803004A
:1010E000083B20213800CA1AD0409E4002009F4091
:1010F00032439C4200DDA6E1181B0130091A3E0074
:101100008F40C6407B1E9F4113008B4037431F43D7
:10111000C2403B0016000024134300D1DFE17B07EF
:1011200000D132E30F233A003B40042B04D03A1D98
:10113000BA42BF417F42F619330200D423E39C4BED
:1011400001349C4200D1B4E09A4B64051E40640D0A
:101150007707D20876021743360BACE0002900D19E
:101160007EE04146091B002C00D060E13400484677
:10117000044300D1C9E14C1E012900D12EE28C4D5F
:10118000A94200D124E20127382C11DC21001F29BB
:1011900000DD0BE2202437004846641AA740C8400F
:1011A00007434846A040CE40441EA0419B1B074336
:1011B000D71BBA4292415242654644469E1A83E783
:1011C000002900DC9CE04746002F67D11F00174331
:1011D00000D1E4E0481E012900D19BE1744FB942DF
:1011E00000D1EBE001270100382811DC1F2900DDC8
:1011F000C7E12027781A1F00844687401000C840A6
:10120000074360468240CB40501E8241F618174388
:101210004F444F45804140423618330257D5644B06
:1012200001349C4245D00121624B7A081E4039406E
:101230000A43F7071743760871E71F00174300D1E9
:10124000ADE04F1EBC46012900D182E1584FB942A2
:1012500000D190E161460127382900DD2EE718E72B
:10126000554F611C394200D0D0E0310048461F0084
:1012700001431743002C00D03DE1002900D1BCE11F
:10128000002F00D0BFE14B460021D8087707074365
:10129000F00806034C05360B640D0CE0444FBC42CD
:1012A00000D18BE001273829B2DC80273F043B4383
:1012B0009CE70026002724053443ED072C43380023
:1012C000210002B0E0BCBA46B146A846F0BD7B079B
:1012D00004D00F233B40042B00D028E7F808344B00
:1012E00077070743F0089C4200D04AE23B000343E3
:1012F00059D080263603064336032D4C360BDAE7E9
:10130000002961D04146091B002C00D1B9E0284CCE
:10131000A04500D1A5E10127382913DC802424044D
:1013200026431F2900DDC8E1202437004846641AFF
:10133000A740C84007434846A040CE40441EA041B5
:101340009B190743BF189742924152424446D61810
:1013500063E7380001F0D0FE030018331F2B00DCD8
:10136000BFE63A00083882409C4200DD83E01B1B48
:10137000581C1F2800DCB4E117001F3BDF40202869
:1013800005D040231B1A9A40531E9A41174300244C
:10139000002F0AD07B0700D0C4E626009EE74B460C
:1013A0000C00D8089BE70027014C002683E7C046C5
:1013B000FF070000FFFF7FFFFE0700004B46770797
:1013C000D8080743F00891E7CD4F611C39426BD133
:1013D000310048460143002C00D04BE11F00174369
:1013E000002900D181E1002F00D14CE74A444A4551
:1013F0008041F61840423618330200D5B0E117009C
:101400009146374300D03EE7002654E74946891A03
:101410008846C145BF41F11A7F42C91B0F0261D402
:1014200047460F4300D1BDE00E00474651E6B54C9C
:10143000A04500D100E10127382900DDB8E680246D
:1014400024042643A3E6B04EE41A16407B0700D0DE
:101450003FE743E70F001800203FF840844620296B
:1014600003D04027791A8B401A43531E9A41634692
:1014700017001F4322E6A448E11A10404707C0089E
:1014800007E734004846044300D1FAE04C1E012926
:1014900000D1D7E09B4FB94200D1E2E00127382CC0
:1014A00000DD4FE721003CE7964CA14200D1DDE092
:1014B0004A444A458041F31840421818C707520869
:1014C00017434608520705D00F220C003A40042A61
:1014D00000D02CE67607FF0837430009D9E600273D
:1014E0000026E8E64946571ABA4292419E1B5242EC
:1014F0006546B61AEDE5002900D0C6E0002F67D199
:10150000802600257F4C3603D5E665460C001E007C
:10151000D008E4E64A444A458041F318404218188E
:101520001100030200D496E0774B49081840C30726
:101530000B434408490700D129E10F221A40042A2D
:1015400000D1EAE01F1D9F42B641764236190224BF
:10155000C4E649468F1AB9458041F61A4042361A08
:10156000330206D47307FF0801211F43F00890E6F9
:1015700065460124ABE54B467707D8080743F008DA
:10158000B4E60F001800203FF8408446202903D01D
:101590004027791A8B401A43531E9A41634617001D
:1015A0001F4335E600250024002684E60C003500A4
:1015B000203CE540202905D04024611A8E40494650
:1015C000314389464846411E884107002F43EFE5D5
:1015D000D2085F0765461743D80887E6171ABA424C
:1015E00092419E1B5242B61A3302C1D47307FF08C0
:1015F000654601211F43F0084BE6002F7BD065466E
:101600001E0091463FE6811A8846C145A441F11A61
:101610006442091B80242404214277D0101A82429C
:10162000924107009E1B5242B61A374300D0A0E0F9
:101630006546002400263EE65F07D208654617434C
:10164000D80853E6811891429241F018524280180E
:10165000030200D568E74707C9080F43C008012106
:1016600017E6D2085F071743D8083FE60C000026AC
:10167000002720E6002956D15F07D2081743D80873
:1016800034E60C001E00D00829E6C10870070143AB
:10169000F008002F62D080242403204207D0DE0807
:1016A000264204D165463000D1085B0719434F0F2D
:1016B000C900C9087F070F4318E60C003000203C22
:1016C000E0408446202905D04024611A8E404946D6
:1016D000314389464846411E8841614607000F4311
:1016E00030E620210027091A0EE51E00002F00D049
:1016F00022E5002458E7002500240026DBE5C0464B
:10170000FE070000FF070000FFFF7FFF47460F4373
:1017100000D147E70E00C146B5E5DF0864070221A6
:1017200027430009B5E51900C008770707431143AF
:10173000F008002900D1D9E580210903084207D02B
:10174000DC080C4204D1D2085B071A4317002000C2
:101750007B0FFF00FF085B071F43C7E50F00C5E5D0
:10176000124BD20833405F075B02012417431E0B64
:10177000A1E5264212D00D4B6546020001241E4011
:10178000E6E4210085E51700A8E53A00D4E4DB088B
:1017900064071C432700022100097AE5C008770787
:1017A000074365460021F00873E5C046FFFF7FFF51
:1017B000F0B5DE46454657464E46E0B587B0009246
:1017C00001930B031B0B9B46CA0F4B000400804682
:1017D0005B0D029200D198E07C4A934237D0594683
:1017E000420FC9000A43802109041143C2009046F8
:1017F000774A894692469A44002300240393009E28
:10180000019F3B031B0B9B467B0030005B0DFD0FD4
:10181000002B59D06D4A934248D05946720FC900E7
:101820000A438021090411438B466949F2008C4622
:1018300051466344CB1A9A460021029E6E40F6B28E
:101840000F2C00D9CEE0634BA4001B599F465A468B
:101850000243914600D090E09A4602239046082425
:101860000393CCE7CB464246029D0399022900D15F
:10187000DEE1032900D18DE0012900D079E12E00BD
:1018800000220023002490461B052343F607334320
:101890004046190007B0F0BCBB46B246A946A04678
:1018A000F0BD002200249046484BEDE75A46009BCD
:1018B0001A43494B9C46E244002A59D102231C4357
:1018C000002302219B46B8E75A46009B1A4349D0A1
:1018D0005B46002B00D19CE1584601F00DFC020054
:1018E00003000B3A1D27009EBA1A19005846D6402D
:1018F00008398840320002439346009A8A403749AB
:1019000053448A4600219A4497E75B46034399462D
:1019100021D05B46002B00D169E1584601F0ECFB79
:101920000B235B429C460200844466461D239B1B9E
:10193000260011005846DE40083988403300034332
:10194000994623008B409846254B00249B1A9A46C3
:101950000023039353E7002398469A460133042457
:1019600003934CE701231C43002301219B4664E7BA
:101970000323320003211C435FE79A460323D94621
:101980000C2403933BE700238024984600260F4B4A
:10199000240379E780245B4624031C4324032E00A0
:1019A00090460A4B240B6FE780244B4624032342C6
:1019B00002D05B462342F0D080244B4624031C43D4
:1019C0002403029E014B240B5EE7C046FF07000084
:1019D00001FCFFFFA05A030801F8FFFFF30300001A
:1019E0000DFCFFFFCB4500D2F8E000D1F3E001236E
:1019F0005B429C46444648460025E2445B46170E3F
:101A00001B021F43190C3B04120200971F0C914646
:101A100002910397FEF724FD02007A430B04210C88
:101A2000804619438A4209D9009F0123BC465B4284
:101A300061449C46E0448F4200D85CE1881A0299D8
:101A4000FEF70EFD039A240442430904240C03000C
:101A50000C43A24206D90099013B8C466444A14242
:101A600000D842E1A01A424612041A4393464B465C
:101A700059461B0C1F0004930B0449460904090C2A
:101A80000C001B0C5C43120C7B43884651437A4389
:101A9000270CBC465B186344994203D98021490254
:101AA0008C466244190C24041B04240C8A181C194B
:101AB000904202D316D1A54214D25B46009F013B4F
:101AC0004D4405934D459B41BC465B426344C01861
:101AD000874200D302E1824200D929E100D124E10A
:101AE000059B9B462C1BA542AD41009B801A6D4275
:101AF000401B834200D10FE10299FEF7B1FC039A2B
:101B00000B044243210C050019438A4200D9CBE063
:101B1000881A0299FEF7A4FC039A2404424309049C
:101B2000240C03000C43A24200D9CAE04146A41A87
:101B30002A041A43049F13041B0C594340467B4359
:101B40009C46150C68430B0C844463447D439842C7
:101B500003D98020400284466544180C09041B0404
:101B6000090C40195B18844227D323D00123350088
:101B70001A43944B5344002B60DD510700D086E09C
:101B80002E00D1085A46D20106D55A468E4B1A402D
:101B900080239346DB0053448C4A934200DD80E669
:101BA0005A4652070A4390465A465B055402240B94
:101BB0005B0D69E63500002BDBD0009D511EAC4665
:101BC0006444AC4200D29EE0844200D2E1E000D105
:101BD000EEE00A00CAE7424500D908E74B46DC07B9
:101BE000580843465B081C434346DD0706E701F0FF
:101BF00083FA15239C4684440200634620321C2B42
:101C000000DC92E62300083883409946002398467A
:101C10009AE601F071FA02000300153220331C2A03
:101C200000DC5FE600990838814000228B4666E6BA
:101C300000222E0000249046654B25E62E0001214F
:101C4000C91A382900DD1BE61F297EDC6148140013
:101C500050445B4682408340CC40501E8241234327
:101C60001A435B46CB40510709D00F21114004298C
:101C700005D0111D9142924152429B180A0019024F
:101C800000D49BE00022012300249046FCE50F21B4
:101C90001140042900D173E7111D91429241524233
:101CA0002E00C90893446DE7009B013D9C466144AA
:101CB0008B4200D92CE78A4200D829E7851E61446F
:101CC00026E70099013B8C466444A14200D92DE7E8
:101CD000A24200D82AE7831E644427E7874200D047
:101CE000FEE6A94500D9FBE6F5E6A24200D8B9E632
:101CF000831E6444B6E68A4200D89FE6BC46831E33
:101D0000984661449AE60A00844200D02EE74B458B
:101D100000D02BE735002CE72A4B2F4A534492453D
:101D200043DB0122002193442CE7AC4200D8D7E6E4
:101D300002235B429C4600994D444D459B41E34440
:101D40008C465B426344C018CCE61F204042C31A55
:101D50005846D840202904D05946204B5344994036
:101D60000A43531E9A4107231900024300241140DD
:101D7000134209D008331340042B1DD0131D934286
:101D800089411A0049424907D2080A439046002374
:101D90007AE54946009F4D004D458941BC46494280
:101DA0006144A946023A6418AEE70122524246E76E
:101DB0009945EED30A00AAE70021E5E759075B023F
:101DC0001C0BE1E7FF030000FFFFFFFEFE07000022
:101DD000FF0700001E04000002FCFFFF3E0400009D
:101DE000F0B55746DE464E464546E0B50D000400C8
:101DF000E80F83460903D80F090B824619488C4621
:101E00001F0369005E00490D3F0B760D814218D01B
:101E100086420FD00120B1420DD1BC450BD1944276
:101E200009D1D3451CD0002905D160462043431E6B
:101E3000984100E00120F0BCBB46B246A946A0464E
:101E4000F0BD01208E42F6D1614639430F001743A1
:101E50002743F0D15B465246981A431E9841EAE761
:101E60000020E8E7FF070000F0B557464E4645461C
:101E7000DE46E0B50D000E034900490D8A46DF0F2E
:101E8000E90FBC4683B02F4F0400804601915800F3
:101E900019039146360B090B400DBA451DD0B842C7
:101EA0000DD05746002F2AD13443002824D10A43AD
:101EB00036D0002C41D163465800013815E011435B
:101EC00038D15346002B01D12643F4D0019B634502
:101ED00007D1019B5800013807E026432AD150451D
:101EE00021D00120019B5F42384303B0F0BCBB46C8
:101EF000B246A946A046F0BD002CDCD0E6E700289B
:101F0000EFD0019B6345ECD18245EADCE1DB8E42F8
:101F1000E7D8DED1C845E4D80020C845E5D2D8E7E7
:101F2000002CE2D0DDE7114304D1019B6345D8D1F9
:101F30000020DAE702204042D7E7019B6345E6D064
:101F4000CFE7C046FF070000F0B557464E4645466E
:101F5000DE46E0B50D000E034900490D8A46DF0F4D
:101F6000E90FBC4683B02E4F040080460191580013
:101F700019039146360B090B400DBA451ED0B842E5
:101F80000DD05746002F27D13443002833D10A43C0
:101F900034D0002C40D163465800013815E011437D
:101FA00012D15346002B01D12643F4D0019B634547
:101FB0001DD00120019B5F42384306E0264303D138
:101FC0005045F6D111431CD0022003B0F0BCBB46F3
:101FD000B246A946A046F0BD0028EAD0019B634561
:101FE000E7D18245E5DC02DB8E42E2D80ED0019BD0
:101FF00058000138E9E7002CCDD0D7E7002CE4D019
:10200000D7E7019B00206345DFD0D2E7C845D0D891
:102010000020C845D9D2EAE7019B6345E4D0C8E770
:10202000FF070000F0B557464E46DE464546E0B590
:102030001F000B031B0B16009A46CA0F4B0004002F
:10204000914685B05B0D00D1CFE1CD4A934255D08A
:102050005146420FC9000A43802109041143C200BE
:102060009046C84A8A4693469B4400230025029323
:102070003C037B00FA0F0196240B5B0D009200D10C
:1020800088E1BF4A934200D192E0BE4A944663443D
:102090009B440A2D42DCE400730F2343802449460D
:1020A00024041C43F3000193009B00205940CBB251
:1020B0000393022D00DC94E00123AB401D00A62316
:1020C0002A00DB001A401D4200D029E290239B0029
:1020D0001D4200D14DE20023802499462403A84BE1
:1020E00010004A461B052343D2071343190005B0CD
:1020F000F0BCBB46B246A946A046F0BD52460243DC
:10210000904600D0ACE19B460223924608250293FC
:10211000AEE7009BA2469946019B9846029B022B84
:1021200000D1CAE1032B00D192E1012B10D1002391
:1021300000240022D4E701227B083A401343524690
:10214000D2071343984653465B089A46039B994629
:102150005B46581C8023DB005B44002B00DCB1E1B4
:10216000424652070BD00F2241460A40042A06D0AD
:102170004246111D41459241884652429244524680
:10218000D20106D55246804B1A4080239246DB008E
:10219000C3187E4A934200DD8FE14246D108524681
:1021A00052070A4351465B054C02240B5B0D97E72F
:1021B000734B26439C46E344002E00D16FE103237A
:1021C00049461D43009B5940CBB203930A2D00DDC5
:1021D00033E10123AB401D000323029388222A42EE
:1021E00097D1424643461204120C160001981D0C6A
:1021F000030C0004000C4643B4461E006E430096D8
:10220000160007005E436146B0466F430E0CB844AB
:102210004644B74205D9802149028846009F474479
:10222000009761460904090C370C36048C463100CE
:10223000614401911100260C2404240C61438C4656
:102240002100694389466146090C884672434A4425
:1022500042447543914503D980214902884645444B
:10226000110C884661460904090C8C46120462442C
:10227000B91802915146090C8C4651460F043F0C87
:102280003900414345448846614641438A464146B8
:102290006046090C894658437B4353444B449A4556
:1022A00003D98021490289464844190C8946414690
:1022B0000904090C8846390061431B0443448846DD
:1022C00061464C4371438C46414677430E0C3F199F
:1022D000F6194844B44203D9802149028946CC44C6
:1022E0000299009F894631044F44894641469742EE
:1022F00092410C04240C4C44FF1852426419A1185A
:102300009F429B41884682465B4299469045924156
:10231000AC42A441C244D144524264421443994560
:102320009B41824592415B42524213434A46360CDE
:10233000A419E31863445B02D20D1A430199924633
:102340007A020A43501E8241FF0D17434A46520249
:102350001743B846DB0100D5EDE60D4B039A5B440D
:102360009146002B00DCACE03A00520700D110E7A8
:102370000F2258463A40042A00D0F9E609E7C04641
:10238000FF07000001FCFFFFFFFFFFFEFE0700004C
:10239000FF030000220032436FD0002C00D1C2E0C6
:1023A000200000F0A9FE020003000B3A1D20821A53
:1023B00030001900D04008398C400200224334001C
:1023C0008C405946CB1A86498B469B440A2D00DD2A
:1023D000A4E64946009B01945940CBB2140000206A
:1023E0000393022D00DD67E6FBE653460343984660
:1023F0003CD05346002B00D1A3E0504600F07CFEB9
:102400000B235B429C46020084441100504608396D
:1024100088401D23804660461B1A2000D8400300D8
:10242000404603439A4623008B4098466C4B002558
:102430009B1A9B46002302931AE60F2D00D0C9E099
:10244000802352461B031A4202D01C4200D192E064
:102450008024534624031C4324034246240B3EE6B7
:102460009B46032380460C25029301E600239A46EF
:102470009B46013304250293FAE501210D430A2D01
:1024800000DD4BE6494600984140C9B20391022D58
:1024900000DC96E000230024012001930CE649466D
:1024A0000223009A2B435140CAB203920A2B00DD4B
:1024B00034E6002D57D1039B994600240022494B56
:1024C0000EE658460121C91A382900DD2FE61F29DA
:1024D00056DD1F2254465242D31ADC40202907D031
:1024E000414B42469C465346604483401A439046C3
:1024F00042460721531E9A410B00224313400024F9
:10250000114209D00F231340042B5DD0111D9142BD
:102510009B410A005B425B07D2081A430023DFE5B8
:10252000039B9946FAE5019800F0E6FD02000300DE
:10253000153220331C2A00DC38E7019A0838824023
:102540003FE700F0D9FD15239C4684440200634612
:1025500020321C2B00DC58E7002398462300083863
:1025600083409A4662E71D00002300240220019365
:10257000A2E5029032E61C43009B019A9946AEE523
:102580001A4B5246C31840469A40C8400243404640
:1025900098400300581E834154461A43CC405307C9
:1025A00009D00F231340042B05D0131D93429241F1
:1025B0005242A4181A00230208D501230024002245
:1025C0008EE5894600248BE50023A5E763076402B6
:1025D000240BA1E7009BA2469946019B984637E74A
:1025E0000DFCFFFFFF0700003E0400001E0400007A
:1025F000F0B557464E464546DE46E0B583B00090FE
:1026000001910C034D00CE0F610A009C5F00640F26
:102610000C43009900920193C80019037B0D994661
:10262000019BCC4FDB0F9C464B0A00998046490F1B
:102630001943009B8B46DA0092466D0DB94500D1D7
:10264000BFE00123614659404B468C46EB1A8E424F
:1026500075D0002B00DCA3E24946002900D1CEE072
:10266000BD4200D100E20127382B19DC80275946F2
:102670003F0439438B461F2B00DDFAE12027F91A6E
:102680008C4659466746B9400F001100D9400F43A8
:1026900061468A40511E8A415946D9401743641AFF
:1026A000C71BB84280414042241A230200D440E1B3
:1026B0006402640A002C00D154E1200000F01CFDEB
:1026C0000300083B20213800CA1AD0409C40020079
:1026D0009F4022439D4200DDA6E1581B0130091AAC
:1026E0003C008F40C4407B1E9F4113008B4027431A
:1026F0001F43C2403B0014000025134300D1F7E103
:102700007B0700D177E30F2338003B40042B04D034
:10271000381DB842BF417F42E419230200D468E368
:102720008C4B01359D4200D1F4E08B4B6D051C4074
:102730006D0D6707C00864020743240BECE0002B13
:1027400000DC29E34946002900D0D6E05946114370
:1027500000D12EE1591E012B00D1E6E1BB4200D190
:1027600082E101270B00382914DC1F2B00DD3CE23D
:102770002027F91A8C4659466746B9400F001100C8
:10278000D9400F4361468A40511E8A415946D9407B
:10279000174364183F18874280414042241823029F
:1027A00000D4C6E06B4B01359D4200D1B2E001215F
:1027B000694B7A081C4039400A43E707174364080D
:1027C0009EE7664B11438A46EB18002928D06645E0
:1027D0002CD0002B5BD0002D00D12CE15B4666464F
:1027E0005F07D2081743DD083B002B4300D1E2E02E
:1027F000802424032C432403564D240B8CE059469B
:10280000114300D1D5E0591E012B00D1B9E1BB42E3
:1028100000D1B1E101270B00382900DD40E72AE7AC
:102820006146012779408C466645D2D1002B00D104
:10283000C5E0002D00D055E14B462500054300D1F1
:1028400012E2591E8C46012B00D149E2414DAB42A8
:1028500000D18FE20127382911DC63461F2B00DDF0
:102860005BE26146202327005B1A050098409F40E9
:10287000CD40431E9841CC402F430743A344BF188B
:102880009742924152425A4414004D4687E7344FD2
:102890006B1C3B4200D0B6E05946230011430F00A9
:1028A0000343002D00D026E1002B00D1C0E1002918
:1028B00000D1A1E0831A98465B464045AD41E31A3A
:1028C0006D425B1B80252D042B4200D14BE15B4602
:1028D000101A824292411C1B070001266346524295
:1028E000A41A27431E40002F00D142E12C4200D100
:1028F0006DE2194B01251C401BE7BD4200D13BE1B5
:102900000127382B00DD45E7802759463F0439432E
:102910008B462AE7002400272D052543F60735437B
:102920003800290003B0F0BCBB46B246A946A04619
:10293000F0BD7B0704D00F233B40042B00D0E7E61B
:102940002B00F808034A67070743E508934200D1C4
:102950004AE7A5E0FF070000FFFF7FFF01F8FFFF48
:10296000FE070000380000F0C7FB030018331F2BE0
:1029700000DCA7E63A00083882409D4200DD8AE08C
:102980005B1B581C1F2800DCD8E117001F3BDF40F1
:10299000202805D040231B1A9A40531E9A41174302
:1029A0000025002F00D1E5E07B0700D0ABE62C002E
:1029B000C6E7C008C6E700270024D14DACE7D14FD9
:1029C0006B1C3B4271D123000343002D00D04EE12C
:1029D0005746002B00D1B5E1002F0DD0831883425C
:1029E00080415C4440422418220200D5C8E11F0007
:1029F0009846274300D1BCE043466707DB081F43E6
:102A0000E50800234CE0831A98465B464045BF41E9
:102A1000E31A7F42DB1B1F027CD447461F4300D1D1
:102A2000A6E01C00474645E6B74CED1A14407B076C
:102A300000D080E784E74B462500054366D05F1E43
:102A4000012B00D1FCE0AE4DAB4200D15EE1664609
:102A5000382F00DCB4E00120171ABA4292415B46DD
:102A600052424D469C1A20E66707C0080743E50816
:102A7000BAE61F005946203FF9400F00202B05D031
:102A80004021CB1A594699400A43924653465A1E52
:102A900093411F4304E6EB1A9B4D15406F07ED0869
:102AA0002C035D05240B6D0D36E7954DAB4200D12F
:102AB000D6E08218210082428041594440420818E1
:102AC000C707520817434408520700D485E10F2274
:102AD0001D003A40042A00D01AE6FF086407274385
:102AE0000509DDE75B46D2085F071743DD087BE693
:102AF0000027002410E7002B00D0D6E0002900D0EA
:102B00002FE1802400267E4D240305E766465C46BF
:102B1000D00817E75B46171ABA4292411C1B0126E0
:102B200063465242A41A1E40C4E583188342804182
:102B30005C44404225182A0200D4DAE0724A5B085D
:102B40001540EA071A4369085B0700D44AE10F23DE
:102B50001340042B00D1FCE0171D9742A4416442AE
:102B600002256418ECE647461C001F4300D043E7EB
:102B7000002600250024CFE6C00867070743E508C4
:102B800032E6871A5B46B8428041E41A4042241A72
:102B9000230228D46307FF081F43E50801237FE7CA
:102BA000002B00D173E64B465F1B3B00002D00D18C
:102BB00042E7382F00DDECE080230E001B041C43AD
:102BC0001F2F25DC20252300ED1B0100A840AB4072
:102BD000F940451EA8410B43FC4018435B461B1BB4
:102BE0009B4639E76646012562E51F005946203FAE
:102BF000F9408C46202B05D040275946FB1A9940B6
:102C00000A43924657467B1E9F4163461F43C1E5D8
:102C10003B002500203BDD40202F04D04023DB1B60
:102C20009C40204380464046431E9841284313E77A
:102C300000299DD0012663465C4690461E40DBE697
:102C4000171A5B46BA4292411C1B5242A41A230235
:102C5000C8D46307FF081F4366460123E5081FE742
:102C60001D000024002757E65C46D0086AE6002BCA
:102C700000D137E75346C00867070743E508002B34
:102C800000D1B1E580231B031D4208D05946C80876
:102C9000184204D1D20849070A43170005007B0FE8
:102CA000FF00FF085B071F439EE5C008630718434A
:102CB000E508002953D080231B031D420AD0594642
:102CC000CC081C4206D1012663462500D0084907DE
:102CD00008431E40470FC000C0087F07074383E535
:102CE0008318934292415C445242A5182A0200D5AF
:102CF00024E76F07DB081F43ED080123D0E6C04639
:102D0000FF070000FE070000FFFF7FFF5B46D208C1
:102D10005F0766461743DD0866E52500203BDD407A
:102D20006346202B05D0402361465B1A9C4020431C
:102D3000804647467B1E9F412F43A0E52021002768
:102D4000091AD2E4002F00D113E75C4617000025D2
:102D5000F6E5D708490702230F432D09A0E607002F
:102D600042E55B4601265F07DD086346D20817434C
:102D70001E4039E55B46D2085F071743DD0833E59F
:102D80001E4ADB0822405707520201251F43140B3D
:102D9000C2E50E0001205FE6002B0DD04B465B1B09
:102DA0009C46002D00D148E50127382B00DD66E563
:102DB00080231B041C4350E56B1C114D2B4200D09B
:102DC00073E65946230011438A46034300E667072A
:102DD000C00800230743E50862E66407FF082743AD
:102DE00005095DE6D208490711430F0002232D09AA
:102DF00056E60700A4E538008FE4C046FFFF7FFFDA
:102E0000FE070000F0B5C6461E03360BB0460D4E59
:102E10000C034D005F0000B5240B6D0D7F0DB54216
:102E20000BD0084900208F4204D14646164330009B
:102E3000431E984180BCB846F0BD04430120002CDD
:102E4000F8D1EEE7FF0700000B00020070B5164D49
:102E50000C0382B04900002000920193240B490D1D
:102E6000DE0FA94204DD1148814203DD104BF0184A
:102E700002B070BD8020400320430E4C641A1F2C0A
:102E800008DD0D4B5B1AD84003005842002EEFD1ED
:102E90001800EDE7094B009A9C46030061448B4003
:102EA000E2401343F1E7C046FE0300001D040000AA
:102EB000FFFFFF7F3304000013040000EDFBFFFF62
:102EC00070B5002816D0C317C5185D40C40F280080
:102ED00000F012F9104B1B1A5B055B0D0A2814DC7D
:102EE00002002E00153296400B22121AD5402D03F7
:102EF0002D0B03E000240023002500261B052B4397
:102F0000E40723433000190070BD0B3885402D03C2
:102F100000262D0BF2E7C0461E04000010B5041E6B
:102F200010D000F0E9F80E4B1B1A5B055B0D0A2868
:102F30000FDC0B222100121AD14015300A03844005
:102F4000120B01E0002300221B051343200019008F
:102F500010BD22000B38824012030024120BF3E74D
:102F60001E04000070B542024300C40FFE201B0E79
:102F7000591C550A08420CD0E02189008C466D0787
:102F8000120B63441B051343E40723432800190075
:102F900070BD002B14D1002D1BD0280000F0ACF820
:102FA0000A281CDC0B232A001B1ADA400300153305
:102FB0009D400E4B12031B1A5B05120B5B0DE1E7E4
:102FC000002D09D0130B802212031A436D07084B02
:102FD000D8E700230022D5E70022054BD2E7030003
:102FE0002A000B3B9A400025E3E7C0468903000016
:102FF000FF070000F0B54B000F035B0D3A4C450F87
:1030000083B07F0A5E1C2F4300900191CA0FC50058
:1030100026420BD035495C18FE2C13DDFF2000231F
:10302000C0051843D207104303B0F0BD3D43002B49
:1030300001D10020F4E7002DF0D08023DB03FF2036
:103040003B43EDE7002C0CDD009BFF009B01581E6D
:103050008341690F3B430B43590727D1DB08E0B29B
:10306000DEE72100173131DB80211E2009043943BE
:10307000001B1F282DDD02267642341B0E00E64081
:103080003400202804D01A488446634499400D43F4
:103090002B00591E8B412343590703D00F211940A0
:1030A00004290BD19B0100205B0AB9E70F211940CD
:1030B000042904D19B015B0AE0B2B1E70024043388
:1030C0005901F7D501340023E0B2A9E7002000231D
:1030D000A6E7084C1C192B00A540C340A140681E60
:1030E000854129430B43D7E7FE07000080FCFFFF23
:1030F000A2FCFFFF82FCFFFF1C2101231B0498425E
:1031000001D3000C10391B0A984201D3000A083978
:103110001B09984201D30009043902A2105C40182F
:103120007047C046040302020101010100000000D3
:103130000000000010B5002903D1FFF7DDFF2030AB
:1031400002E00800FFF7D8FF10BDC04680B582B08E
:1031500000AF7860391D05480A2301220CF02AF9D6
:103160007B681800BD4602B080BDC046DC0600206A
:1031700080B500AF05F0CEFC08F00CFE62B6C0468C
:1031800005F0A8FC00F020F800F012FB00F086FC2F
:1031900000F0BEFC00F02EFF00F04CFF00F03EFE01
:1031A00001F006F801F0BAF801F0C0F901F00CFAEC
:1031B00001F058FA00F0EEFD05F0C0F800F05CF9FF
:1031C00005F0DEF8C046FDE790B593B000AF1024DF
:1031D0003B19180038231A0000211CF0CBFF3B00DC
:1031E000180010231A0000211CF0C4FF80239B004C
:1031F000180008F083FD08F073FD264BDA6D254BAF
:1032000018218A43DA653B190D221A603B19802286
:1032100052025A6021007B1801229A607B18012219
:103220009A617B180222DA617B1803221A627B18EA
:1032300010225A627B1810229A627B188022920216
:10324000DA627B18802292041A637B188022D205EE
:103250005A637B18180008F019FE031E01D000F015
:103260002DF83B0007221A603B0002225A603B0007
:1032700000229A603B000022DA603B000221180025
:1032800009F01EF9031E01D000F018F8C046BD4633
:1032900013B090BD0010024080B582B000AF7860DE
:1032A0007B681B68044A934201D105F05FFCC0466D
:1032B000BD4602B080BDC0460048014080B500AFA9
:1032C00072B6C046C046FDE780B500AFC046FDE718
:1032D00080B500AF024B18001CF0D0FDC046FDE7E2
:1032E000D02B030880B500AF042008F06DFC082047
:1032F00008F06AFCC046BD4680BD80B500AF202006
:1033000008F062FC402008F05FFC80239B0118005D
:1033100008F05AFC8023DB01180008F055FCC04679
:10332000BD4680BD80B500AF034B180007F088FE96
:10333000C046BD4680BDC0469808002080B500AF9D
:10334000054B180007F07CFE044B180007F078FED0
:10335000C046BD4680BDC046F8080020B809002020
:1033600080B500AF0D4B180007F06AFE0C4B18003B
:1033700007F066FE0B4B180007F062FE0A4B1800C0
:1033800007F05EFE094B180007F05AFE084B1800C4
:1033900007F056FEC046BD4680BDC0465809002015
:1033A000180A0020780A002048050020A8050020FF
:1033B0006004002080B500AF034B180006F020FA2F
:1033C000C046BD4680BDC046FC03002080B500AFAE
:1033D000034B18000BF096F8C046BD4680BDC046B2
:1033E000AC03002080B500AF034B18000AF06EFB61
:1033F000C046BD4680BDC046E404002080B500AF95
:10340000034B18000CF0B4FBC046BD4680BDC0465F
:10341000DC06002080B500AF034B18000CF0A8FBC1
:10342000C046BD4680BDC0467007002080B500AFD5
:10343000034B18000CF09CFBC046BD4680BDC04647
:103440000408002080B500AF034B180008F038FCDA
:10345000C046BD4680BDC0460806002080B582B08B
:1034600000AF78603960C046BD4602B080BD80B50F
:1034700000AFC046BD4680BD80B500AF054A064BD3
:103480000021180004F0B9FF0200044B1A60C04686
:10349000BD4680BDE05A0308A1340108A8030020FE
:1034A00080B582B000AF78600DF07AFF002003F0A5
:1034B0001BF8C046BD4602B080BD000080B582B09A
:1034C00000AF154B1A6C144B01210A431A64124BBE
:1034D0001B6C012213407B607B680F4BDA6B0E4B39
:1034E000802149050A43DA630B4BDA6B80235B05C5
:1034F00013403B603B6802235B420022032118001B
:1035000007F09AF8C023DB00180005F06FFBC046F7
:10351000BD4602B080BDC04600100240B0B58CB0C0
:1035200000AF78602B23FB1800221A70384B1A6CFE
:10353000374B8021C9020A431A64354B1A6C802329
:10354000DB021340BB60BB680C23FA1810243B1944
:103550001100180009F05EF93B19DB687B627B6A99
:10356000002B04D109F040F90300FB6204E009F0EC
:103570003BF903005B00FB62FB6A26491800FCF77D
:10358000E9FE0300013B3B62234B244A1A60224BB5
:10359000234ADA60204B3A6A5A601F4B00221A61B4
:1035A0001D4B00229A601C4B00229A612B257C192E
:1035B000194B18000AF01CFD030023707B191B78BF
:1035C000002B1ED17C19144B18000AF071FD03006A
:1035D00023707B191B78002B13D1162007F041F8BC
:1035E0007B68032B09D87B6800221900162007F09E
:1035F00023F80C4B7A681A6003E02B23FB18012296
:103600001A702B23FB181B781800BD460CB0B0BDF8
:103610000010024040420F00AC030020004801406F
:10362000E70300000800002080B500AFC046BD469B
:1036300080BD80B500AF01231800BD4680BD80B5B8
:1036400082B000AF786039601CF0A4FE030016223F
:103650001A6001235B421800BD4602B080BD80B5F0
:1036600082B000AF786001235A427B6811001800D5
:10367000FFF7E5FFC046FDE780B586B000AFF86014
:10368000B9607A6000237B610AE000E000BF0100BE
:10369000BB685A1CBA60CAB21A707B6901337B617D
:1036A0007A697B689A42F0DB7B681800BD4606B0F9
:1036B00080BD80B586B000AFF860B9607A60002345
:1036C0007B6109E0BB685A1CBA601B781800FFF7E1
:1036D0003DFD7B6901337B617A697B689A42F1DB4E
:1036E0007B681800BD4606B080BD80B582B000AFD3
:1036F000786001235B421800BD4602B080BD80B5F2
:1037000082B000AF786039603B68802292015A60D5
:1037100000231800BD4602B080BD80B582B000AF66
:10372000786001231800BD4602B080BD80B584B02A
:1037300000AFF860B9607A6000231800BD4604B09D
:1037400080BD000080B586B000AF7860144A154B8C
:10375000D31A7B617B693B61134B1B68002B02D141
:10376000114B124A1A60104B1A687B68D3183A69D9
:103770009A4207D21CF00EFE03000C221A600123AD
:103780005B4209E0084B1B68FB60074B1A687B68CB
:10379000D218054B1A60FB681800BD4606B080BD04
:1037A0000040022000080000F803002090AC012037
:1037B00090B58BB000AF14243B19180014231A00E5
:1037C00000211CF0D7FCAB4B5A6BAA4B04210A43D7
:1037D0005A63A84B5B6B042213403B613B69A54BCA
:1037E0005A6BA44B20210A435A63A24B5B6B2022E5
:1037F0001340FB60FB689F4B5A6B9E4B01210A43B1
:103800005A639C4B5B6B01221340BB60BB68994BB6
:103810005A6B984B02210A435A63964B5B6B022208
:1038200013407B607B68934B5A6B924B08210A4391
:103830005A63904B5B6B082213403B603B688323C9
:103840009B018D480022190008F085F98B49A023BF
:10385000DB050022180008F07EF98949894B002217
:10386000180008F078F98849884B0022180008F001
:1038700072F9864B01221021180008F06CF984239C
:103880005B0080480122190008F065F93B1980228D
:1038900092011A603B1901225A603B1900229A607A
:1038A0003B190022DA603B19734A1900100007F037
:1038B000F1FE21007B18882252001A600C003B198F
:1038C00001225A603B1900229A603B190322DA60F8
:1038D0003A19A023DB051100180007F0DBFE3B19A5
:1038E0006B4A1A603B1901225A603B1902229A6006
:1038F0003B190322DA603B19624A1900100007F0F5
:10390000C9FE21007B18C022D2011A607B18C42294
:1039100092035A607B1801229A600C007B18594A66
:103920001900100007F0B6FE21007B188022120259
:103930001A600C003B1901225A603B1900229A6060
:103940003B190022DA603B194E4A1900100007F0BB
:10395000A1FE3B19C0221A603B1901225A603B1993
:1039600000229A603B190322DA603B19424A19008F
:10397000100007F08FFE3B19464A1A603B190122DE
:103980005A603B1900229A603B190322DA603B1906
:103990003E4A1900100007F07DFE21007B188022AE
:1039A00012021A600C003B1901225A603B190222D4
:1039B0009A603B190322DA603A19A023DB05110053
:1039C000180007F067FE21007B186C221A607B1834
:1039D000842292035A607B1801229A600C007B18A3
:1039E0002A4A1900100007F055FE21007B18842296
:1039F00052001A607B1801225A607B1801229A60DB
:103A00007B180322DA607B181E4A1900100007F0A9
:103A100041FE214B1A68204B802149020A431A605B
:103A20001D4B1A681C4B802189020A431A601A4BED
:103A30001A68194B8021C9020A431A60164B1A688A
:103A4000154B802109030A431A6000220321062036
:103A500006F0F2FD062006F004FE002203210720F6
:103A600006F0EAFD072006F0FCFDC046BD460BB09F
:103A700090BDC046001002400008005010810000B8
:103A8000C18200000004005003030000000C00503D
:103A9000C1020000130300000000014080B582B0A5
:103AA00000AF1A4B9A6B194B01210A439A63174BCB
:103AB0009B6B012213407B607B68144B9A6B134B0A
:103AC00002210A439A63114B9B6B022213403B6015
:103AD0003B6800220321092006F0AEFD092006F014
:103AE000C0FD002203210A2006F0A6FD0A2006F0F0
:103AF000B8FD002203210B2006F09EFD0B2006F0EE
:103B0000B0FDC046BD4602B080BDC04600100240B8
:103B100080B584B000AF3B1D18000C231A000021B3
:103B20001CF028FB344B354A1A60334B8022D205F7
:103B30005A60314B00229A602F4B0022DA602E4BE4
:103B4000802292031A612C4B04225A612A4B0022D4
:103B50001A76294B00225A76274B01229A76264B59
:103B60000222DA61244B00225A62234B00229A621D
:103B7000214B2C22012199541F4B00221A631E4B0A
:103B800005225A631C4B05229A631B4B3C220021E1
:103B90009954194B0022DA64174B180005F0C2F94A
:103BA000031E01D0FFF78AFB3B1D154A1A603B1D1F
:103BB00000225A603B1D00229A603A1D0E4B1100F4
:103BC000180005F045FF031E01D0FFF777FB3B1DF2
:103BD0000C4A1A603B1D04225A603A1D064B110024
:103BE000180005F035FF031E01D0FFF767FBC04644
:103BF000BD4604B080BDC046FC0300200024014047
:103C0000020000040004002890B58BB000AF78607B
:103C100014243B19180014231A0000211CF0AAFADE
:103C20007B681B683F4A934277D13F4B1A6C3E4BEF
:103C3000802149030A431A643B4B1A6C80235B03BF
:103C400013403B613B69384B5A6B374B01210A43A8
:103C50005A63354B5B6B01221340FB60FB68324BB0
:103C60005A6B314B02210A435A632F4B5B6B022282
:103C70001340BB60BB683B1902221A603B19032248
:103C80005A603B1900229A603A19A023DB05110003
:103C9000180007F0FFFC3B1904221A603B190322AD
:103CA0005A603B1900229A603B19204A1900100003
:103CB00007F0F0FC1E4B1F4A1A601D4B05225A608C
:103CC0001B4B00229A601A4B0022DA60184B8022AC
:103CD0001A61174B802252005A61154B8022D20084
:103CE0009A61134B0022DA61114B00221A62104BC9
:103CF000180006F013FF031E01D0FFF7DFFA7B6800
:103D00000B4A1A650A4B7A689A62002203210C203A
:103D100006F092FC0C2006F0A4FCC046BD460BB099
:103D200090BDC04600240140001002400004005035
:103D3000600400201C04024080B582B000AF7860AF
:103D40007B681B680F4A934218D10F4B1A6C0E4BBD
:103D50000E490A401A64A023DB050221180007F06F
:103D600005FE0B4B0421180007F000FE7B681B6D5D
:103D7000180006F07FFF0C2006F083FCC046BD460D
:103D800002B080BD0024014000100240FFFFEFFFA1
:103D90000004005080B500AF0E4B0F4A1A600D4B67
:103DA00000221A710B4B00225A710A4B00225A61F1
:103DB000084B00229A61074B01221A62054B18003A
:103DC00006F070FC031E01D0FFF778FAC046BD462E
:103DD00080BDC046C00400200030024080B584B0E1
:103DE00000AF78607B681B680A4A93420DD10A4B8A
:103DF0009A6B094B802149010A439A63064B9A6BDF
:103E000080235B011340FB60FB68C046BD4604B0E5
:103E100080BDC046003002400010024080B500AFB7
:103E20001B4B1C4A1A601A4B822252005A60184BD4
:103E300000229A60164BE022D200DA60144B022274
:103E40001A61134B01225A61114B802292009A6130
:103E50000F4B0022DA610E4B80221A620C4B0022BB
:103E60005A620B4B00229A62094B0722DA62084B16
:103E700000221A63064B00225A63054B180009F012
:103E80002BFA031E01D0FFF719FAC046BD4680BDCC
:103E9000E40400200030014090B58BB000AF7860A2
:103EA00014243B19180014231A0000211CF062F995
:103EB0007B681B68494A934200D08AE0484B1A6CE1
:103EC000474B802149010A431A64454B1A6C8023F1
:103ED0005B0113403B613B69414B5A6B404B0121F5
:103EE0000A435A633E4B5B6B01221340FB60FB6845
:103EF00021007B18E0221A607B1802225A607B188E
:103F000000229A607B180322DA607B1800221A6173
:103F10007A18A023DB051100180007F0BBFB314B1A
:103F2000314A1A602F4B10225A602E4B00229A60A1
:103F30002C4B0022DA602B4B80221A61294B002285
:103F40005A61284B00229A61264B0022DA61254BE8
:103F500000221A62234B180006F0E0FD031E01D078
:103F6000FFF7ACF97B681F4A9A651E4B7A689A6224
:103F70001E4B1F4A1A601D4B11225A601B4B102208
:103F80009A601A4B0022DA60184B80221A61174B94
:103F900000225A61154B00229A61144B0022DA610B
:103FA000124B00221A62114B180006F0B7FD031ED7
:103FB00001D0FFF783F97B680C4A5A650B4B7A688E
:103FC0009A6200220321192006F036FB192006F020
:103FD00048FBC046BD460BB090BDC0460030014016
:103FE000001002404805002080000240A805002083
:103FF0000804024080B500AF0B4B0C4A1A600A4B14
:1040000003225A60084B0A4ADA60074B084A9A6052
:10401000054B180007F002FE031E01D0FFF74EF912
:10402000C046BD4680BDC0460806002000300040A6
:10403000B80B000080B586B000AF3B1D18001423FC
:104040001A0000211CF096F83B0000221A60364B43
:10405000364A1A60344B00229A60334B7F22DA6072
:10406000314BFF221A61304B00225A612E4B002245
:104070009A612D4B0022DA612B4B8022D2051A6205
:10408000294B00225A62284B180008F075FD031EC8
:1040900001D0FFF713F907F023FE234B002118008E
:1040A00009F0FEF80300224A934238D0204A1E4B02
:1040B0000021180009F0D7F83B1D00221A703B1DA3
:1040C00000225A703B1D00229A703B1D00225A604C
:1040D0003B1D0022DA603B1D00221A61391D124B84
:1040E0000122180008F0EAFD031E01D0FFF7E6F8F0
:1040F0003B0001221A703B0003225A703B0002224F
:104100009A703B002622DA703900074B0122180012
:1041100008F0D8FE031E03D0FFF7D0F800E0C04639
:10412000BD4606B080BDC0461806002000280040ED
:104130001290785690B58FB000AF78600C243B1980
:1041400018002C231A0000211CF014F87B681B684F
:10415000154A934224D13B19802292021A603B19DE
:10416000802252005A623B19180008F07DFB031EA2
:1041700001D0FFF7A3F80D4BDA6D0C4B802109023B
:104180000A43DA65094BDA6B084B8021C9000A4300
:10419000DA63064BDA6B8023DB001340BB60BB683D
:1041A000C046BD460FB090BD002800400010024040
:1041B00080B598B000AF5423FB1818000C231A00E8
:1041C00000211BF0D7FF3823FB1818001C231A000E
:1041D00000211BF0CFFF3B1D180034231A000021E3
:1041E0001BF0C8FF4B4B4C4A1A604A4B0F225A60D7
:1041F000484B00229A60474BC722DA60454B0022A9
:104200001A61444B00225A61424B80229A61414B11
:10421000180009F0A9FF031E01D0FFF74FF8542141
:104220007B1800221A607B1800225A607B1800223B
:104230009A607A18374B110018000AF001FF031E2C
:1042400001D0FFF73BF838217B1860221A607B18F9
:1042500000225A607B1800229A607B180022DA60E4
:104260007B1804221A617B1800225A617B180022F5
:104270009A617918274B002218000AF04BFA031EA6
:1042800001D0FFF71BF83823F918224B042218003D
:104290000AF040FA031E01D0FFF710F83B1D002280
:1042A0001A603B1D00225A603B1D00229A603B1D94
:1042B0000022DA603B1D00221A613B1D8022920120
:1042C0005A613B1D00229A613B1D0022DA613B1DB1
:1042D00000221A623B1D802292045A623B1D00227A
:1042E0009A623B1D0022DA623B1D00221A633A1DCE
:1042F000084B110018000AF013FF031E01D0FEF74F
:10430000DDFF044B180000F0A7F8C046BD4618B00A
:1043100080BDC04644060020002C014080B58AB014
:1043200000AF1C23FB1818000C231A0000211BF0FF
:1043300021FF3B0018001C231A0000211BF01AFF6C
:10434000294B2A4A1A60284B0F225A60264B00221A
:104350009A60254BC722DA60234B00221A61224B58
:1043600000229A61204B180009F0FEFE031E01D0C6
:10437000FEF7A4FF1C217B1800221A607B18002284
:104380009A607A18184B110018000AF059FE031EA3
:1043900001D0FEF793FF3B0060221A603B00002231
:1043A0005A603B0000229A603B0004221A613900E7
:1043B0000D4B002218000AF0ADF9031E01D0FEF7E4
:1043C0007DFF3900084B042218000AF0A3F9031EF0
:1043D00001D0FEF773FF044B180000F03DF8C04613
:1043E000BD460AB080BDC0469006002000040040D3
:1043F00080B584B000AF78607B681B68134A934235
:104400000ED1134B1A6C124B802109010A431A6416
:104410000F4B1A6C80231B011340FB60FB6810E0FC
:104420007B681B680B4A93420BD1094BDA6B084B34
:1044300002210A43DA63064BDB6B02221340BB60A6
:10444000BB68C046BD4604B080BDC046002C0140DC
:10445000001002400004004090B58BB000AF7860BF
:1044600014243B19180014231A0000211BF082FEAB
:104470007B681B68284A934223D1284B5A6B274BF1
:1044800004210A435A63254B5B6B042213403B61B2
:104490003B693B19C02292001A6021007B1802225E
:1044A0005A607B1800229A607B180322DA607B181E
:1044B00002221A617B181A4A1900100007F0EAF864
:1044C00026E07B681B68174A934221D1134B5A6B35
:1044D000124B02210A435A63104B5B6B02221340BA
:1044E000FB60FB6814217B1830221A607B180222C3
:1044F0005A607B1800229A607B180322DA607B18CE
:1045000001221A617B18084A1900100007F0C2F84E
:10451000C046BD460BB090BD002C014000100240CB
:1045200000080050000400400004005080B500AFB7
:10453000234B244A1A60224BE12252025A60204B3C
:1045400000229A601E4B0022DA601D4B00221A6185
:104550001B4B0C225A611A4B00229A61184B002205
:10456000DA61174B00221A62154B00225A62144B73
:1045700000229A62124B18000AF086FE031E01D038
:10458000FEF79CFE0E4B002118000CF08BFD031E65
:1045900001D0FEF793FE0A4B002118000CF0C2FD7B
:1045A000031E01D0FEF78AFE054B18000CF040FDFB
:1045B000031E01D0FEF782FEC046BD4680BDC04648
:1045C000DC0600200038014080B500AF234B244AB0
:1045D0001A60224BE12212035A60204B00229A609B
:1045E0001E4B0022DA601D4B00221A611B4B0C226D
:1045F0005A611A4B00229A61184B0022DA61174B5C
:1046000000221A62154B00225A62144B00229A6251
:10461000124B18000AF038FE031E01D0FEF74EFEC2
:104620000E4B002118000CF03DFD031E01D0FEF7DB
:1046300045FE0A4B002118000CF074FD031E01D04A
:10464000FEF73CFE054B18000CF0F2FC031E01D0F7
:10465000FEF734FEC046BD4680BDC0467007002050
:104660000044004080B500AF244B254A1A60234B1C
:10467000E12252025A60214B00229A601F4B002215
:10468000DA601E4B00221A611C4B0C225A611B4B34
:1046900000229A61194B0022DA61184B00221A623B
:1046A000164B00225A62154B00229A6213480023CF
:1046B000002200210CF032FC031E01D0FEF7FEFDAB
:1046C0000E4B002118000CF0EDFC031E01D0FEF78C
:1046D000F5FD0A4B002118000CF024FD031E01D04B
:1046E000FEF7ECFD054B18000CF0A2FC031E01D0F8
:1046F000FEF7E4FDC046BD4680BDC046040800206C
:104700000048004090B59BB000AF78605423FB1880
:10471000180014231A0000211BF02CFD28243B193B
:1047200018002C231A0000211BF024FD7B681B6855
:10473000A14A934200D09BE03B1901221A603B1929
:1047400000225A603B19180008F08EF8031E01D0B1
:10475000FEF7B4FD994B1A6C984B8021C9010A43AE
:104760001A64964B1A6C8023DB0113407B627B6AD0
:10477000924B5A6B914B01210A435A638F4B5B6BEF
:10478000012213403B623B6A54217B18C022D200B5
:104790001A607B1802225A607B1800229A607B18EC
:1047A0000322DA607B1801221A617A18A023DB0544
:1047B0001100180006F06EFF814B824A1A60804B90
:1047C00032225A607E4B00229A607D4B0022DA60D2
:1047D0007B4B80221A617A4B00225A61784B00226F
:1047E0009A61774B2022DA61754B00221A62744B72
:1047F000180006F093F9031E01D0FEF75FFD7B68F9
:1048000080216F4A5A506E4B7A689A626E4B6F4A9B
:104810001A606D4B33225A606B4B10229A606A4BC0
:104820000022DA60684B80221A61674B00225A61CD
:10483000654B00229A61644B0022DA61624B0022D0
:104840001A62614B180006F069F9031E01D0FEF7E9
:1048500035FD7B685C4ADA675B4B7A689A620022B6
:1048600003211B2005F0E8FE1B2005F0FAFE7BE18A
:104870007B681B68564A934200D0B3E028217B181E
:1048800002221A607B1800229A607B18180007F039
:10489000EBFF031E01D0FEF711FD484BDA6B474BCF
:1048A000802189020A43DA63444BDA6B80239B023E
:1048B0001340FB61FB69414B5A6B404B01210A439A
:1048C0005A633E4B5B6B01221340BB61BB695421B1
:1048D0007B180C221A607B1802225A607B18002277
:1048E0009A607B180322DA607B1801221A617A1819
:1048F000A023DB051100180006F0CCFE354B364A2C
:104900001A60344B34225A60324B00229A60314B89
:104910000022DA602F4B80221A612E4B00225A614E
:104920002C4B00229A612B4B2022DA61294B8022EA
:1049300092011A62274B180006F0F0F8031E01D00E
:10494000FEF7BCFC7B688021224A5A50214B7A68D2
:104950009A62224B224A1A60204B35225A601F4B22
:1049600010229A601D4B0022DA601C4B80221A61D3
:104970001A4B00225A61194B00229A61174B0022F0
:10498000DA61164B802292011A62144B180006F06D
:10499000C5F8031E01D0FEF791FC7B680F4ADA6769
:1049A0000E4B7A689A62002203211C2005F044FE17
:1049B0001C2005F056FED7E00038014000100240F0
:1049C0009808002008000240F80800201C0002405F
:1049D000004400405809002044000240B80900206B
:1049E000300002407B681B68614A934200D0BBE004
:1049F00028217B1804221A607B180022DA607B18B9
:104A0000180007F031FF031E01D0FEF757FC594B89
:104A1000DA6B584B8021C9020A43DA63554BDA6BD3
:104A20008023DB0213407B617B69524B5A6B514BF5
:104A300004210A435A634F4B5B6B042213403B61D2
:104A40003B694C4B5A6B4B4B02210A435A63494B0F
:104A50005B6B02221340FB60FB6854243B1930223D
:104A60001A603B1902225A603B1900229A603B19D6
:104A70000322DA603B1900221A613B193E4A1900F1
:104A8000100006F007FE21007B1802221A607B1836
:104A900002225A607B1800229A607B180322DA6097
:104AA0007B1804221A617B18344A1900100006F0A2
:104AB000F1FD334B334A1A60314B36225A60304B8A
:104AC00000229A602E4B0022DA602D4B80221A6160
:104AD0002B4B00225A612A4B00229A61284B00225C
:104AE000DA61274B00221A62254B180006F016F8EF
:104AF000031E01D0FEF7E2FB7B688021204A5A505A
:104B00001F4B7A689A62204B204A1A601E4B37224C
:104B10005A601D4B10229A601B4B0022DA601A4B20
:104B200080221A61184B00225A61174B00229A61A9
:104B3000154B0022DA61144B00221A62124B180046
:104B400005F0ECFF031E01D0FEF7B8FB7B680E4AB0
:104B5000DA670D4B7A689A62002203211D2005F066
:104B60006BFD1D2005F07DFDC046BD461BB090BD10
:104B700000480040001002400008005000040050AF
:104B8000180A002058000240780A00206C000240F9
:104B900080B582B000AF78607B681B68334A93426F
:104BA0001CD1334B1A6C324B32490A401A64C02371
:104BB000DA00A023DB051100180006F0D7FE7B68A1
:104BC00080229B58180006F055F87B68DB6F1800B0
:104BD00006F050F81B2005F054FD42E07B681B688E
:104BE000254A93421AD1224BDA6B214B23490A40C2
:104BF000DA63A023DB050C21180006F0B7FE7B6802
:104C000080229B58180006F035F87B68DB6F18008F
:104C100006F030F81C2005F034FD22E07B681B68AC
:104C2000174A93421DD1124BDA6B114B15490A40BA
:104C3000DA63154B3021180006F098FE134B022161
:104C4000180006F093FE7B6880229B58180006F03F
:104C500011F87B68DB6F180006F00CF81D2005F0DA
:104C600010FDC046BD4602B080BDC04600380140C0
:104C700000100240FFBFFFFF00440040FFFFFDFFA8
:104C800000480040FFFFFBFF0008005000040050F8
:104C900080B582B000AF78600A00BB1C1A807B68C8
:104CA0001B68144A934207D1BB1C1A887B68110009
:104CB000180017F0D9FD18E07B681B680E4A934274
:104CC00007D1BB1C1A887B681100180011F020F96D
:104CD0000BE07B681B68094A934206D1BB1C1A880B
:104CE0007B681100180012F00FFFC046BD4602B0ED
:104CF00080BDC046003801400044004000480040EC
:104D000080B582B000AF78607B681B680F4A934221
:104D100004D17B68180017F0BBFD12E07B681B68AC
:104D20000B4A934204D17B68180011F0FDF808E0AB
:104D30007B681B68074A934203D17B68180012F016
:104D40001FFFC046BD4602B080BDC04600380140CE
:104D5000004400400048004080B582B000AF786059
:104D60007B681B680F4A934204D17B68180017F0D8
:104D7000A1FD12E07B681B680B4A934204D17B685B
:104D8000180011F0FBF808E07B681B68074A9342A3
:104D900003D17B68180012F025FFC046BD4602B063
:104DA00080BDC0460038014000440040004800403B
:104DB00080B582B000AF202003F07AF803007B605A
:104DC0007B68002B0AD07B6800221A607B68043362
:104DD000180000F0CBF97B6800221A777B68180076
:104DE000BD4602B080BD80B58CB000AFF860B96040
:104DF0007A603B60FB687B620023BB6200233B62FE
:104E0000FB68002B02D172B6C046FDE7BA6880236A
:104E10005B049A4202D372B6C046FDE7BB68002B22
:104E200002D172B6C046FDE702F0A8F8031E02D117
:104E3000BB6B002B01D1012300E00023002B02D12A
:104E400072B6C046FDE701F039FC7B6A1B68FB6166
:104E50003A68B968FB69180000F052F90300BB61B9
:104E6000BB69002B0ED0FB69FB620023BB637B6830
:104E7000002B2AD07B6A1B68BA68D2431A407B6A2F
:104E80001A6022E0BB6B002B04D1FB69FB6201239B
:104E90003B621AE07B68002B04D0BB6A802252047C
:104EA0001343BB623B68002B04D0BB6A8022D20450
:104EB0001343BB627B6A181DBA68BB6A1343BA6BA3
:104EC000190001F003FE0023FB6201F003FC030064
:104ED0007B61BB6B002B2CD07B69002B01D102F0D6
:104EE0003FFF02F09FF90300FB62FA6A80239B04F4
:104EF00013401AD102F044FF7B6A1B68FB623A68D8
:104F0000B968FB6A180000F0FBF8031E09D07B6843
:104F1000002B06D07B6A1B68BA68D2431A407B6AB2
:104F20001A6001233B6202F03DFFFB6A1B021B0A71
:104F3000FB62FB6A1800BD460CB080BD80B584B032
:104F400000AF786039607B68FB607B68002B02D122
:104F500072B6C046FDE73A6880235B049A4202D3EA
:104F600072B6C046FDE702F00BFFFB681B68BB6032
:104F7000FB681B683A68D2431A40FB681A6002F06B
:104F800011FFBB681800BD4604B080BD80B58CB071
:104F900000AF786039600023BB627B683B6200230E
:104FA0007B627B68002B02D172B6C046FDE73A688F
:104FB00080235B049A4202D372B6C046FDE73B6A87
:104FC0000433FB61FB690833BB6101F077FBFB69CC
:104FD000DB68FB623B6A1A683B681A433B6A1A60EB
:104FE0003DE0FB6A5B687B61FB6A1B683B610023F9
:104FF0007B623B691B0E1B06FB603B691B021B0AA5
:105000003B61FA688023DB04134007D13B6A1B68CD
:105010003A6913400BD001237B6208E03B6A1B68AE
:105020003A6913403A699A4201D101237B627B6A53
:10503000002B12D0FA6880235B04134003D0BA6AB5
:105040003B691343BB623B6A1B68802292041A438C
:10505000FB6A1100180001F0EFFD7B69FB62FA6A40
:10506000BB699A42BDD13B6A1B68BA6AD2431A40F7
:105070003B6A1A6001F02EFB3B6A1B681800BD46B4
:105080000CB080BD80B584B000AF78607B68FB60F9
:10509000FB680433BB6001F011FB10E0BB68DA6809
:1050A000BB6808339A4202D172B6C046FDE7BB68BE
:1050B000DB68802292041100180001F0BDFDBB687E
:1050C0001B68002BEAD1FB681B7F002B03D1FB6818
:1050D000180002F0A1FF01F0FDFAC046BD4604B081
:1050E00080BD80B582B000AF786039603A687B6877
:1050F00011001800FFF74AFFC046BD4602B080BD50
:1051000080B586B000AFF860B9607A6000237B613B
:105110007B68002B06D1FB68BA6813400AD00123D4
:105120007B6107E0FB68BA681340BA689A4201D114
:1051300001237B617B691800BD4606B080BD00007D
:1051400080B586B000AFF860B9607A607B68BA68F5
:10515000F968054802F052FD03007B617B69180085
:10516000BD4606B080BDC046E350010880B582B0A0
:1051700000AF78607B6808331A007B685A607B68F0
:10518000012252429A607B6808331A007B68DA6019
:105190007B6808331A007B681A617B6800221A60FA
:1051A000C046BD4602B080BD80B582B000AF786019
:1051B0007B6800221A61C046BD4602B080BD80B542
:1051C00084B000AF786039607B685B68FB603B68E7
:1051D000FA685A60FB689A683B689A60FB689B684B
:1051E0003A685A60FB683A689A603B687A681A6164
:1051F0007B681B685A1C7B681A60C046BD4604B0B9
:1052000080BD80B584B000AF786039603B681B68B2
:10521000BB60BB68013303D17B681B69FB600CE09A
:105220007B680833FB6002E0FB685B68FB60FB683F
:105230005B681B68BA689A42F6D2FB685A683B689A
:105240005A603B685B683A689A603B68FA689A60A3
:10525000FB683A685A603B687A681A617B681B6829
:105260005A1C7B681A60C046BD4604B080BD80B53C
:1052700084B000AF78607B681B69FB607B685B680B
:105280007A6892689A607B689B687A6852685A600C
:10529000FB685B687A689A4203D17B689A68FB680E
:1052A0005A607B6800221A61FB681B685A1EFB6803
:1052B0001A60FB681B681800BD4604B080BD80B54D
:1052C00084B000AF786039607B68FB60FB68002BBE
:1052D00002D172B6C046FDE702F052FDFB681A68C3
:1052E000FB68D96BFB681B6C4B43D218FB689A6058
:1052F000FB6800229A63FB681A68FB685A60FB68C7
:105300001A68FB68DB6B591EFB681B6C4B43D21899
:10531000FB68DA60FB684422FF219954FB68452250
:10532000FF2199543B68002B0DD1FB681B69002BB2
:1053300013D0FB681033180001F020FC031E0CD0C2
:1053400002F00EFD09E0FB6810331800FFF70EFFB6
:10535000FB6824331800FFF709FF02F023FD012347
:105360001800BD4604B080BD90B589B002AFF860AA
:10537000B9607A603B60FB68002B02D172B6C04610
:10538000FDE73B68002B02D172B6C046FDE77B68A3
:10539000002B02D0BB68002B01D0012300E00023CA
:1053A000002B02D172B6C046FDE77B68002B02D10C
:1053B000BB68002B01D1012300E00023002B02D1A8
:1053C00072B6C046FDE750233B613B69502B02D0CB
:1053D00072B6C046FDE73B693B687B617B69002B89
:1053E0000ED07B694622012199542823FB181C7892
:1053F0007A68B968F8687B690093230000F038F890
:105400007B691800BD4607B090BD90B58BB002AF68
:10541000F860B960FB1D1A70FB68002B02D172B6F0
:10542000C046FDE7FB68BA685343FB61FB69503334
:10543000180002F03DFD0300BB61BB69002B12D0D8
:10544000BB697B617B6950337B61BB69462200216C
:105450009954FB1D1C787A69B968F868BB69009398
:10546000230000F005F8BB691800BD4609B090BDE7
:1054700080B584B000AFF860B9607A601A00FB1C98
:105480001A70BB68002B03D1BB69BA691A6002E0CD
:10549000BB697A681A60BB69FA68DA63BB69BA6883
:1054A0001A64BB6901211800FFF709FFBB69FA1CE8
:1054B0004C2112785A54C046BD4604B080BD80B518
:1054C00082B000AF78607B68002B0ED07B68002232
:1054D0009A607B6800221A607B680022DA60786834
:1054E00000230022002100F0EAF8C046BD4602B0C9
:1054F00080BD80B586B000AF0200FB1D1A7001238D
:105500007B6100233B61FB1D1A7839697B691800B8
:10551000FFF77BFF0300FB60FB681800FFF7CFFF7E
:10552000FB681800BD4606B080BD80B588B002AFEC
:1055300002003960FB1D1A7001237B6100233B616F
:105540003A6839697869FB1D1B78009313000022C3
:10555000FFF70AFF0300FB60FB681800FFF7AFFFCF
:10556000FB681800BD4606B080BD90B585B000AFA1
:1055700078607B68BB60BB68002B02D172B6C04606
:10558000FDE7BB689C6801F0EBFC03009C4211D175
:10559000BB68DB685A1EBB68DA60BB68DB68002B3F
:1055A00005D1B86800230022002100F088F801230B
:1055B000FB6001E00023FB60FB681800BD4605B0FE
:1055C00090BD90B585B000AF786039607B68BB60F6
:1055D000BB68002B02D172B6C046FDE7BB689C6871
:1055E00001F0BEFC03009C4207D1BB68DB685A1C7B
:1055F000BB68DA600123FB600FE03A68BB6811000A
:10560000180000F0BBFA0300FB60FB68002B04D01D
:10561000BB68DB685A1CBB68DA60FB681800BD46D3
:1056200005B090BD80B588B002AFF860B9607A600F
:10563000FB68002B02D172B6C046FDE7BA68FB6872
:105640009A4202D972B6C046FDE77B68F86802222A
:10565000009200220021FFF787FE03007B617B6937
:10566000002B02D07B69BA689A637B691800BD463B
:1056700006B080BD80B584B000AF786039607B68CB
:10568000002B02D172B6C046FDE73A687B689A42A9
:1056900002D972B6C046FDE77B68022200211800DD
:1056A000FFF7B3FE0300FB60FB68002B02D0FB6832
:1056B0003A689A63FB681800BD4604B080BD80B5A7
:1056C0008AB000AFF860B9607A603B6000237B620B
:1056D000FB683B623B6A002B02D172B6C046FDE715
:1056E000BB68002B03D13B6A1B6C002B01D101234B
:1056F00000E00023002B02D172B6C046FDE73B68F4
:10570000022B03D13B6ADB6B012B01D1012300E0AB
:105710000023002B02D172B6C046FDE701F02EFC3B
:10572000031E02D17B68002B01D1012300E000237E
:10573000002B02D172B6C046FDE702F021FB3B6AA6
:105740009A6B3B6ADB6B9A4202D33B68022B1ED1F9
:105750003A68B9683B6A180000F086FB0300FB61F9
:105760003B6A5B6A002B09D03B6A2433180001F0C6
:1057700005FA031E07D002F0F3FA04E0FB69002BE0
:1057800001D002F0EDFA02F00DFB01235BE07B6833
:10579000002B03D102F006FB002354E07B6A002BB0
:1057A00006D11423FB18180001F09AFA01237B623A
:1057B00002F0F8FA00F082FF02F0E2FA3B6A4422BB
:1057C0009B5C5BB2013303D13B6A442200219954B4
:1057D0003B6A45229B5C5BB2013303D13B6A4522A5
:1057E0000021995402F0DEFA3A1D1423FB1811002F
:1057F000180001F089FA031E1ED13B6A180000F060
:1058000038FC031E11D03B6A10337A68110018006F
:1058100001F03CF93B6A180000F0B7FB00F05AFFBA
:10582000031E8AD102F09CFA87E73B6A180000F059
:10583000ACFB00F04FFF80E73B6A180000F0A5FBCF
:1058400000F048FF00231800BD460AB080BD90B5A7
:105850008BB000AFF860B9607A603B60FB683B6278
:105860003B6A002B02D172B6C046FDE7BB68002B35
:1058700003D13B6A1B6C002B01D1012300E0002304
:10588000002B02D172B6C046FDE73B68022B03D164
:105890003B6ADB6B012B01D1012300E00023002BCD
:1058A00002D172B6C046FDE702F094FA0300FB6134
:1058B0003B6A9A6B3B6ADB6B9A4202D33B68022BD2
:1058C00031D11B243B193A6A4521525C1A703B6A5C
:1058D0009B6B7B613A68B9683B6A180000F0C4FAB8
:1058E0003B191B785BB2013311D13B6A5B6A002B19
:1058F00016D03B6A2433180001F040F9031E0FD084
:105900007B68002B0CD07B6801221A6008E01B2307
:10591000FB181B780133DBB259B23B6A452299541C
:1059200001237B6201E000237B62FB69180002F027
:1059300057FA7B6A1800BD460BB090BD80B588B0A1
:1059400000AF786039607B68BB61BB69002B02D116
:1059500072B6C046FDE7BB691B6C002B02D072B665
:10596000C046FDE7BB691B68002B03D1BB699B6880
:10597000002B01D1012300E00023002B02D172B6DD
:10598000C046FDE702F026FA03007B61BB699B6B12
:105990003B61BB69DB6B3A699A422CD20F203B1802
:1059A000BA694521525C1A703B695A1CBB699A63FB
:1059B0003B181B785BB2013311D1BB695B6A002BCA
:1059C00016D0BB692433180001F0D8F8031E0FD09D
:1059D0003B68002B0CD03B6801221A6008E00F23C3
:1059E000FB181B780133DBB259B2BB6945229954CD
:1059F0000123FB6101E00023FB617B69180002F0D9
:105A0000EFF9FB691800BD4608B080BD80B58AB0CB
:105A100000AFF860B9607A6000237B62FB683B628C
:105A20003B6A002B02D172B6C046FDE7BB68002B73
:105A300003D13B6A1B6C002B01D1012300E0002342
:105A4000002B02D172B6C046FDE701F097FA031EA3
:105A500002D17B68002B01D1012300E00023002B41
:105A600002D172B6C046FDE702F08AF93B6A9B6B31
:105A7000FB61FB69002B1AD0BA683B6A1100180061
:105A800000F05DFAFB695A1E3B6A9A633B6A1B6928
:105A9000002B08D03B6A1033180001F06FF8031E8A
:105AA00001D002F05DF902F07DF9012362E07B682C
:105AB000002B03D102F076F900235BE07B6A002B18
:105AC00006D11423FB18180001F00AF901237B62A8
:105AD00002F068F900F0F2FD02F052F93B6A44224C
:105AE0009B5C5BB2013303D13B6A44220021995491
:105AF0003B6A45229B5C5BB2013303D13B6A452282
:105B00000021995402F04EF93A1D1423FB1811009C
:105B1000180001F0F9F8031E1ED13B6A180000F0CE
:105B200092FA031E11D03B6A24337A6811001800E0
:105B300000F0ACFF3B6A180000F027FA00F0CAFD45
:105B4000031E91D102F00CF98EE73B6A180000F0B9
:105B50001CFA00F0BFFD87E73B6A180000F015FA59
:105B600000F0B8FD3B6A180000F06DFA031E00D18A
:105B70007AE700231800BD460AB080BD80B58AB020
:105B800000AF7860396000237B627B68FB61002393
:105B90003B62FB69002B02D172B6C046FDE7FB6990
:105BA0001B6C002B02D072B6C046FDE701F0E6F98F
:105BB000031E02D13B68002B01D1012300E000232A
:105BC000002B02D172B6C046FDE702F0D9F8FB699E
:105BD0009B6BBB61BB69002B1DD0BB695A1EFB6967
:105BE0009A63FB691B68002B04D101F031FB0200B2
:105BF000FB699A60FB691B69002B08D0FB691033B5
:105C0000180000F0BBFF031E01D002F0A9F802F05B
:105C1000C9F801238CE03B68002B09D13B6A002BBB
:105C200002D072B6C046FDE702F0BCF800237FE068
:105C30007B6A002B06D10C23FB18180001F050F8EA
:105C400001237B6202F0AEF800F038FD02F098F814
:105C5000FB6944229B5C5BB2013303D1FB694422A4
:105C600000219954FB6945229B5C5BB2013303D14F
:105C7000FB6945220021995402F094F83A000C2364
:105C8000FB181100180001F03FF8031E2ED1FB692C
:105C9000180000F0D8F9031E21D0FB691B68002B07
:105CA0000AD102F06DF8FB699B68180001F082F9D7
:105CB00003003B6202F076F8FB6924333A68110076
:105CC000180000F0E3FEFB69180000F05EF900F038
:105CD00001FD031E00D078E702F042F875E7FB698A
:105CE000180000F052F900F0F5FC6EE7FB691800AF
:105CF00000F04BF900F0EEFCFB69180000F0A3F98E
:105D0000031E00D161E73B6A002B10D002F038F887
:105D1000FB69180000F092F803007B61FB699B6847
:105D20007A691100180001F00BFA02F03BF8002329
:105D30001800BD460AB080BD90B58BB000AFF860CA
:105D4000B9607A60FB683B623B6A002B02D172B695
:105D5000C046FDE7BB68002B03D13B6A1B6C002BE0
:105D600001D1012300E00023002B02D172B6C0460E
:105D7000FDE702F02FF80300FB613B6A9B6BBB6100
:105D8000BB69002B32D017243B193A6A4421525C7C
:105D90001A70BA683B6A1100180000F0D0F8BB69AD
:105DA0005A1E3B6A9A633B191B785BB2013311D1CF
:105DB0003B6A1B69002B16D03B6A1033180000F0B9
:105DC000DDFE031E0FD07B68002B0CD07B68012208
:105DD0001A6008E01723FB181B780133DBB259B2B5
:105DE0003B6A4422995401237B6201E000237B62D9
:105DF000FB69180001F0F4FF7B6A1800BD460BB088
:105E000090BD80B584B000AF78607B68FB60FB68B4
:105E1000002B02D172B6C046FDE7FB68180000F007
:105E200069F9FB6846229B5C002B03D1FB681800D4
:105E300002F0F2F8C046BD4604B080BD80B584B023
:105E400000AF78607B685B6A002B06D07B681B6BB9
:105E50001B683822D31AFB6001E00023FB60FB685B
:105E60001800BD4604B080BD80B586B000AFF860B4
:105E7000B9607A6000237B61FB689B6B3B61FB68C8
:105E80001B6C002B0ED1FB681B68002B4ED1FB68EE
:105E90009B68180001F0F6F803007B61FB680022A4
:105EA0009A6043E07B68002B19D1FB685868FB6857
:105EB0001A6CBB6819001AF0ADFAFB685A68FB68E7
:105EC0001B6CD218FB685A60FB685A68FB689B68B9
:105ED0009A422BD3FB681A68FB685A6026E0FB687D
:105EE000D868FB681A6CBB6819001AF093FAFB6853
:105EF000DA68FB681B6C5B42D218FB68DA60FB68EF
:105F0000DA68FB681B689A4207D2FB689A68FB68EC
:105F10001B6C5B42D218FB68DA607B68022B05D1F0
:105F20003B69002B02D03B69013B3B613B695A1C3A
:105F3000FB689A637B691800BD4606B080BD80B5DA
:105F400082B000AF786039607B681B6C002B18D082
:105F50007B68DA687B681B6CD2187B68DA607B68C8
:105F6000DA687B689B689A4203D37B681A687B680F
:105F7000DA607B68D9687B681A6C3B6818001AF095
:105F800049FAC046BD4602B080BD80B584B000AFBE
:105F9000786001F0F5FE0F23FB187A684521525C0A
:105FA0001A7013E07B685B6A002B16D07B68243381
:105FB000180000F0E3FD031E01D000F0F7FE0F21F2
:105FC0007B181B78013BDAB27B181A700F23FB1881
:105FD0001B785BB2002BE5DC00E0C0467B68452205
:105FE000FF21995401F0DEFE01F0CAFE0E23FB18DA
:105FF0007A684421525C1A7013E07B681B69002B9D
:1060000016D07B681033180000F0B8FD031E01D0D5
:1060100000F0CCFE0E217B181B78013BDAB27B1816
:106020001A700E23FB181B785BB2002BE5DC00E036
:10603000C0467B684422FF21995401F0B3FEC0465C
:10604000BD4604B080BD80B584B000AF786001F07B
:1060500097FE7B689B6B002B02D10123FB6001E064
:106060000023FB6001F09EFEFB681800BD4604B0F3
:1060700080BD80B584B000AF786001F081FE7B68A0
:106080009A6B7B68DB6B9A4202D10123FB6001E0D3
:106090000023FB6001F086FEFB681800BD4604B0DB
:1060A00080BD000080B584B000AF78603960002307
:1060B000FB6015E00E4BFA68D200D358002B0CD1D0
:1060C0000B4BFA68D2003968D150094AFB68DB00F3
:1060D000D31804337A681A6006E0FB680133FB606A
:1060E000FB68072BE6D9C046C046BD4604B080BD5C
:1060F000D80A002080B584B000AF78600023FB6030
:1061000018E0104AFB68DB00D31804331B687A6878
:106110009A420CD10B4BFA68D2000021D150094AA7
:10612000FB68DB00D318043300221A6006E0FB682A
:106130000133FB60FB68072BE3D9C046C046BD4670
:1061400004B080BDD80A002080B586B000AFF860EA
:10615000B9607A60FB687B6101F012FE7B694422C2
:106160009B5C5BB2013303D17B69442200219954CB
:106170007B6945229B5C5BB2013303D17B6945227D
:106180000021995401F00EFE7B699B6B002B06D118
:106190007B6924337A68B968180000F0C7FC7B6912
:1061A0001800FFF7F2FEC046BD4606B080BD90B5B0
:1061B0008DB004AFF860B9607A603B607B6B002BF8
:1061C00002D172B6C046FDE7BB6B002B02D172B69E
:1061D000C046FDE7A8237B617B69A82B02D072B67D
:1061E000C046FDE77B69BB6B002B20D07B6B002B8F
:1061F0001DD0BB6BFB61FB697A6B1A63FB69A5223F
:10620000022199543C687A68B968F86800230393BE
:10621000FB6902931823FB1801933B6B0093230047
:1062200000F058F8FB69180000F0F6F801E00023D0
:10623000BB61BB691800BD4609B090BD90B58DB07B
:1062400004AFF860B9603B60BB1D1A80BB1D1B88A2
:106250009B00180001F02CFE03007B617B69002B82
:1062600010D0A82001F024FE0300FB61FB69002B85
:1062700003D0FB697A691A6306E07B69180001F0B4
:10628000CBFE01E00023FB61FB69002B1AD0FB6908
:10629000A52200219954BB1D1A883C68B968F8688A
:1062A00000230393FB6902937B6B01933B6B009389
:1062B000230000F00FF8FB69180000F0ADF801238F
:1062C000BB6102E001235B42BB61BB691800BD46B4
:1062D00009B090BD80B586B000AFF860B9607A6053
:1062E0003B60BB6A186B7B689B001A00A52119F004
:1062F00041FFBB6A1A6B7B6843498C4663449B0031
:10630000D3183B613B69072293433B613B690722FA
:10631000134002D072B6C046FDE7BB68002B20D008
:1063200000237B6113E0BA687B69D3181878BA6AD6
:1063300034217B69D3185B18021C1A70BA687B6918
:10634000D3181B78002B06D07B6901337B617B69F6
:106350000F2BE8D900E0C046BB6A432200219954C4
:1063600003E0BB6A3422002199543B6A372B01D9E0
:1063700037233B62BB6A3A6ADA62BB6A3A6ADA641A
:10638000BB6A00221A65BB6A04331800FEF70CFFD3
:10639000BB6A18331800FEF707FFBB6ABA6A1A61B6
:1063A0003B6A3822D21ABB6A9A61BB6ABA6A5A62DD
:1063B000BB6AA02200219950BB6AA42200219954F3
:1063C000BB6A54334C220021180019F0D3FEBB6A7B
:1063D0000E4A9A65BB6A0E4ADA65BB6A0D4A1A66AE
:1063E0003A68F9683B69180001F02EFC0200BB6AAC
:1063F0001A607B6A002B02D07B6ABA6A1A60C046B8
:10640000BD4606B080BDC046FFFFFF3F48AB012040
:10641000B0AB012018AC012080B582B000AF78602D
:1064200001F0AEFC2A4B1B685A1C294B1A60294B01
:106430001B68002B09D1274B7A681A60244B1B6814
:10644000012B10D100F0CEFC0DE0234B1B68002B7C
:1064500009D1204B1B68DA6A7B68DB6A9A4202D852
:106460001C4B7A681A601D4B1B685A1C1B4B1A6028
:106470001A4B1A687B685A647B68DA6A184B1B6887
:106480009A4203D97B68DA6A154B1A607B68DA6A2C
:1064900013009B009B189B00124A9A187B680433D8
:1064A00019001000FEF78BFE01F07CFC0A4B1B6804
:1064B000002B08D0074B1B68DA6A7B68DB6A9A42BC
:1064C00001D201F04DFCC046BD4602B080BDC046C1
:1064D000EC0F0020180B0020F80F002008100020FF
:1064E000F40F00201C0B002080B584B000AF786052
:1064F00001F046FC7B68002B02D1264B1B6800E0B4
:106500007B68FB60FB6804331800FEF7B0FEFB6895
:106510009B6A002B04D0FB6818331800FEF7A7FE17
:106520001D4B1B685A1C1C4B1A601A4B1B68FA68DF
:106530009A420CD1FB681A1D184B11001800FEF787
:106540003EFE174B1B685A1C154B1A600AE0154B90
:106550001B685A1E134B1A60FB68180000F0B4FC4D
:1065600000F0E0FC01F01EFC0F4B1B68002B0DD06F
:10657000084B1B68FA689A4208D10C4B1B68002B29
:1065800002D072B6C046FDE701F0EAFBC046BD4648
:1065900004B080BD180B002008100020C00F0020A0
:1065A000D40F0020EC0F0020F80F00201410002062
:1065B00080B584B000AF78600023FB607B68002B5F
:1065C00011D00D4B1B68002B02D072B6C046FDE700
:1065D00000F074F87B680021180000F02FFF00F035
:1065E00079F80300FB60FB68002B01D101F0B8FBD8
:1065F000C046BD4604B080BD1410002090B589B0DF
:1066000004AF0023BB6000237B603A00391D0823E0
:10661000FB18180002F02EFA3C687B68BA681F4924
:106620001F48029201930023009300232200FFF7EA
:10663000BEFD02001B4B1A601A4B1B68002B02D0D8
:106640000123FB6001E00023FB60FB68012B03D109
:1066500000F048FF0300FB60FB68012B13D172B60A
:10666000114B1B6854331A00104B1A60104B012257
:1066700052421A600F4B01221A600F4B00221A601F
:1066800001F04AFB05E0FB68013302D172B6C04657
:10669000FDE7C046BD4605B090BDC046E82B0308E7
:1066A000C16D010810100020180B0020B40200205A
:1066B0000C100020F80F0020F00F002080B500AF74
:1066C000034B1B685A1C024B1A60C046BD4680BD76
:1066D0001410002080B584B000AF0023FB600023BD
:1066E000BB603A4B1B68002B02D172B6C046FDE777
:1066F00001F046FB354B1B685A1E344B1A60334B76
:106700001B68002B5BD1324B1B68002B57D02FE04E
:10671000304BDB68DB68FB60FB6818331800FEF762
:10672000A6FDFB6804331800FEF7A1FDFB68DA6ADA
:10673000294B1B689A4203D9FB68DA6A264B1A6018
:10674000FB68DA6A13009B009B189B00234A9A1887
:10675000FB68043319001000FEF731FDFB68DA6AAC
:106760001F4B1B68DB6A9A4202D31E4B01221A6040
:10677000184B1B68002BCBD1FB68002B01D000F01D
:10678000D1FB194B1B687B607B68002B0FD000F09E
:106790004BF8031E02D0134B01221A607B68013BA9
:1067A0007B607B68002BF2D10F4B00221A600D4BEF
:1067B0001B68002B03D00123BB6001F0D1FA01F06C
:1067C000F1FABB681800BD4604B080BD141000206B
:1067D000EC0F0020AC0F0020F40F00201C0B002059
:1067E000180B002000100020FC0F002080B582B0A4
:1067F00000AF044B1B687B607B681800BD4602B08D
:1068000080BDC046F00F002080B582B000AF0023ED
:106810007B60044B1B683B603B681800BD4602B0C0
:1068200080BDC046F00F002080B586B000AF0023C9
:106830007B614A4B1B68002B00D085E0484B1B68EE
:1068400001333B61464B3A691A603B69002B18D112
:10685000444B1B681B68002B02D072B6C046FDE794
:10686000404B1B68FB60404B1A683E4B1A603E4B26
:10687000FA681A603D4B1B685A1C3C4B1A6000F0CA
:1068800051FB3B4B1B683A699A4249D3354B1B6815
:106890001B68002B04D1364B012252421A603FE0A4
:1068A000304B1B68DB68DB68BB60BB685B687B6088
:1068B0003A697B689A4203D22D4B7A681A602FE0BE
:1068C000BB6804331800FEF7D2FCBB689B6A002B40
:1068D00004D0BB6818331800FEF7C9FCBB68DA6A3D
:1068E000244B1B689A4203D9BB68DA6A214B1A60B1
:1068F000BB68DA6A13009B009B189B001E4A9A181B
:10690000BB68043319001000FEF759FCBB68DA6A53
:106910001A4B1B68DB6A9A42B8D301237B61B5E747
:10692000164B1B68DA6A144913009B009B189B00E6
:106930005B58012B01D901237B61114B1B68002B94
:1069400007D001237B6104E00E4B1B685A1C0D4BE2
:106950001A607B691800BD4606B080BD1410002087
:10696000F00F0020A40F0020A80F0020041000202A
:106970000C100020F40F00201C0B0020180B00202E
:1069800000100020FC0F002080B584B000AF384B11
:106990001B68002B03D0374B01221A6064E0354B93
:1069A00000221A60344B1B681B6BBB60334B7B604F
:1069B000BB681B687A689A4211D1BB6804331B68B4
:1069C0007A689A420BD1BB6808331B687A689A428E
:1069D00005D1BB680C331B687A689A4208D0264BF5
:1069E0001A68254B1B68343319001000FCF736FD7C
:1069F000234B1B68FB6008E0FB68002B02D172B6DA
:106A0000C046FDE7FB68013BFB601E49FA681300C6
:106A10009B009B189B005B58002BEDD0FA6813007D
:106A20009B009B189B00174A9B183B603B685B6868
:106A30005A683B685A603B685A683B6808339A4218
:106A400004D13B685B685A683B685A603B685B6886
:106A5000DA68094B1A600A4BFA681A60064B1B6821
:106A600054331A00084B1A60C046BD4604B080BDBE
:106A70001410002000100020180B0020A5A5A5A5CB
:106A8000F40F00201C0B0020B402002080B582B05F
:106A900000AF786039607B68002B02D172B6C046C7
:106AA000FDE7094B1B6818331A007B6811001800BA
:106AB000FEF7A7FB3B680121180000F0BFFCC046B1
:106AC000BD4602B080BDC046180B002080B584B022
:106AD00000AFF860B9607A60FB68002B02D172B633
:106AE000C046FDE70F4B1B68002B02D172B6C046B3
:106AF000FDE70D4B1B68BA68802109060A439A61BD
:106B0000094B1B6818331A00FB6811001800FEF7C8
:106B100056FB7B680121180000F090FCC046BD4682
:106B200004B080BD14100020180B002080B584B084
:106B300000AFF860B9607A60FB68002B02D172B6D2
:106B4000C046FDE70C4B1B6818331A00FB681100A8
:106B50001800FEF734FB7B68002B02D001235B4258
:106B6000BB607A68BB681100180000F067FCC04683
:106B7000BD4604B080BDC046180B002080B584B06F
:106B800000AF78607B68DB68DB68BB60BB68002BAC
:106B900002D172B6C046FDE7BB6818331800FEF795
:106BA00066FB1F4B1B68002B1DD1BB68043318000C
:106BB000FEF75DFBBB68DA6A1A4B1B689A4203D981
:106BC000BB68DA6A174B1A60BB68DA6A13009B006D
:106BD0009B189B00144A9A18BB68043319001000D4
:106BE000FEF7EDFA07E0BB6818331A000F4B1100EF
:106BF0001800FEF7E4FABB68DA6A0D4B1B68DB6A23
:106C00009A4205D90123FB600A4B01221A6001E078
:106C10000023FB60FB681800BD4604B080BDC04681
:106C200014100020F40F00201C0B0020AC0F0020DB
:106C3000180B00200010002080B584B000AF7860F1
:106C40003960224B1B68002B02D172B6C046FDE7AB
:106C50003B68802212061A437B681A607B68DB68F7
:106C6000FB60FB68002B02D172B6C046FDE77B6873
:106C70001800FEF7FCFAFB6804331800FEF7F7FA79
:106C8000FB68DA6A124B1B689A4203D9FB68DA6A1E
:106C90000F4B1A60FB68DA6A13009B009B189B007D
:106CA0000C4A9A18FB68043319001000FEF787FAA3
:106CB000FB68DA6A084B1B68DB6A9A4202D9074B09
:106CC00001221A60C046BD4604B080BD14100020E9
:106CD000F40F00201C0B0020180B002000100020D7
:106CE00080B582B000AF7860054B1A687B681A6087
:106CF000044B1A687B685A60C046BD4602B080BD2E
:106D000004100020F00F002080B586B000AF78603E
:106D100039607B68002B02D172B6C046FDE73B6844
:106D2000002B02D172B6C046FDE701F029F81D4BD9
:106D30001B683B617B685B683A69D31AFB603B6800
:106D40001B68013302D100237B6124E07B681A6851
:106D5000154B1B689A4207D07B685B683A699A4278
:106D600002D301237B6116E03B681B68FA689A42F4
:106D70000CD23B681A68FB68D21A3B681A607B68C1
:106D80001800FFF7ADFF00237B6104E03B680022A1
:106D90001A6001237B6101F005F87B691800BD468C
:106DA00006B080BDF00F00200410002080B500AFB9
:106DB000024B01221A60C046BD4680BD0010002073
:106DC00080B582B000AF786000F050F8044B1B68CB
:106DD000012B01D900F0C4FFFCF734FBF4E7C046F7
:106DE0001C0B002080B582B000AF00237B600CE05C
:106DF0007A6813009B009B189B00144A9B1818008C
:106E0000FEF7B4F97B6801337B607B68372BEFD9E1
:106E10000F4B1800FEF7AAF90E4B1800FEF7A6F963
:106E20000D4B1800FEF7A2F90C4B1800FEF79EF967
:106E30000B4B1800FEF79AF90A4B054A1A600A4BE9
:106E4000044A1A60C046BD4602B080BD1C0B00203B
:106E50007C0F0020900F0020AC0F0020C00F0020FE
:106E6000D80F0020A40F0020A80F002080B582B00A
:106E700000AF1AE000F084FF104BDB68DB687B603A
:106E80007B6804331800FEF7F2F90D4B1B685A1E9D
:106E90000B4B1A600B4B1B685A1E0A4B1A6000F012
:106EA00081FF7B68180000F00FF8064B1B68002B71
:106EB000E0D1C046C046BD4602B080BDC00F002034
:106EC000EC0F0020D40F002080B582B000AF7860B6
:106ED0007B685433180019F0A5F97B68A5229B5CE8
:106EE000002B09D17B681B6B180001F095F87B68BB
:106EF000180001F091F811E07B68A5229B5C012B42
:106F000004D17B68180001F087F807E07B68A522B0
:106F10009B5C022B02D072B6C046FDE7C046BD4660
:106F200002B080BD80B582B000AF0B4B1B681B6800
:106F3000002B04D1094B012252421A6008E0064B93
:106F40001B68DB68DB687B607B685A68034B1A60F0
:106F5000C046BD4602B080BDA40F00200C1000202A
:106F600080B582B000AF044B1B687B607B68180063
:106F7000BD4602B080BDC046180B002080B582B06F
:106F800000AF0A4B1B68002B02D101237B6008E095
:106F9000074B1B68002B02D102237B6001E000231A
:106FA0007B607B681800BD4602B080BDF80F0020F2
:106FB0001410002080B584B000AF78607B68BB609F
:106FC0000023FB607B68002B51D0BB68DA6A2A4B38
:106FD0001B68DB6A9A4241D2BB689B69002B06DBC7
:106FE000254B1B68DB6A3822D21ABB689A61BB68E2
:106FF0005969BB68DA6A13009B009B189B001F4A03
:107000009B18994222D1BB6804331800FEF72FF970
:10701000194B1B68DA6ABB68DA62BB68DA6A184B1C
:107020001B689A4203D9BB68DA6A154B1A60BB68C1
:10703000DA6A13009B009B189B00104A9A18BB68E1
:10704000043319001000FEF7BAF804E00A4B1B687D
:10705000DA6ABB68DA620123FB6008E0BB68DA6CBD
:10706000054B1B68DB6A9A4201D20123FB60FB6877
:107070001800BD4604B080BD180B00201C0B00207A
:10708000F40F002080B584B000AF78607B68BB60EF
:107090000023FB607B68002B46D0264B1B68BA6838
:1070A0009A4202D072B6C046FDE7BB681B6D002B4A
:1070B00002D172B6C046FDE7BB681B6D5A1EBB68A5
:1070C0001A65BB68DA6ABB68DB6C9A422CD0BB6875
:1070D0001B6D002B28D1BB6804331800FEF7C7F8DE
:1070E000BB68DA6CBB68DA62BB68DB6A3822D21A2A
:1070F000BB689A61BB68DA6A0F4B1B689A4203D976
:10710000BB68DA6A0C4B1A60BB68DA6A13009B0032
:107110009B189B00094A9A18BB6804331900100099
:10712000FEF74DF80123FB60FB681800BD4604B074
:1071300080BDC046180B0020F40F00201C0B00205F
:1071400080B586B000AF786039607B683B61012311
:10715000FB607B68002B5AD03B691B6D002B02D172
:1071600072B6C046FDE73B69DB6C3A689A4202D9C9
:107170003B687B6102E03B69DB6C7B613B69DB6AFE
:107180007A699A4243D03B691B6DFA689A423ED1B4
:10719000214B1B683A699A4202D172B6C046FDE79C
:1071A0003B69DB6ABB603B697A69DA623B699B6970
:1071B000002B04DB7B693822D21A3B699A613B6958
:1071C0005969BA6813009B009B189B00134A9B18CF
:1071D00099421CD13B6904331800FEF748F83B691B
:1071E000DA6A0F4B1B689A4203D93B69DA6A0C4B87
:1071F0001A603B69DA6A13009B009B189B00074AE0
:107200009A183B69043319001000FDF7D8FFC046F7
:10721000BD4606B080BDC046180B00201C0B0020E8
:10722000F40F002080B582B000AF084B1B689B694B
:107230007B60064B1B68DA6A044B1B6838218A1A8C
:107240009A617B681800BD4602B080BD180B002013
:1072500080B500AF064B1B68002B04D0044B1B68A5
:107260001A6D01321A65024B1B681800BD4680BDBD
:10727000180B002080B584B000AF7860396000F052
:107280007FFD1E4B1B68A0229B58002B0ED11B4B71
:107290001B68A422012199543B68002B06D03B684F
:1072A0000121180000F0CAF800F05AFD00F07AFD44
:1072B00000F066FD114B1B68A0229B58FB60FB6829
:1072C000002B0ED07B68002B05D00C4B1B68A02236
:1072D0000021995005E0094B1B68FA68013AA0218A
:1072E0005A50064B1B68A4220021995400F05AFD05
:1072F000FB681800BD4604B080BDC046180B0020D6
:1073000080B588B000AFF860B9603B60FB1D1A70B3
:107310000123FB61FB68002B02D172B6C046FDE77A
:10732000FB68BB6100F02CFD3B68002B04D0BB69FF
:10733000A0229A583B681A601723FB18BA69A42147
:10734000525C1A70BB69A42202219954FB1D1B7860
:10735000042B27D89A00354BD3181B689F46BB696E
:10736000A0229A58BB681A43BB69A0215A5024E056
:10737000BB69A0229B585A1CBB69A0215A501CE033
:10738000BB69A021BA685A5017E01723FB181B7875
:10739000022B04D0BB69A021BA685A500DE000232B
:1073A000FB610AE0BB69A0229B58013304D072B68E
:1073B000C046FDE7C04600E0C0461723FB181B7817
:1073C000012B2CD1BB6904331800FDF750FFBB69BA
:1073D000DA6A174B1B689A4203D9BB69DA6A144B05
:1073E0001A60BB69DA6A13009B009B189B00114A64
:1073F0009A18BB69043319001000FDF7E0FEBB6961
:107400009B6A002B02D072B6C046FDE7BB69DA6A00
:10741000094B1B68DB6A9A4201D900F0A1FC00F01D
:10742000C1FCFB691800BD4608B080BD645B030861
:10743000F40F00201C0B0020180B002080B584B036
:1074400000AF78603960214B1B68FB60204B1B68E4
:1074500004331800FDF70BFF7B6801330BD13B6849
:10746000002B08D01A4B1B681A1D1A4B110018006C
:10747000FDF7A5FE26E0FA687B68D318BB60144BC5
:107480001B68BA685A60BA68FB689A4209D2124B04
:107490001A680F4B1B68043319001000FDF7B1FE8A
:1074A00010E00E4B1A680A4B1B68043319001000D9
:1074B000FDF7A7FE0A4B1B68BA689A4202D2084B36
:1074C000BA681A60C046BD4604B080BDF00F002007
:1074D000180B0020D80F0020A80F0020A40F0020B8
:1074E0000C10002090B589B004AF0023FB6000F0C1
:1074F0002BFB184B1B68002B20D00023BB60002304
:107500007B603A00391D0823FB18180001F0CAFA05
:107510003C687B68BA6810491048029201930223C4
:10752000009300232200FEF742FE02000C4B1A607B
:107530000B4B1B68002B01D00123FB60FB68002B69
:1075400002D172B6C046FDE7FB681800BD4605B023
:1075500090BDC04648100020F02B03083577010885
:107560004C10002090B589B002AFF860B9607A6025
:107570003B602C2000F09CFC03007B617B69002BAE
:107580000ED07B692822002199543C687A68B9683A
:10759000F8687B690193BB6A0093230000F005F84B
:1075A0007B691800BD4607B090BD80B584B000AFC0
:1075B000F860B9607A603B60BB68002B02D172B69C
:1075C000C046FDE7FB69002B1ED000F0BDFAFB6949
:1075D000FA681A60FB69BA689A61FB693A68DA610D
:1075E000FB69BA691A62FB6904331800FDF7DCFD18
:1075F0007B68002B08D0FB6928229B5C0422134384
:10760000D9B2FB6928229954C046BD4604B080BD5A
:1076100090B58BB000AFF860B9607A603B60002332
:107620007B62FB68002B02D172B6C046FDE71D4BA2
:107630001B68002B30D014243B19BA681A603B1920
:107640007A685A603B19FA689A60BB68052B19DCA6
:10765000FFF794FC0300022B09D1124B1868BA6B98
:1076600039190023FEF72BF803007B6214E00D4B61
:1076700018681423F91800230022FEF720F80300ED
:107680007B6209E0074B18683A681423F918002355
:10769000FEF7DDF803007B627B6A1800BD460BB085
:1076A00090BDC0464810002080B586B002AF78601B
:1076B00039601F4B1B68DB68DB68FB60FB680433C9
:1076C0001800FDF7D4FDFB6828229B5C1A000423F8
:1076D00013401AD0FB689A697B68D1187B683A68B6
:1076E000F86800F0C7F8031E18D07A68F86800231D
:1076F000009300230021FFF78BFF0300BB60BB68F2
:10770000002B0BD172B6C046FDE7FB6828229B5CBC
:1077100001229343D9B2FB6828229954FB681B6A63
:10772000FA6810009847C046BD4604B080BDC04608
:107730004010002080B584B000AF78600823FB18AB
:10774000180000F055F80300FB60BA68FB681100F0
:10775000180000F005F800F0CFF8C046EEE7000092
:1077600080B584B000AF78603960FEF7A7FF0823CA
:10777000FB18180000F05EF80300FB60BB68002BEC
:107780002BD13B68002B0CD17A68FB689A4208D851
:10779000FEF7A0FFFA687B6811001800FFF784FF6E
:1077A0001DE03B68002B08D00F4B1B681B68002BAB
:1077B00001D1012300E000233B600C4B18687A687C
:1077C000FB68D31A3A681900FEF7BEFCFEF782FF89
:1077D000031E04D100F0C4FA01E0FEF77BFFC046AF
:1077E000BD4604B080BDC0464410002048100020B3
:1077F00080B584B000AF78600D4B1B681B68002B10
:1078000001D1012200E000227B681A607B681B68BE
:10781000002B05D1064B1B68DB681B68FB6001E091
:107820000023FB60FB681800BD4604B080BDC04665
:107830004010002080B584B000AF7860FEF7D6FF1E
:107840000300FB600A4B1B68FA689A4205D200F0FD
:107850001DF97B6801221A6002E07B6800221A6031
:10786000034BFA681A60FB681800BD4604B080BD7F
:107870005010002080B586B000AFF860B9607A6023
:107880003B6000237B61FB68BA685A60FB68FA685A
:107890001A61BA687B689A4212D87A683B68D21A31
:1078A000FB689B699A4202D301237B611BE0104B6A
:1078B0001A68FB68043319001000FDF7A2FC12E0FF
:1078C0007A683B689A4206D2BA683B689A4202D309
:1078D00001237B6107E0074B1A68FB68043319003A
:1078E0001000FDF78EFC7B691800BD4606B080BD18
:1078F000441000204010002090B58DB002AFB1E0E0
:107900000822BB181B68002B10DABB1804337B62FB
:107910007B6A002B02D172B6C046FDE77B6A1A680B
:107920007B6A58687B6A9B68190090470822BB18DD
:107930001B68002B00DA95E0BB189B683B623B6A32
:107940005B69002B04D03B6A04331800FDF78FFC01
:107950003B1D1800FFF76EFF0300FB610823FB18B7
:107960001B68092B00D97AE09A00464BD3181B6894
:107970009F463B6A28229B5C01221343D9B23B6A93
:107980002822995408243B195A683B6A9B69D118EC
:107990003B195B68FA69386AFFF76CFF031E60D019
:1079A0003B6A1B6A3A6A100098473B6A28229B5C34
:1079B0001A000423134054D03B195A683B6A9B6950
:1079C000D218386A0023009300230021FFF720FE1D
:1079D0000300BB61BB69002B43D172B6C046FDE713
:1079E0003B6A28229B5C01229343D9B23B6A28223E
:1079F000995437E03B6A28229B5C01221343D9B299
:107A00003B6A282299540823FB185A683B6A9A61FA
:107A10003B6A9B69002B02D172B6C046FDE73B6A08
:107A20009A69FB69D118FB69FA69386AFFF722FF86
:107A300018E03B6A28229B5C1A000223134004D101
:107A40003B6A180000F0E8FA0CE03B6A28229B5CD5
:107A500001229343D9B23B6A2822995402E0C046DE
:107A600000E0C046084B1B680822B9180022180025
:107A7000FDF7CCFF031E00D042E7C046C046BD461E
:107A80000BB090BD785B03084810002080B588B02B
:107A900002AF42E02A4B1B68DB681B683B61284B46
:107AA0001B68DB68DB68FB60FB6804331800FDF7CC
:107AB000DEFBFB681B6AFA6810009847FB68282207
:107AC0009B5C1A000423134027D0FB689B693A692A
:107AD000D318BB60BA683B699A420ED9FB68BA6892
:107AE0005A60FB68FA681A61154B1A68FB68043320
:107AF00019001000FDF785FB0FE03A69F8680023D4
:107B0000009300230021FFF783FD03007B607B6867
:107B1000002B02D172B6C046FDE7094B1B681B68FB
:107B2000002BB7D1064B1B687B61064B1A68044BD0
:107B30001A60044B7A691A60C046BD4606B080BD23
:107B4000401000204410002080B582B002AF00F049
:107B500017F9164B1B68002B23D1154B1800FDF7A6
:107B600005FB144B1800FDF701FB134B104A1A607C
:107B7000124B104A1A60124B124A00210091102138
:107B80000A20FDF7F1FB0200084B1A60074B1B6847
:107B9000002B06D0054B1B680B4A11001800FEF79E
:107BA00081FA00F0FFF8C046BD4680BD48100020B5
:107BB000181000202C10002040100020441000203D
:107BC000F410002054100020F82B030880B584B076
:107BD00000AF78607B68FB607B68002B02D172B6D7
:107BE000C046FDE700F0CCF8FB68DB69BB6000F045
:107BF000D9F8BB681800BD4604B080BD80B58AB016
:107C000000AFF860B9607A603B6014217B180222F3
:107C100052421A607B18FA685A607B18BA689A60F8
:107C20007B187A68DA60074B18683A68791800237D
:107C3000FDF70DFE03007B627B6A1800BD460AB0AB
:107C400080BDC0464810002080B584B000AFF86009
:107C5000B9607A60FB68043BFB60FB6880225204D9
:107C60001A60FB68043BFB60BA68FB681A60FB683B
:107C7000043BFB60084AFB681A60FB68143BFB602E
:107C80007A68FB681A60FB68203BFB60FB681800A1
:107C9000BD4604B080BDC0469D7C010880B582B061
:107CA00000AF00237B60084B1B68013302D072B623
:107CB000C046FDE772B6C0467B68002BFCD0C046CC
:107CC000C046BD4602B080BD0400002080B500AFB4
:107CD000C046BD4680BD000000000000000000005E
:107CE0000B4A13681868203080F30988022080F35B
:107CF0001488BFF36F8F3FBCAE4608BC04BC62B6AD
:107D00001847C046C046C046C046C046C046C046EA
:107D1000180B0020C046C04680B500AF0E4B1A6855
:107D20000D4BFF2109040A431A600B4B1A680A4BDA
:107D3000FF2109060A431A6000F098F8074B002259
:107D40001A60FFF7CDFFFEF71FFEFFF7A7FF002326
:107D50001800BD4680BDC04620ED00E004000020B4
:107D600080B500AF054B802252051A60BFF34F8FDC
:107D7000BFF36F8FC046BD4680BDC04604ED00E036
:107D800080B500AF72B6064B1B685A1C044B1A60D4
:107D9000BFF34F8FBFF36F8FC046BD4680BDC04657
:107DA0000400002080B500AF094B1B68002B02D1F6
:107DB00072B6C046FDE7064B1B685A1E044B1A609C
:107DC000034B1B68002B00D162B6C046BD4680BD88
:107DD00004000020EFF3108072B67047C046180010
:107DE00080F310887047C0460000000000000000CB
:107DF000EFF309800E4B1A6820381060F0C044463B
:107E00004D4656465F46F0C008B572B6FEF7BCFD5B
:107E100062B60CBC116808681030F0C8A046A946CC
:107E2000B246BB4680F309882038F0C81847C046E0
:107E3000180B0020C046C04680B582B000AFFFF7E7
:107E4000C9FF03007B60FEF7EFFC031E03D0064B67
:107E5000802252051A607B681800FFF7C1FFC046F8
:107E6000BD4602B080BDC04604ED00E080B500AF65
:107E70000B4B00221A600B4B00221A600A4B1B6846
:107E8000FA2291001800F8F765FA03001A00074B70
:107E9000013A1A60024B07221A60C046BD4680BDF7
:107EA00010E000E018E000E00000002014E000E036
:107EB00080B586B000AF78600023FB60FEF7FEFB64
:107EC0004F4B1B68002B01D100F0F6F84D4B1B689F
:107ED0007A68134000D080E07B68002B13D0082222
:107EE0007B689B187B607B68072213400BD07B6804
:107EF0000722934308337B607B680722134002D03C
:107F000072B6C046FDE77B68002B66D03E4B1B680F
:107F10007A689A4261D83D4B3B613C4B1B687B6160
:107F200004E07B693B617B691B687B617B695B6803
:107F30007A689A4203D97B691B68002BF1D1304BD8
:107F40001B687A699A4248D03B691B6808229B18D3
:107F5000FB607B691A683B691A607B695A687B68B9
:107F6000D21A08235B009A4217D97A697B68D31822
:107F7000BB60BB680722134002D072B6C046FDE763
:107F80007B695A687B68D21ABB685A607B697A68D9
:107F90005A60BB68180000F0EFF81B4B1A687B6949
:107FA0005B68D21A184B1A60174B1A68184B1B687B
:107FB0009A4203D2144B1A68154B1A607B695A68AF
:107FC000104B1B681A437B695A607B6900221A6058
:107FD000104B1B685A1C0F4B1A60FEF77BFBFB68AB
:107FE000002B01D1FBF743FAFB680722134002D0B4
:107FF00072B6C046FDE7FB681800BD4606B080BDFE
:108000004C91012060910120509101204491012068
:10801000549101205891012080B584B000AF786060
:108020007B68FB607B68002B3CD008235B42FA68CE
:10803000D318FB60FB68BB60BB685A681B4B1B68AE
:10804000134002D172B6C046FDE7BB681B68002B27
:1080500002D072B6C046FDE7BB685A68134B1B6876
:1080600013401FD0BB681B68002B1BD1BB685A682C
:108070000E4B1B68DB431A40BB685A60FEF71EFBC1
:10808000BB685A680A4B1B68D218094B1A60BB6858
:10809000180000F071F8074B1B685A1C054B1A605A
:1080A000FEF718FBC046BD4604B080BD60910120BC
:1080B000509101205C91012080B584B000AFC023B5
:1080C0005B02BB60264BFB60FB68072213400CD0B1
:1080D000FB680733FB60FB6807229343FB60BA68C9
:1080E000FB68D21A1E4BD318BB60FB687B601D4B2C
:1080F0007A681A601B4B00225A607B68BA68D318F2
:10810000FB600822FB689B1AFB60FB680722934315
